:10000000F8FF022099010000ADF9000069F9000035
:1000100069F9000069F9000069F9000069F9000058
:1000200069F9000069F9000069F90000ADF9000004
:10003000ADF9000069F90000C5190100C9190100F6
:10004000ADF90000ADF90000ADF90000ADF9000018
:10005000ADF90000ADF90000ADF90000ADF9000008
:10006000ADF90000ADF90000ADF90000ADF90000F8
:10007000ADF90000ADF90000ADF90000ADF90000E8
:10008000ADF90000ADF90000ADF90000ADF90000D8
:10009000ADF90000ADF90000ADF90000ADF90000C8
:1000A000ADF90000ADF90000ADF90000ADF90000B8
:1000B000ADF90000ADF90000ADF90000ADF90000A8
:1000C000ADF900003D040100ADF90000850B010011
:1000D000ADF90000ADF90000ADF900002D9200006F
:1000E000ADF90000ADF90000ADF90000ADF9000078
:1000F000ADF90000ADF90000ADF90000ADF9000068
:10010000ADF90000ADF90000ADF90000ADF9000057
:10011000ADF900007D0E0100ADF90000ADF9000061
:10012000ADF90000ADF90000ADF90000ADF9000037
:10013000ADF90000ADF90000ADF90000ADF9000027
:10014000ADF90000ADF90000ADF90000ADF9000017
:10015000ADF90000ADF90000ADF90000ADF9000007
:10016000ADF90000ADF90000ADF90000ADF90000F7
:10017000ADF90000ADF90000ADF90000ADF90000E7
:10018000ADF90000ADF90000ADF90000ADF90000D7
:10019000ADF90000ADF900005A4B4CF2205210B5F9
:1001A000DA814DF62812DA8100BF00BF0FF002FCA1
:1001B000554B4FF030621A63544A9A63544ADA63DB
:1001C0004FF0E0234FF47002C3F8882D514A1369B1
:1001D00013F4807303D153614FF4A85313614E4B52
:1001E0009A78110703D59A7842F008029A704B4B1F
:1001F0004B482A221A704B4BDA1C121AC11E22F0ED
:100200000302994288BF002247490FF0D9FA474BB1
:100210004748DA1C121AC11E22F00302994288BF15
:100220000022002113F094FD424943484FF4CC7260
:100230000FF0C6FA414B424A802103F8011B93425A
:10024000FBD14FF0E0233C4AC3F8082D3D4B8A22F6
:100250001A70A3F5805324225A70A0221A709A793A
:100260009207FCD59A79D406FCD4374B9A7902F0E0
:100270000C02082AFAD103221A7146225A719A797D
:100280009006FCD5304A93795906FCD51E4B4FF0A9
:10029000827159640921996420211170917901F0CA
:1002A0000C010C29FAD1294A5A604FF0E023284A60
:1002B0005A6100229A6107221A61264AC3F8202D4A
:1002C00062B60FF0C7FB134B5B69DA0705D522480E
:1002D0000FF0B4FB214B224ADA61224B1B785B06FC
:1002E00009D51E4C1E4BE2699A4204D11A480FF000
:1002F000A5FB0023E3610FF063FB13F093FD11F006
:10030000DBFCFEE70020054000800440823F040043
:100310000100002B00D0034000D0074000E0074060
:10032000F806FF1F7816FF1FCC9A0100F405002085
:100330007816FF1F000000000002FF1F00E400E02D
:1003400056E400E00050064000400640C0100500A2
:10035000BFD401000000202049C46B6700E00340C7
:10036000A5C3945A00F00740FFFFFFFFFFFFFFFF08
:10037000FFFFFFFFFFFFFFFFFFFFFFFFFFFFFFFF8D
:10038000FFFFFFFFFFFFFFFFFFFFFFFFFFFFFFFF7D
:10039000FFFFFFFFFFFFFFFFFFFFFFFFFFFFFFFF6D
:1003A000FFFFFFFFFFFFFFFFFFFFFFFFFFFFFFFF5D
:1003B000FFFFFFFFFFFFFFFFFFFFFFFFFFFFFFFF4D
:1003C000FFFFFFFFFFFFFFFFFFFFFFFFFFFFFFFF3D
:1003D000FFFFFFFFFFFFFFFFFFFFFFFFFFFFFFFF2D
:1003E000FFFFFFFFFFFFFFFFFFFFFFFFFFFFFFFF1D
:1003F000FFFFFFFFFFFFFFFFFFFFFFFFFFFFFFFF0D
:10040000FFFFFFFFFFFFFFFFFFFFFFFFDEF9FFFF23
:100410000548064B1B1AD90F01EBA301491002D066
:10042000034B03B1184770477816FF1F7816FF1F5C
:100430000000000008B5054B1BB105490548AFF3A6
:100440000080BDE80840FFF7E3BF00BF00000000E8
:100450007816FF1FCC9A01002DE9F04182B00446C6
:100460000025019104F5CC7800F07EFA019904F59D
:10047000987000F0F1FD04F50E7729468C22A4F85F
:100480008C51C4F89051C4F89451404613F060FC6C
:1004900029465022C4F82452A4F8285284F82A523B
:1004A000A4F82C52C4F83052C4F83452384613F031
:1004B0004FFC00264FF48073A4F88832142229469A
:1004C000C4F88C62C4F8906284F8945204F52670E3
:1004D00013F03EFCA4F8AC5284F8AE52C4F8B0520B
:1004E00084F8B4520B2011F0EFFB3023A4F88C31C8
:1004F0000E4BC4F894310E4BC4F824020722204658
:10050000C4F89081A4F82C22C4F83072C4F83432B4
:10051000C4F89862C4F89C62C4F8A062C4F8A462EB
:10052000C4F8A86202B0BDE8F08100BFF806FF1F62
:100530005807FF1FB0F8ACC2BCF1050F10B5044658
:100540003BD0B0F8B032B0F8B2225B08A9B90132A2
:10055000A0F8AC1290F8AE12A0F8B03292B2A0F8A7
:10056000B222002949D194F8B412012918D00229E5
:1005700001D1082A19D0002010BD013290F8AE1226
:1005800043F0800392B20CF1010CA0F8B032A0F855
:10059000B222A0F8ACC219BB94F8B4120129E6D17A
:1005A000082AE8D1022284F8B4221946204600F035
:1005B000E9F90020A4F8B20210BD81B3B0F8B0325E
:1005C000B0F8B2225B08012043F080030244062108
:1005D00084F8AE02A4F8B032A4F8B222A4F8AC12A7
:1005E000FE2B4FF00000C7D1A4F82C0184F8B40210
:1005F00084F8AE02A4F8B20210BD7E2BF0D1B4F89C
:100600002C31102B11D80020A4F82C01002301223A
:1006100084F8B42284F8AE32A4F8B23210BD80F867
:10062000AE12A0F8AC12084610BD00F0B9F90028CF
:10063000ECD1E8E700F5987000F028BDD0EDA47A81
:100640009FED0C7AF4EEC77AF1EE10FA04D801238C
:1006500080F8943218467047B0EE087AF4EEC77A04
:10066000F1EE10FAA9BF002390F8940280F89432BA
:10067000184670479999193FD0EDA65A9FED1A7AFE
:1006800090EDA76AD0EDA86ADFED184ADFED183AC1
:100690009FED185A9FED184A80EDA86AF0EE407A57
:1006A000E5EEC77A9FED157A9FED150AC0EDA75AC2
:1006B000E6EE477A90EDA97AC0EDA96AE6EEE47A13
:1006C000DFED104A80EDAA7AE7EE637AA7EE850A9D
:1006D000C0EDA67AA5EEA40AA6EE040AA6EEA40A28
:1006E000A7EE050A704700BF819231C00E10B8BF57
:1006F000E49D883E3D2C8D3A5DC2D33B23A13D4015
:10070000000000003F2C8D3B10B590F888322DED95
:10071000028B8B4282B0044650D090EDA37A90F8C1
:10072000893280F88812F2EE047AB4EEE77AF1EEBC
:1007300010FA3CDCDFED337AB1EE048A102B98BF5F
:10074000B0EE678A07EE903AF8EE677A0123C7EEBB
:10075000276A04F50B7001AA6946CDED006A12F014
:10076000FDFB9DED000AB5EEC00AF1EE10FA204641
:100770004CBF38EE400A30EE080AFFF77DFFDDED92
:10078000016AD4EDA37A84EDA40AB6EE007AE6EE0F
:10079000C77A012384F889320020B7EE007A77EE19
:1007A000877AC4EDA37A02B0BDEC028B10BDF3EEE4
:1007B000047A37EE677A84EDA37ABBE790F8893242
:1007C000102B0BD990EDA37AF2EE047AB4EEE77A0F
:1007D000F1EE10FAEBDCB1EE048AB3E7D0EDA37AC8
:1007E000B2EE047AF4EEC77AF1EE10FA08DDB3EE59
:1007F000047A013380F8893277EEC77A0120CCE79A
:100800000020CAE7000000002DE9F04784B015463B
:1008100004461F4601AA022300F5987000F034FC3C
:10082000002D69D0D4F824E2B4F8282201A80DF1F3
:10083000080C002630F9021B1EF80280531CC94325
:100840009BB2C90FA4F828320A2B0EF8021006F149
:10085000010381EA08014FEA4101DBB294BFB4F819
:100860002822002201399D422CF8021BA4F82822DC
:1008700001D01E46DEE7022303AA02A904F5C670D2
:1008800090464FF0020912F00FF900250DF10E030A
:1008900019FB0639AA4638F9026BF643F60F2046D3
:1008A0003146FFF731FF58B194F82A1284F82A62D2
:1008B000891BB1FA81F1204649093DB1FFF73AFEA3
:1008C000C145E8D1284604B0BDE8F087FFF732FE05
:1008D00005460028F4D04FF49672214638460EF0B3
:1008E0006FFFB4F82C31A7F82C31B4F82E31A7F8EB
:1008F0002E31A4F82CA1E3E704F5C670022303AA65
:1009000002A912F0D1F8284604B0BDE8F08700BF74
:1009100070B5064615460C464FF49672002113F04A
:1009200017FA0023A6F82C31A6F82E319DB1611ECE
:100930000123741E40F22B1201E093420DD01FFAE6
:1009400083FC11F801EF04F801EF654503F10103A1
:10095000F3D8A6F82CC1304670BD4FF49573A6F8B5
:100960002C31304670BD00BF10B54FF4967204466E
:10097000002113F0EDF90023A4F82C31A4F82E3156
:10098000204610BDB0F82C21B2F5967F034605D065
:10099000501CA3F82C019954012070470020704787
:1009A00030B5B0F82C51B5F1020E24D0FF23144C11
:1009B0009C46002202E04FEA132CDBB2815C4B40E4
:1009C000013234F8133092B272458CEA0303F2D349
:1009D000DB4399B2DBB210F80E209A4205D10544F0
:1009E00015F8013CB3EB112F01D0002030BDA0F869
:1009F0002E11012030BD734671460225EBE700BF82
:100A0000D842010030B5B0F82C412CB304F1FF3EC0
:100A1000FF23174D421E10FA8EFE9C4602E04FEA5D
:100A2000132CDBB212F8011F4B40964535F81330FA
:100A30008CEA0303F3D1621CDB43A11C92B21FFAC0
:100A400083FCDDB289B2C3F30723A0F82EC105559C
:100A5000A0F82C11835430BD0122A4460221234664
:100A60002546A0F82EC10555A0F82C11835430BDA1
:100A7000D842010070B5002500F10C0604464FF481
:100A8000A0722946058045608560304613F060F904
:100A9000032104F5A670FFF7DFFC062104F20440F1
:100AA000FFF7DAFC092104F2BC60FFF7D5FC8223D2
:100AB0000C4A23801E230C49A260C4F87C394BF2F7
:100AC00040320F23C4F88419A4F8882984F88A399D
:100AD000A4F874596660C4F87859C4F8805920465F
:100AE00070BD00BF7407FF1F80000001F0B5044611
:100AF000CFB01546022301AA11F0D6FFD4F87839F9
:100B00000133C4F8783902A804F5A677FFF72CFF63
:100B100002AB2A4601A93846FFF776FED0B1BDF8F0
:100B20003631B4F874299A4203D1D4F87829022ACC
:100B30000CD9BDF83421A4F87439023A00235B487B
:100B4000C4F8783992B202A90DF008FE5849574806
:100B50000DF0AEFE04F2044602AB2A4601A930466F
:100B6000FFF752FED0B1BDF83631B4F874299A427D
:100B700003D1D4F87829022A0CD9BDF83421A4F87D
:100B80007439023A00234948C4F8783992B202A96C
:100B90000DF0E4FD474945480DF08AFE2A4604F26F
:100BA000BC6501A902AB2846FFF72EFED0B1BDF807
:100BB0003631B4F874299A4203D1D4F87829022A3C
:100BC0000CD9BDF83421A4F87439023A002337480F
:100BD000C4F8783902A992B20DF0C0FD3649334805
:100BE0000DF066FED4F88039D4F87C2902339342A4
:100BF000C4F8803901D24FB0F0BD0023C4F8803969
:100C00003846FFF71BFD034630461E46FFF716FD2C
:100C1000034628461D46FFF711FD07463EBB35BB80
:100C200028BB94F88539B3BB94F8870994F88A39BE
:100C300094F8882994F8891994F884590130C0B23D
:100C40005A4042401144C9B203EB51035340DBB256
:100C50009D4284F8882934BF0022012284F8870944
:100C600084F8891984F88A3984F88629C3E794F8C6
:100C7000853923B1002384F886394FB0F0BD0F4881
:100C8000012107F049FD0D48012107F051FD012325
:100C900084F88539EEE70948394607F03DFD0748F5
:100CA000394607F045FD84F88579BDE720E6FF1F4A
:100CB000D8440100EC44010000450100D096FF1F1C
:100CC00090F88609704700BF2DE9F041CEB20F467B
:100CD000F11E054649B200F5A67014469846FFF786
:100CE000A9FC394605F20440FFF7A4FCF11C49B207
:100CF00005F2BC60C4EB0414FFF79CFC240185F8EA
:100D00008489C5F87C49BDE8F08100BF10B54FF477
:100D100016720446002113F01BF800234FF4B4723E
:100D2000A4F85832A4F85A32A4F85C22A4F85E322F
:100D300084F86032204610BD2DE9F047CCB004465F
:100D40006846FFF7E5FD6846FFF75CFEB4F85C0215
:100D50000025A4F85852A4F85A5284F86052A4F816
:100D60005E52002800F0ED80794E20214FF04009BE
:100D70004FF080082A462B4611E014F80C3048EA60
:100D800003085FFA88FE0135ABB29F1C984204F855
:100D90000CE007F007070ED9C8468946F15D92F0CE
:100DA00001024FEAD30CE8D14FEAD30C14F80CE05F
:100DB0002EEA080EE7E784F86022A4F85802644F90
:100DC000431C9BB207F107083E46BE464FF0800A1F
:100DD00010E014F80C5049EA0505EDB201339BB25E
:100DE000F04504F80C5003F0070519D089461EF8A9
:100DF00001AF715D1AF07E0F03F1FF35ADB208BF90
:100E000082F001024FEAD50C08BF84F86022002A64
:100E1000DFD14FEAD50C14F80C5025EA0905DDE7BF
:100E2000BDF82C3100F1080C1FFA8CFCA4F858C254
:100E30004FEAC308002B00F089800020DFF81491EE
:100E40004FF0010A864619E00B4304F80A300CF112
:100E500001039BB22DB10EF1010E5FFA8EF5052D47
:100E600020D0013080B2404532D203F0070100F0BB
:100E7000070C715C19F80CA0AE469C46C3081DF81F
:100E800003501AEA050508BF82F00102CCF3CF0A2D
:100E900008BF84F8602214F80A30002AD4D123EA6B
:100EA0000103D2E782F0010284F86022002A3FD0D9
:100EB000D90803F00703655CF35C2B43013080B273
:100EC000635440450CF102039BB24FF00005CCD3B4
:100ED00003F00701A4F85832715C03F1080E1FFA01
:100EE0008EFE80200CE0605D014301339BB27345B0
:100EF000615503F0070C15D017F8010F16F80C1008
:100F000010F07E0F08BF82F00102C3F3CF0508BFC7
:100F100084F86022002AE6D1C3F3CF05605D20EAA1
:100F20000101E2E70020A4F858324CB0BDE8F08798
:100F3000C3F3CF0103F00703F55C635C23EA050309
:100F4000BCE740214FF08009024638E76346C4E71A
:100F5000144501001C45010030B58DB0B0F85E327B
:100F6000134C0DF1060C0DF12E050BE092101FFA3B
:100F70008EF35210772B2CF8022F84BF783B9BB254
:100F8000AC4508D034F9132003F1060E0029EDD149
:100F90000B339BB2EDE70022A0F85E320B210092EA
:100FA0000448142302AA07F0CDFA0DB030BD00BFEB
:100FB00024450100D096FF1FB0F858324BB31B4BAD
:100FC0001B7870B5044613B9B0F85A3243B31848C9
:100FD000184E07F079FB054617E0B4F85A32D908E5
:100FE00003F00702615CB25C01331142A4F85A328B
:100FF00014BF01210021FFF7AFFFB4F85A22B4F863
:101000005832143D9A42ADB204D2142D2046E4D891
:1010100070BD70470023A4F85A32A4F8583270BD4E
:101020000548FFF74DFE0028D1D170BD550EFF1FBA
:10103000D096FF1F14450100C016FF1F01EB4101B0
:101040008900A0F85C127047B0F85802B0FA80F03E
:1010500040094042C0B2704738B500F10C030D465C
:101060000446502200211846063512F071FEEDB2FA
:10107000044A606052F82520A260092121802046A0
:1010800038BD00BF7808FF1F11F00EBD03460631C2
:10109000054A4FF0090CC9B223F80CCB52F82120B5
:1010A00082604360704700BF7808FF1F10B54FF49F
:1010B0007A720446002112F04BFE002384F8EC33D0
:1010C000A4F8E833A4F8EA33204610BDB0F8E833BA
:1010D00003B970472DE9F043044683B02748284FF1
:1010E000DFF8A480254E07F0EFFA05461EE0CDF8A4
:1010F000009007F027FA94F8EC330133DBB2312B80
:1011000084F8EC33B4F8EA334FF0000284BF0133C3
:1011100084F8EC23B4F8E82388BF9BB2A5F1180546
:1011200088BFA4F8EA339A42ADB21FD9182D154AE8
:101130004FF000094FF018034FF0610130461AD903
:10114000B4F8EAC34FEADC0E0CF0070C14F80EE01A
:1011500017F80CC01EEA0C0EC9D1CDF800E0182318
:1011600042466121304607F0EDF9C4E70023A4F8B8
:10117000EA33A4F8E83303B0BDE8F083D096FF1F4C
:1011800040480100400AFF1F9016FF1F2DE9F84F4D
:10119000054616460F464FF47A72002112F0D8FD2C
:1011A00000214FF0080CA5F8E8C3A5F8EA1385F86C
:1011B000EC13002E5CD0314ADFF8CC8040F2E230F4
:1011C000002317F801A04124994603E012F82E40AD
:1011D0009946CCB30133DBB2A24503EB430EF5D104
:1011E00009EB490902EB89031C7A6CB3D3F804A01C
:1011F00004F1FF390CF1010353FA89F91FFA89F957
:101200004FF0004E11E02B5D18F80BB023EA0B03F2
:101210000CF1010B84452B551FFA8BFC4FEA5E0E37
:1012200026D8CC45A5F8E8C30ED03EEA0A034FEA1B
:10123000DC040CF0070BE6D15B4615F804B018F897
:10124000033043EA0B03E3E70131C9B2B142B7DB34
:10125000BCF1080F0CD00CF1050292B2A5F8E823FE
:101260000749084812B20DF053FB0020BDE8F88F83
:101270000023A5F8E8330420BDE8F88F30460100CC
:101280001446010020E6FF1F404801000023A0F89B
:10129000E833A0F8EA3380F8EC33704710B5002348
:1012A0000446038043600349232208300EF088FA85
:1012B000204610BD48480100154AC1EBC101531832
:1012C00000B593F801C080F817C093F802C080F809
:1012D00018C093F803C0525C93F804E0997980F841
:1012E00019C093F805C0037F80F81AE021F00F01C0
:1012F00003F00F030B430377837D80F81BC002F0DC
:101300000F0223F00F03134383755DF804FB00BF46
:1013100078480100154AC1EBC101531800B593F894
:1013200001C080F817C093F802C080F818C093F885
:1013300003C0525C93F804E0997980F819C093F8DF
:1013400005C0037F80F81AE021F00F0103F00F03BE
:101350000B430377837D80F81BC002F00F0223F05C
:101360000F03134383755DF804FB00BFA44801001D
:1013700010B50446304802F08DFD2F4802F084FB82
:1013800090B16378013B032B53D8DFE803F021369B
:10139000020E2A492848222202F038FA264802F092
:1013A000EFFD04236060637010BD234802F0E8FD88
:1013B00063681E339842F7D91F48002102F0E8FA0B
:1013C0001D4802F0D7FD002384F82A30637010BD59
:1013D0001948012102F0B6FD19491748092202F007
:1013E0007FFA18491448222202F010FA124801210B
:1013F00002F0CEFA0223637010BD94F82A10204642
:10140000FFF75AFF0C48222204F1080102F0FEF90E
:1014100094F82A30052B03D0013384F82A3010BD0C
:101420002378002284F82A20002BBDD10323637087
:1014300010BD0023637010BDE464FF1FF448010079
:101440006C480100D048010010B504461F4801F067
:1014500055F91E4801F0E8F950B16378022B18D015
:10146000032B0ED0012B04D00023637084F82A30A4
:1014700010BD17491548222201F0B6F80223637007
:1014800010BD14491148222201F0AEF80023637008
:1014900010BD94F82A102046FFF73CFF0B4822228B
:1014A00004F1080101F0A0F894F82A30052B03D0CC
:1014B000013384F82A3010BD2378002284F82A20D2
:1014C000002BD5D10323637010BD00BFF83DFF1F73
:1014D000184901003C49010008B5114B1B785C3BE1
:1014E000062B10D8DFE803F0140F10040F0F0400D0
:1014F00001780C4881B1012102F056FABDE808409C
:10150000084802F0C7BC08BDBDE80840FFF730BF7F
:10151000BDE80840FFF798BFBDE8084002F044BAB4
:1015200009A7FF1FE464FF1F012A14D10A78012ACA
:101530000CBF01230023037002D00023184670471C
:101540004378002BF9D10549097801F0FD015C29A8
:10155000F4D14270F2E704231846704709A7FF1F31
:1015600038B500250446056005718560302229469E
:101570000C3012F0EDFB84F83C50204638BD00BF23
:1015800010B5836800294FEA4303B8BF43F0010355
:101590008360044690F83C00421C04EB4000D2B249
:1015A0008181182A364828BF002223F07F4382B069
:1015B00084F83C2058400DF02DFB022814D8314906
:1015C00004F10A0304F13A004FF47A5C33F9022F74
:1015D0009142B8BF11469445A8BF94469842F5D1B0
:1015E000A1EB0C03052B35DCA368274823F07F43D0
:1015F00058400DF00FFB022814D8224904F10A03C9
:1016000004F13A004FF47A5C33F9022F9142B8BFEB
:1016100011469445A8BF94469842F5D1A1EB0C031E
:10162000052B01DC02B010BDC1F307228020CCF3F2
:1016300007238DF800008DF801208DF80210134863
:101640008DF80330052269468DF804C00DF0CCF802
:1016500002B010BDC1F3072300228DF800208DF8E1
:1016600001308DF80210CCF3072308488DF80330C1
:10167000052269468DF804C00DF0B6F8B4E700BF46
:1016800068B4AA0080C1FFFF974B550020E6FF1FFA
:1016900092B3013A92B22DE9F04104468D1E01EB5E
:1016A000420743F2333843F2CC4607E0B3F5004F2C
:1016B0001ED220713344BD42236017D035F9021F7A
:1016C0002379B3EBD17F4FEAD1702368EED1A3F534
:1016D0004C424344B3F5803F2071A2F1CD02204635
:1016E000E9D32260FFF74CFFBD42E7D1BDE8F081AE
:1016F0006FF4CC721344EAE7704700BF0022027017
:101700004280704710B5044684B0A14803F028FD1C
:1017100023780BB904B010BD9D4803F09BFE04284C
:10172000F8D99C4901AB04A89E2201E011F8012FD1
:1017300003F8012B8342F9D16288974BA3FB021374
:10174000D11A03EB51031B0903EB4303C3EBC303A0
:10175000D31A9BB293B901A90C228D4803F00CFB5C
:1017600063888E4901335A08A1FB0212120A40F223
:10177000762101FB1233638004B010BD511E07298E
:1017800069D8DFE801F06058504840383028092A0D
:1017900000F0B480092B00F0B9800A2A00F0AE8076
:1017A0000A2B00F0BB800B2A00F0A8800B2B00F066
:1017B000BD800C2A00F0A2800C2B00F0BF800D2A07
:1017C00000F09C800D2B00F0C1800E2A00F0968066
:1017D0000E2B40F0898050224BF26F338DF80D2094
:1017E000ADF80E30B7E733224BF23B338DF80D20C6
:1017F000ADF80E30AFE724224EF22A038DF80D200B
:10180000ADF80E30A7E732224BF222338DF80D20CF
:10181000ADF80E309FE71F224FF22B638DF80D209D
:10182000ADF80E3097E731224DF66F638DF80D203D
:10183000ADF80E308FE734224DF619638DF80D2088
:10184000ADF80E3087E730224DF602638DF80D209B
:10185000ADF80E307FE7591E072998D8DFE801F070
:101860002C241C143C340C0450224DF26F038DF8D0
:101870000D20ADF80E306EE725224CF20C738DF87A
:101880000D20ADF80E3066E733224BF21B338DF896
:101890000D20ADF80E305EE725224DF21D638DF868
:1018A0000D20ADF80E3056E770224DF60B238DF863
:1018B0000D20ADF80E304EE7252249F24F338DF85A
:1018C0000D20ADF80E3046E739224DF21D638DF83C
:1018D0000D20ADF80E303EE725224DF26F738DF8E6
:1018E0000D20ADF80E3036E70F2A07D00F2B35D07C
:1018F000102A03D0102B39D0112A3FD116224FF2D3
:1019000029538DF80D20ADF80E3024E725224DF235
:101910001E038DF80D20ADF80E301CE721224CF28D
:101920000C238DF80D20ADF80E3014E725224BF274
:101930006F338DF80D20ADF80E300CE73D224DF2DF
:1019400002738DF80D20ADF80E3004E725224DF618
:1019500019638DF80D20ADF80E30FCE625224DF20E
:101960001B638DF80D20ADF80E30F4E6232243F60C
:101970001B238DF80D20ADF80E30ECE6112BBDD1F8
:1019800021224FF225538DF80D20ADF80E30E2E6FE
:10199000A086FF1F6049010087611886D1000DD025
:1019A000012A15D138B50B78012B044603780CBFFA
:1019B0000125002503D06BB92570002038BD002B10
:1019C000FAD1438006490748292203F051F9F3E789
:1019D00004207047034803F055FA2570002038BDF5
:1019E0006C490100A086FF1F00224FF4C061026015
:1019F00042608160027370472DE9F0413B4E027BEB
:101A000033789A4282B0044636D0663B052B6AD8BA
:101A1000DFE803F003555A5F64504FF46F7303809F
:101A20000523334D606805EBC3056B88638010B1F7
:101A300010F04CF96388580010F046F96388606034
:101A4000C3B10027B846404611F05EFEB4F9083035
:101A50006268B9B283FB0030DB0F43EA400303F353
:101A60000F0322F81130013762886968BBB29A42CD
:101A70008844E8D833782373A37A13B902B0BDE859
:101A8000F0811C4806F020FE638883420546F5D2AB
:101A9000184F4FF0000862683178CDF80080384662
:101AA00006F050FD6388ED1AADB2AB42F3D302B03D
:101AB000BDE8F08140F6BF1303800023B1E740F298
:101AC0000F4303800423ACE740F2DF43038003238A
:101AD000A7E740F2616303800223A2E740F61F03F9
:101AE000038001239DE700230380C7E709A7FF1FA9
:101AF00098490100D096FF1F012A034608D10A78B1
:101B0000A2F10102B2FA82F2520900209A727047E1
:101B10000420704700220270704700BF10B50446D1
:101B2000084808F0CFF8237803B910BD054808F03D
:101B300095F90128F9D9BDE810400349014831223F
:101B400008F036B80CA2FF1FC8490100012A03465D
:101B500008D10A78A2F10102B2FA82F252090020F9
:101B60001A70704704207047002202704270827021
:101B7000704700BF10B50446114808F0DBFF10485D
:101B800009F0A2F828B16378012B03D00023637019
:101B9000A37010BDA3780B490948C3EBC303C3EB83
:101BA000C3033122194408F015FFA37822780133CA
:101BB00003F00303A370002AEBD1627010BD00BFD5
:101BC00088B6FF1FFC490100012A0FD10A78012ABB
:101BD0000CBF01230023037002D000231846704776
:101BE0004378002BF9D142701846704704231846F9
:101BF000704700BF002202704270704710B5044663
:101C0000104809F0E5FE0F4809F0B8FF30B16378DD
:101C1000012B0FD0022B02D00023637010BD0A49A4
:101C20000848D92209F0F4FD2378002BF5D00123D0
:101C3000637010BD05490348D92209F0E9FD02236C
:101C4000637010BD60DEFF1F4C0BFF1F700AFF1F8B
:101C5000012A0FD10A78012A0CBF01230023037047
:101C600002D00023184670474378002BF9D1427008
:101C70001846704704231846704700BF00220270C0
:101C8000704700BF08B5037803B908BD054806F0E2
:101C90001BFDA528F9D9BDE808400348AA210AF090
:101CA00055B800BFD096FF1FE0E3FF1F012A03468F
:101CB00008D10A78A2F10102B2FA82F25209002098
:101CC0001A7070470420704700224FF6FF710260BF
:101CD00042608160704700BF002A3BD02DE9F0418F
:101CE000013A92B2DFF8708082B004468D1E01EB9B
:101CF000420645F6BF5701E0AE4228D035F8022F24
:101D0000618963689142218938BF6281914221686B
:101D100088BF228101311344B94263602160EBD94D
:101D2000B3FBF1F3A2685BBA92FA82FC6946062221
:101D30004046ADF80430CDF800C00CF087FD00231C
:101D40004FF6FF72AE4223606360A260D6D102B04C
:101D5000BDE8F081704700BF20E6FF1F38B51422B0
:101D600004464FF43465002111F0F2FF2A460021A9
:101D700004F1140011F0ECFF002142F20F73C4F8DB
:101D8000541BC4F8581BA4F85C3BC4F8601BC4F88F
:101D9000641BC4F8681BC4F86C1BC4F8701BC4F83F
:101DA000741BA4F8781B84F87A1B2A4604F67C304E
:101DB00011F0CEFF204638BD002342F20F72C0F86A
:101DC000603B80F8753B80F8763B80F8783BC0F844
:101DD000583BA0F85C2B70472DE9F047BDF820E098
:101DE000BDF92470BDF92890002A00F08980013ADD
:101DF0000EF10406D2B20EF1020406EB42060EF119
:101E0000010E404DBFB2B6B2A4B21FFA8EFEC9F1A8
:101E100000082AE04FEAD20C02F0070215F802A0EF
:101E200013F80C2022EA0A0203F80C204FEADE0223
:101E30000EF0070C13F802A015F80CC04CEA0A0CBF
:101E400003F802C04A1D92B2B2F5B46F04F1020465
:101E500028BFA1F29B51A4B22CBF89B211460EF14A
:101E6000020EA6421FFA8EFE4AD000EB410CA21EC3
:101E7000BCF814C0ACEB070C0FFA8CFCC44592B252
:101E8000C8DBBCF1000F19DBCC454FEAD20C02F0E5
:101E9000070213F80CA0AA5C42EA0A0203F80C201D
:101EA0004FEADE020EF0070C21DA15F80CA013F849
:101EB00002C02CEA0A0C03F802C0C3E74FEAD20CB6
:101EC00002F0070215F802A013F80C2022EA0A0219
:101ED00003F80C204FEADE020EF0070C15F80CA0F8
:101EE00013F802C02CEA0A0C03F802C0AAE713F8A0
:101EF00002A015F80CC04CEA0A0C03F802C0A1E7D6
:101F0000BDE8F087284C01002DE9F04F07469748BF
:101F1000B7F8543B57F8233089B023F07F4358403B
:101F200004910CF077FEC31EDBB2122B4FD9B7F829
:101F3000563B8F4C8F4D03F22D5189B2B1F5B46FE2
:101F400024BF733B99B2804604F118098A480B46B6
:101F50004FF47A5E00264FF6FD7B4FF0030A14E043
:101F6000BCF1FF3F2DD012FB0A665A1D92B2B2F5AA
:101F7000B46F28BFA3F29B5304F101042CBF9BB2A2
:101F800013464C4505F101051DD007EB4302B2F99C
:101F900014209042B8BF10469645A8BF9646B8F1A7
:101FA000020F94BF94F900C095F900C0BCF1010F75
:101FB00005D0BCF1030FD3D112FB0B66D5E7B61ADF
:101FC000D3E71644D1E7D7F8603BB34202DB09B050
:101FD000BDE8F08F0EEB0005A0EB650044F6314341
:101FE00003FB00F040F3CF330593029345F34F0515
:101FF00004230093019506AB18223846FFF7ECFE48
:10200000B8F1020FDFF8749152D8DFF874810DF146
:1020100017040DF11E0A0D200F214FF0000B03E0F5
:1020200019F8011F18F8010F14F8013F0B40584030
:102030000CF0EAFDA24558445FFA80FBF0D1BBF1F9
:10204000030FC4D8049B002B66D197F8743B059905
:1020500007EB43020133DBB2032B88BF049BA2F8DA
:102060006C1BA2F8645B87F8743BB7F8563B4021C1
:1020700003F21A4292B2B2F5B46F28BFA3F5C3724D
:10208000A7F85A2B03F20D1292B2B2F5B46FA7F86B
:10209000583B28BFA3F29343C7F8606B87F8751BC2
:1020A00034BFA7F85C2BA7F85C3B09B0BDE8F08F04
:1020B000DFF8D0800DF117040DF11E0A07200F2163
:1020C0004FF0000B03E019F8011F18F8010F14F886
:1020D000013F0B4058400CF097FD544558445FFABF
:1020E00080FBF0D1BBF1030F3FF671AF049B43BB04
:1020F00097F8743B059907EB43020133DBB2032BDE
:1021000088BF049BA2F86C1BA2F8645B87F8743B41
:10211000B7F8563B2021ABE7059AA7F8722B0023AE
:10212000A7F8702BA7F86E2BA7F86C2BA7F86A5BA3
:10213000A7F8685BA7F8665BA7F8645B87F8743B51
:1021400093E7059AA7F8722B0023A7F8702BA7F83E
:102150006E2BA7F86C2BA7F86A5BA7F8685BA7F84B
:10216000665BA7F8645B87F8743BD1E76E2876005E
:10217000484C0100604C010080C1FFFF304C010061
:10218000384C0100404C010080F8771B704700BFBD
:10219000B0F85A3B3C3310B50A469BB24FF4077473
:1021A0004FF0000E00EB430103F1010C1FFA8CFC11
:1021B000B1F87C1B013CBCF5B46FA3F29F53A4B2F1
:1021C0008E442CBF9BB26346002CEBD108490948D2
:1021D000A1FB0E1E4FEA5E21CEF3474E82F823107C
:1021E00082F822E0BDE81040242301210BF0E0BF7B
:1021F00049D6B9F220E6FF1FB0F856CB00EB4C03EE
:1022000070B59982A3F87C2BB0F8542B50F822308B
:1022100000294FEA4303B8BF43F0010340F82230DE
:1022200090F8783B8EB00446002B00F0A480B0F804
:10223000581B01F29F539BB2B3F5B46F01F1010239
:1022400028BF01F1FF3392B228BF9BB2B2F5B46F41
:1022500024BFA1F29F518AB2934222D39C4524D23B
:10226000944522D9B4F85C3B634528D094F8780BA8
:10227000003818BF0120B4F8543B0CF1010C1FFAD0
:102280008CFC01339BB2BCF5B46F28BF4FF0000C3F
:10229000052B28BF0023A4F856CBA4F8543B0EB05E
:1022A00070BD9C45DED39445DCD800212046FFF765
:1022B0002BFEB4F856CBB4F85C3B6345D6D1B4F9E9
:1022C000662BB4F9646BB4F9683BB4F96C5B1644E3
:1022D0001E44B4F96A3B1E44B4F96E3B1D44B4F984
:1022E000703B0CF212311D44B4F9723B89B2B1F566
:1022F000B46F1D4494F8753B8DF8143028BFACF2D0
:102300008E214FF0080346F38F0645F38F0528BF53
:1023100089B20093029505AB019684222046FFF70F
:102320005BFD94F8753B402B43D0202B69D094F88B
:10233000782BAAB394F8763B0133DBB20C2B84F8EC
:10234000763B1ED8012A40F0E18094F8793B042BBB
:102350006AD80133DBB284F8793B8DF814307548C4
:10236000222305AA01210BF023FF94F8780B0038F3
:1023700018BF012015E00121FFF7C6FDB4F856CBC8
:1023800070E76C4801210BF04DFF002342F20F7201
:1023900084F8763B84F8783BC4F8583BA4F85C2B6F
:1023A00000200023B4F856CBC4F8603B84F8753B9A
:1023B00061E704A801F0DAF80DF113030DF1120240
:1023C00004A80DF1150101F005F994F8772B9DF89B
:1023D00012309A42C9D100239DF8142084F8763B2C
:1023E00084F8793B9DF813301A438DF814200A2B9A
:1023F0003BD8DFE803F0815D523A3A3A6D20203A4B
:102400002000B4F9582B4C494A48009533460CF04B
:10241000E5FA204605A9FFF7BBFE0120002384F85A
:10242000763BA4F8780BBCE7202200238DF814201B
:1024300084F8793B93E794F8780B022897D1B4F9A4
:10244000582B3E493B48009533460CF0C7FA2046CE
:1024500005A9FFF79DFE94F8780B9DF8133084F8DA
:102460007A3B003818BF01209BE73549B4F9582B57
:10247000009533462F480CF0B1FA204605A9FFF726
:1024800087FE002042F20F7384F8760B84F8780BF5
:10249000C4F8580BA4F85C3B83E794F8780B012848
:1024A0007FF465AFB4F9582B264900953346E1E730
:1024B0002549B4F9582B009533461E480CF08EFA86
:1024C00005A92046FFF764FE012084F8780B68E731
:1024D000B4F9582B1D491748009533460CF07EFA85
:1024E000204605A9FFF754FE0222002384F8782B2A
:1024F00084F87A3B012054E794F8783B012BE3D130
:10250000B4F9582B124900953346D6E7022A02D176
:1025100094F87A3B0BB9012043E743F0400305A947
:102520008DF81430FFF734FE94F8780B003818BF9C
:10253000012036E720E6FF1FF84B0100F44A0100B6
:10254000CC4B0100944B0100284B0100C04A010014
:102550005C4B0100B3B1F8B5013BDBB205468C1E04
:10256000961E01EB430734F9021F36F8022F284666
:10257000FFF742FEBC420146F5D1BDE8F8400348F2
:1025800006F0CAB80148194606F0C6B8D096FF1F33
:1025900070B5044600254FF4B9702581208065810F
:1025A000657325730FF090FB294660604FF49662C7
:1025B00004F13C0011F0CCFB04F11C06F023C4F83C
:1025C000F034C4F8EC5420222946304611F0C0FB08
:1025D000034A044B22616361A661204670BD00BFBF
:1025E00005000900280CFF1F222A01D00420704793
:1025F0004289038992B29BB29A4230B544D0428953
:10260000038992B29BB29A4208D343890489028813
:102610001B1B9BB29A420AD2052030BD0489028856
:10262000438912FA83F31B1B9BB29A42F4D3202BEB
:10263000F2D901F1210C4FF0010E18E04568038931
:102640009BB2EA54038901339BB203810289038858
:1026500092B29BB29A4228BF04810289438992B206
:102660009BB29A4208BF80F80CE061450AD0037B18
:1026700011F8012F03F0FF04002BDFD0614580F833
:102680000DE0F4D1002030BD037B002BC4D10388C2
:10269000CDE700BF70B58EB002AB04AD4FF4E3766A
:1026A00040F2525E4FF6AE2C4FF63A6201F0C00493
:1026B000802C1ED0C02C19D0B4B1A3F800C00233B6
:1026C00089009D42C9B2F1D12A4602A904231030E3
:1026D0000FF000FD00230093074814232A4602212F
:1026E00005F030FF0EB070BD1A80E8E7A3F800E0F7
:1026F000E5E71E80E3E700BFD096FF1F38B5B0F8CE
:10270000EC340446D3B1454805F0DEFF054611E040
:10271000B4F8EE345A1C2344A4F8EE2493F83C1089
:10272000FFF7B8FFB4F8EE24B4F8EC34143D9A4245
:10273000ADB233D2142D2046EAD838BD4189028982
:1027400089B292B291422DD04189028989B292B266
:1027500091421BD202894189521A92B2002AECD0CE
:102760002F4A12781ABBD4F8F024002A52D05F20E6
:10277000E11801339BB29A4281F83C00F8D892B23A
:102780000023A4F8EC24A4F8EE34BCE741890088C7
:10279000228910FA82F2521A92B2DFE70023C4F8BB
:1027A000EC3438BD027B002AC7D00288D6E704F19A
:1027B0003C0104F15D05002013E0626863899BB26F
:1027C000D35C0B702073638901339BB26381628990
:1027D000238892B29BB29A4228BF60810131A942FC
:1027E00009D02289638992B29BB29A42E5D1237BB8
:1027F000002BE2D1F2E70B4B04F15C0203F126005F
:10280000632101E013F8011B02F8011F8342F9D193
:102810004822B5E7A4F8EE2438BD00BFD096FF1FCC
:102820000AA7FF1F794C01004289038992B29BB22B
:102830009A4220D04289038992B29BB29A4208D32D
:102840004389018902885B1A9BB29A420AD200200E
:10285000704701890288438912FA83F35B1A9BB29D
:102860009A42F4D30648A0FB03201B1A00EB530046
:10287000C0F347107047037B002BE8D10388F1E7D2
:10288000D5411DD40C224FF4167302FB0133B3F56E
:10289000966F28BF4FF49663C0F8F034704700BFBE
:1028A00010B514220446002111F052FA4FF4A5622B
:1028B000002104F1140011F04BFA002342F20F72D0
:1028C00084F84C35C4F83C35A4F84025C4F84435A8
:1028D000C4F84835204610BD002342F20F72C0F8FC
:1028E0004435C0F84835C0F83C35A0F8402570475D
:1028F0002DE9F047BDF820E0BDF92470BDF928901E
:10290000002A00F08980013A0EF10406D2B20EF1DD
:10291000020406EB42060EF1010E404DBFB2B6B204
:10292000A4B21FFA8EFEC9F100082AE04FEAD20CC9
:1029300002F0070215F802A013F80C2022EA0A029E
:1029400003F80C204FEADE020EF0070C13F802A089
:1029500015F80CC04CEA0A0C03F802C04A1D92B2EA
:10296000B2F5257F04F1020428BFA1F28F21A4B2A1
:102970002CBF89B211460EF1020EA6421FFA8EFE3E
:102980004AD000EB410CA21EBCF814C0ACEB070C03
:102990000FFA8CFCC44592B2C8DBBCF1000F19DB06
:1029A000CC454FEAD20C02F0070213F80CA0AA5C47
:1029B00042EA0A0203F80C204FEADE020EF0070C8E
:1029C00021DA15F80CA013F802C02CEA0A0C03F85F
:1029D00002C0C3E74FEAD20C02F0070215F802A0CA
:1029E00013F80C2022EA0A0203F80C204FEADE0258
:1029F0000EF0070C15F80CA013F802C02CEA0A0C14
:102A000003F802C0AAE713F802A015F80CC04CEABC
:102A10000A0C03F802C0A1E7BDE8F087CC4C010026
:102A2000B0F83C2550F8223000294FEA43032DE945
:102A3000F04FB8BF43F0010340F82230B0F83E2514
:102A4000054605EB42027D48918223F07F4391B019
:102A500058400CF0DFF80228B5F83E7543D807F26D
:102A6000212189B2B1F5257F28BFA7F17301744CEC
:102A7000744828BF89B204F1170E8A466FF002022B
:102A80004FF47A5C00264FF6FD794FF0030811E011
:102A9000013222D013FB08660AF105039BB2B3F59D
:102AA000257F24BFAAF28F239BB2744517D014F957
:102AB000012F9A4605EB4A03B3F914309842B8BF88
:102AC00018469C45A8BF9C46012A04D0032ADFD1A2
:102AD00013FB0966E0E7F61ADEE71E44DCE7D5F8EB
:102AE0004435B34248DBB5F84035BB4213D0B5F8A6
:102AF0003C350137BFB201339BB2B7F5257F28BF04
:102B00000027052B28BF0023A5F83E75A5F83C3506
:102B100011B0BDE8F08F991D89B2B1F5257F24BFB2
:102B2000A3F28E2399B2B5F94A35B5F94825029337
:102B3000082301920093842207AB2846FFF7D8FEB2
:102B400006A800F013FD0DF11B030DF11A0206A8F3
:102B50000DF11D0100F03EFD95F84C259DF81A3051
:102B60009A423FD042F20F720023B5F83E75A5F8A5
:102B70004025C5F84435BAE784444CF34F03A0EB35
:102B80006C000593019344F6314303FB00F040F3DE
:102B9000CF3404230093284607AB02941822FFF792
:102BA000A7FEDFF8B090284F0DF11B0B0DF1220AA4
:102BB0000D200F234FF0000803E019F8013F17F82C
:102BC000010F1BF8011F0B4058400CF01DF8DA45AF
:102BD00040445FFA80F8F0D1B8F1030F10D9B5F88E
:102BE0003E7580E79DF81B30032BBBD1C3218DF8C8
:102BF0001C101648222307AA00210BF0D9FAB1E7CE
:102C0000DDF8148012491148234642460BF086FE37
:102C1000B5F83E75C5F8446507F20D139BB2B3F5E0
:102C2000257F22BF6FF4C373FB189BB2A5F84885BC
:102C3000A5F84A45A5F8403557E700BF6E2876004D
:102C4000E44C010080C1FFFFDC4C010020E6FF1FC7
:102C5000A04C0100D44C010072B1013AD2B270B55F
:102C600006468C1E01EB420534F9021F3046FFF781
:102C7000D7FEAC42F8D170BD704700BF80F84C154C
:102C8000704700BF10B50021044600F065F801212F
:102C900004F6546000F060F8204610BD2DE9F047BE
:102CA0009DF8207067B3013F82468E1E951E13FA71
:102CB00087F95C1E00F6546815E0082B504601D1D8
:102CC00000F07AF835F8022F36F9021F504600F06E
:102CD0006DFA2A88B6F900100746404600F066FAF9
:102CE0004C45034605D014F8013F042BE5D140467E
:102CF000E6E737B139460648BDE8F04705F00CBDB8
:102D00003B461F4639460248BDE8F04705F004BD82
:102D1000D096FF1F38B504460D4600F013FA294639
:102D200004F65460BDE8384000F00CBA38B50446EB
:102D30000D4600F00BFA294604F65460BDE8384011
:102D400000F004BA10B5044600F040F804F65460F0
:102D5000BDE8104000F03AB810B51422044600F85F
:102D6000041B002110F0F4FF4FF4E162002104F194
:102D7000180010F0EDFF002142F20F73C4F8201785
:102D8000C4F82417C4F82837C4F82C17C4F830172F
:102D9000C4F83417C4F83817C4F83C17C4F84017FF
:102DA000C4F8441784F848174FF4E16204F24A70FB
:102DB00010F0CEFF204610BD0023A0F82A37C0F83F
:102DC0002037C0F82C3780F841377047002342F293
:102DD0000F7280F8413780F8423780F84637C0F8E4
:102DE0002037C0F82437C0F82827C0F82C377047A0
:102DF0002DE9F04F85B0BDF94060BDF838C0BDF990
:102E00003CB00396002A76D0013AD2B20CF1030806
:102E100008EB42080CF1020472420CF1010C374D30
:102E200001921FFA8BFB1FFA88F8A4B21FFA8CFCE0
:102E3000029016E015F80A6015F8092013F80E90B4
:102E400029EA060903F80E90DE5D3243DA550CF1EB
:102E5000020C1FFA8CFC05310234E04589B2A4B2A1
:102E600049D0029801F10C024FEADC0730F81260F9
:102E70000198A6EB0B06A21E36B292B286420CF067
:102E800007094FEAD20E02F0070AD3DB002E4FEA01
:102E9000D20702F0070E17DB039886424FEAD20EE4
:102EA00002F0070917DA13F80E6015F8092032430B
:102EB00003F80E204FEADC020CF00706AF5D9E5CC3
:102EC00026EA07069E54C2E7DA5D15F80E6022EA8C
:102ED0000602DA55EEE713F80E6015F809203243C2
:102EE00003F80E200CF007064FEADC02AE5D9F5C93
:102EF0003E439E54ABE705B0BDE8F08F844E010021
:102F00002DE9F04F07468848B7F8203707EB8303D1
:102F100089B05B68049123F07F4358400BF07AFE40
:102F2000C31EDBB2122B40D9B7F822177F4C804D5D
:102F3000733989B2804604F118097E480B464FF474
:102F40007A5E00264FF6FD7B4FF0030A0BE0BCF1E2
:102F5000FF3F24D012FB0A66013405334C459BB277
:102F600005F101051DD003F10C0237F91220904242
:102F7000B8BF10469645A8BF9646B8F1020F94BF59
:102F800094F900C095F900C0BCF1010F05D0BCF167
:102F9000030FDCD112FB0B66DEE7B61ADCE7164442
:102FA000DAE7D7F82C37B34202DB09B0BDE8F08F7F
:102FB0000EEB0005A0EB650044F6314303FB00F087
:102FC00040F3CF330593029345F34F050423009359
:102FD000019506AB18223846FFF70AFFB8F1020F39
:102FE000DFF8549143D8DFF854810DF117040DF147
:102FF0001E0A0D200F214FF0000B03E019F8011FEE
:1030000018F8010F14F8013F0B4058400BF0FCFD7D
:10301000544558445FFA80FBF0D1BBF1030FC4D88C
:10302000049B002B56D197F84037059907EB4302D4
:103030000133DBB2032B88BF049BA2F83817A2F838
:10304000305787F84037B7F822374022A3F5C371CD
:1030500087F8412703F20D12C7F82C67A7F8243729
:10306000A7F82617A7F8282709B0BDE8F08FDFF8E2
:10307000D0800DF117040DF11E0A07200F214FF02B
:10308000000B03E019F8011F18F8010F14F8013FB5
:103090000B4058400BF0B8FD544558445FFA80FB94
:1030A000F0D1BBF1030F80D8049B43BB97F84037A6
:1030B000059907EB43020133DBB2032B88BF049B66
:1030C000A2F83817A2F8305787F84037B7F82237F8
:1030D0002022BBE7059AA7F83E270023A7F83C2744
:1030E000A7F83A27A7F83827A7F83657A7F834578C
:1030F000A7F83257A7F8305787F84037A3E7059A63
:10310000A7F83E270023A7F83C27A7F83A27A7F8F7
:103110003827A7F83657A7F83457A7F83257A7F833
:10312000305787F84037D1E76E287600A44E01006B
:10313000BC4E010080C1FFFF8C4E0100944E010087
:103140009C4E010080F84317704700BFA0F8441759
:10315000704700BF10B5B0F8264704F13C0304F5F2
:1031600016740A469BB2A4B24FF0000C00EB430E5B
:103170000133BEF84AE79BB2A342F444F6D1094BAF
:10318000A3FB0C3C4FEA5C23CCF3474C82F8233082
:1031900082F822C001780448BDE8104024230BF0D7
:1031A00007B800BF49D6B9F220E6FF1F70B5B0F8E6
:1031B0002A3704460133B0F844079BB298428EB0D8
:1031C000A4F82A3736D8B4F82237B4F8280783424F
:1031D00030D8B3F5617F2DD204EB43050029A5F863
:1031E0004A272983B4F8202704EB820255684FEA66
:1031F0004505B8BF45F00105556094F8462702BB68
:10320000A3F5C8725A2A7FD983422DD094F8460775
:10321000003818BF0120B4F82027013292B2052AE5
:1032200003F1010328BF0022A4F82237A4F82027C5
:103230000EB070BD94F84607003818BF01200EB0DC
:1032400070BDB4F82427511E89B28B42DCD3013201
:1032500092B29342D8D820460021FFF751FEB4F82D
:103260002237B4F82807CFE7B4F93217B4F930574A
:10327000B4F93427B4F938670D441544B4F9362746
:103280001544B4F93A2745F38F051644B4F93C27A1
:1032900001951644B4F93E27A3F28E2399B2164441
:1032A00094F841378DF8143046F38F0608230093C5
:1032B000029605AB84222046FFF79AFD94F8413729
:1032C000402B09D0202B28D094F84627002A54D12F
:1032D0000020B4F822379EE704A800F047F90DF16A
:1032E00013030DF1120204A80DF1150100F072F99B
:1032F00094F843279DF812309A427AD094F8460702
:10330000003818BF0120E4E720460121FFF7F8FD4F
:10331000B4F82237B4F8280776E722780196B4F992
:10332000243789488949009501320BF0D3FBB4F862
:10333000262702F13C0302F5167290B29BB20022DE
:1033400004EB43010133B1F84A179BB283420A44AC
:10335000F6D17F4B2178A3FB0230400A40BA2423E8
:10336000ADF8360005AA78480AF022FF01200023B4
:1033700084F84237A4F84607ABE794F842370133A4
:10338000DBB20C2B84F8423727D8012A15D194F8E8
:103390004737042B1AD9202200238DF8142084F8F3
:1033A000473769482178222305AA0AF001FF94F8DB
:1033B0004607003818BF01208BE7022A04D194F891
:1033C0004817002940F09B80012082E70133DBB2DF
:1033D00084F847378DF81430E3E721785A480AF02B
:1033E00021FF002242F20F7384F84627A4F8283701
:1033F0006EE700239DF8142084F8423784F847379D
:103400009DF813301A438DF814200A2B21D8DFE8D9
:1034100003F06A584B20202036060620060094F858
:10342000460702287FF46CAF22780196B4F924375E
:1034300048494548009501320BF04CFB204605A950
:10344000FFF788FE9DF8133094F8460784F8483754
:1034500056E7227840490196B4F9243700950132A5
:1034600039480BF037FB204605A9FFF773FE002013
:1034700042F20F7384F84607A4F8283740E7227811
:103480000196B4F9243735492F48009501320BF0E5
:1034900021FB204605A9FFF75DFE0220002384F8EA
:1034A000460784F848372BE794F8460701287FF44D
:1034B00027AF22780196B4F92437294900950132C3
:1034C000CEE7227827490196B4F9243700950132D6
:1034D0001D480BF0FFFA05A92046FFF73BFE01202F
:1034E00084F846070CE794F84637012BF7D1227889
:1034F0000196B4F924371C4900950132E8E7B4F885
:10350000262741F0400102F13C0302F5167290B209
:103510008DF814109BB2002204EB43010133B1F883
:103520004A179BB283420A44F6D1094B2178A3FB88
:103530000230400A40BAADF836002423024805AAFA
:103540000AF036FEDAE600BF20E6FF1F4C4E01000F
:1035500049D6B9F2344D01001C4E0100FC4C01006B
:10356000E04D01006C4D0100A44D0100704700BF0B
:1035700048780A788B78C00000EBC22000EB53102B
:10358000B0F5006F1BDB10B4104C204202460DD08A
:103590004FF4802340F6754C134208BF5B08FBD004
:1035A000D90A0CFB01F14A402242F5D1084B5DF8E3
:1035B000044B53F822305840C0F3C7207047044BE7
:1035C00053F820305840C0F3C720704700F8FFFF81
:1035D000D44E010070B591F80DE091F813C00E7B48
:1035E00015464FEA8C0C4FEA8E021C460CF03C0C40
:1035F0000B7D22F03F0282B04CEA020141EA9311B6
:103600004FEA9E1E9B004EEA860E8DF8051023F0B1
:103610000F0301A98DF806308DF804E0FFF7A8FF2D
:10362000030900F00F002B70207002B070BD00BFC6
:1036300002F00F0210B5187B93F80DE042EA011278
:10364000D2B2134920F03F000EF00F0E31F81210E5
:103650004EEA821E40EA92021A731A7DC1F3850C6B
:10366000CCB202F00302890A01F03C0142EA841262
:103670000A431A75DA7C0CF00F000CF0300122F0CE
:103680000F024EEA010102435973DA7410BD00BF04
:10369000D46E0100F8B500254FF4B97604460581D3
:1036A000068045814573057330460EF00DFB25837A
:1036B0006060658326822577657730460EF004FBCF
:1036C000282729466061212284F84C5004F14D00DE
:1036D00010F03EFB3A46294684F86E5004F187000C
:1036E00010F036FB04F12C063A46294604F1AF00EF
:1036F00010F02EFB29462022C4F8D850C4F8DC5024
:10370000304610F025FB094B094A226209496362E1
:10371000A662182204F16F000CF052F8C4F8E050D1
:10372000C4F8E450A4F8E8502046F8BD840CFF1F0C
:1037300005000900D4700100222A01D0042070473E
:103740004289038992B29BB29A4230B556D04289DF
:10375000038992B29BB29A4208D3438904890288B2
:103760001B1B9BB29A420AD2052030BD04890288F5
:10377000438912FA83F31B1B9BB29A42F4D3202B8A
:10378000F2D990F8E83033B10023038143734381C9
:1037900080F8E830037301F1210C4FF0010E18E0BE
:1037A000456803899BB2EA54038901339BB20381C4
:1037B0000289038892B29BB29A4228BF048102898F
:1037C000438992B29BB29A4208BF80F80CE06145EF
:1037D0000AD0037B11F8012F03F0FF04002BDFD088
:1037E000614580F80DE0F4D1074B1B7823B9012225
:1037F00080F84C20184630BD002030BD037B002BE4
:10380000B2D10388BBE700BF0AA7FF1F222A01D05D
:1038100004207047428B038B92B29BB29A4230B520
:1038200056D0428B038B92B29BB29A4208D3438B01
:10383000048B028A1B1B9BB29A420AD2052030BD20
:10384000048B028A438B12FA83F31B1B9BB29A42AE
:10385000F4D3202BF2D990F8E93033B1002303835D
:103860004377438380F8E930037701F1210C4FF06F
:10387000010E18E04569038B9BB2EA54038B0133B8
:103880009BB20383028B038A92B29BB29A4228BFF7
:103890000483028B438B92B29BB29A4208BF80F89A
:1038A0001CE061450AD0037F11F8012F03F0FF04EB
:1038B000002BDFD0614580F81DE0F4D1074B1B7869
:1038C00023B9012280F84C20184630BD002030BDBD
:1038D000037F002BB2D1038ABBE700BF0AA7FF1FFB
:1038E000092A01D0042070472DE9F8430C22044630
:1038F0000D467B30002110F02BFA0021164F174E99
:1039000040204FF080080B460A460BE017F8012FC5
:1039100016F8018002F0070004EBD201305C91F848
:103920007B10D2084FEAD30E5FFA82FC15F80E9096
:10393000013318EA090FDBB2A44441EA000E08BFC4
:1039400021EA000E442B03F007018CF87BE0DDD167
:103950000020BDE8F88300BF247101001C71010044
:10396000012A04D1097801290AD0022901D00420B2
:1039700070470023C0F8E43080F8E920184670470B
:103980000023C0F8E03080F8E8101846704700BF08
:10399000002380F84C10C0F8DC30C0F8E030C0F8EC
:1039A000E430A0F8E8307047002914BF0523002355
:1039B00080F84C30704700BFF0B595B003AB05AD53
:1039C0004FF4E37740F252564FF6AE2E4FF63A6C74
:1039D00001F0C004802C25D0C02C21D0ECB1A3F87C
:1039E00000E0023389009D42C9B2F1D10023AB60EF
:1039F00003A9059320306B60EB602B618DF81E20CE
:103A000004230AAA0EF066FB0748009514230AAAAD
:103A1000022104F097FD15B0F0BDA3F800C0E0E767
:103A20001E80DEE71F80DCE7D096FF1F42890389F6
:103A300092B29BB29A4220D04289038992B29BB241
:103A40009A4208D34389018902885B1A9BB29A4241
:103A50000AD20020704701890288438912FA83F351
:103A60005B1A9BB29A42F4D30648A0FB03201B1AB0
:103A700000EB5300C0F347107047037B002BE8D1E5
:103A80000388F1E7D5411DD4428B038B92B29BB2E0
:103A90009A4220D0428B038B92B29BB29A4208D3B7
:103AA000438B018B028A5B1A9BB29A420AD2002096
:103AB0007047018B028A438B12FA83F35B1A9BB225
:103AC0009A42F4D30648A0FB03201B1A00EB5300D4
:103AD000C0F347107047037F002BE8D1038AF1E75A
:103AE000D5411DD400EB011270B5558904461089EB
:103AF000ADB280B285424FEA011363D05589108977
:103B0000ADB280B2854242D35089E55A128915FA86
:103B100082F2121A92B2202A3FD9D4F8DC20132A5A
:103B20003BD901F1380254F82220052A35D904F195
:103B3000860004F1A705234404EB01114FF0000EA9
:103B400019E04E685A8992B2B25C80F8292083F855
:103B50000CE05A89013292B25A81B3F80AC00A883D
:103B60001FFA8CFC92B2944528BFA3F80AE000F833
:103B700001EF854222D0B3F808C05A891FFA8CFCA5
:103B800092B29445DDD11A7B002ADAD1EFE7108991
:103B90005289821A92B2202ABFD86318002504F1F4
:103BA0004D01212283F8E85004F1AF000BF008FE2C
:103BB0002122294604F1870010F0CAF82123C4F815
:103BC000D83070BD127B002AE7D0E25AA3E700BFCD
:103BD00038B5304B93F800C0BCF1620F044646D0B4
:103BE000BCF15F0F3FD15520002384F8AF0084F86B
:103BF000B00084F8B10084F8B20084F8B30084F80F
:103C0000B40084F8B5000F21FF2084F8873084F8D1
:103C1000883084F8893084F88A3084F88B3084F8CE
:103C20008C3084F88D3084F8B6C084F8B70084F8FE
:103C3000B80084F8B90084F8BA0084F8BB0084F8AE
:103C4000BC0084F8BD0084F88F3084F8903084F88C
:103C5000913084F8923084F8933084F8943084F86A
:103C60009530A4F8D8100023A4F8DA3038BD21220A
:103C700015465F21AF3010F06BF82A46002104F1A1
:103C8000870010F065F80023A4F8D850A4F8DA30C3
:103C900038BD00BF09A7FF1F2DE9F8430446D0F83F
:103CA000DC00D4F8E03094F86E700133C4F8E030F2
:103CB000D4F8E43000F1010901330B2FC4F8DC9093
:103CC0000D46C4F8E430904624D9002384F86E30C1
:103CD0006289238992B29BB29A4200F0C4806289C1
:103CE000238992B29BB29A4280F0908023896289A4
:103CF0009B1A9BB2002B00F0938004F16F030C22FF
:103D000004F17B0118460BF05BFD002103460326FE
:103D10000F4606E0002FDBD0FE1CF6B204F16F0365
:103D200039461944032204F1AF000BF049FDB8F104
:103D3000010F4FF000000CBF08230423B9F1130F4B
:103D400084F8870084F8880084F8893038D80146E0
:103D5000A5F1010CBCFA8CFC4FEA5C1C5FB3093F77
:103D600018BF0127FA006B1E18BF012342F080051F
:103D7000012281EA0C017B404F40514094F8AF2072
:103D800084F86E6042EACC02104394F8B02084F8C4
:103D9000AF005B0194F8B10043EA47032A4342EACB
:103DA00041020343032184F8B02084F8B130C4F801
:103DB000D810BDE8F8833A46634608250127D8E7BE
:103DC00004EB08134FEA081859891A8989B292B28C
:103DD00091423DD059891A8989B292B2914208D252
:103DE00019895B8989B29BB2C91A18BF0121C80120
:103DF000AEE734F808005A89198910FA81F193B2B4
:103E000089B2C91A18BF0121C801A1E762892188B6
:103E1000238911FA83F39B1A9BB2002B7FF46DAFB9
:103E2000628B238B92B29BB29A4223D0628B238BFC
:103E300092B29BB29A4222D2238B628B9B1A9BB284
:103E4000002B7FF45AAF124904F16F030C2259E79B
:103E50001B7B03F0FF015BB134F80810091A18BF8F
:103E60000121C80174E7237B002BD9D0238841E7C7
:103E700008466DE7237F002BE5D0238AE0E7628BBD
:103E8000218A238B11FA83F39B1A9BB2D8E700BFD8
:103E9000EC70010038B590F84C30FBB1B0F8D82088
:103EA0000446E2B1264804F00FFC054613E0B4F8DE
:103EB000DA30E218013392F8AF1092F88720A4F8B4
:103EC000DA30FFF779FDB4F8DA20B4F8D830143DD1
:103ED0009A42ADB230D2142D2046E8D838BD013B0D
:103EE000042B21D8DFE803F01920120A0300FFF7A2
:103EF0006FFEB4F8D830002BD4D138BD0022012198
:103F0000FFF7CAFE032384F84C30F2E70121FFF7E4
:103F1000E9FD022384F84C30EBE70021FFF7E2FDD6
:103F2000042384F84C30E4E701220021FFF7B4FEBB
:103F3000012384F84C30DCE70023C4F8D83038BDC6
:103F4000D096FF1F10B500F14D0384B021220C461E
:103F50001846074901930BF033FC03A8FFF706FB53
:103F6000019B0922214603A8FFF762FB04B010BDA4
:103F7000F87001000023038343774383037770477E
:103F8000D0F8DC00704700BF38B500240546214654
:103F900000F8084B28220FF0DBFE214641F6DC1228
:103FA00005F130000FF0D4FE05F5D05021464FF456
:103FB00070720C300FF0CCFE05F580532449C3F825
:103FC000D01D2449C3F8D41D05F5EF5042F20F71FE
:103FD000C3F8CC4DA3F8D81DC3F8DC4DC3F8E04DB1
:103FE000A3F8E44D83F8E64DC3F8E84DC3F8EC4D73
:103FF000C3F8F04DC3F8F44DC3F8F84D2146A8229C
:104000001C300FF0A5FE05F5F5502146A82204301E
:104010000FF09EFE05F5FA502146A8220C300FF055
:1040200097FE05F5FF502146A82214300FF090FEB0
:1040300005F502502A2221461C300FF089FE05F5B5
:1040400000532846C3F8C840A3F8CC4038BD00BF91
:1040500000000F270F270F2700F5805210B4002310
:1040600000F500510D4C0370C2F8D04D82F8E63DCA
:104070000B4CC2F8D44D42F20F70C2F8DC3DC2F8CE
:10408000E03DC2F8CC3DA2F8D80DA2F8E43D5DF8C1
:10409000044BC1F8C830A1F8CC30704700000F279E
:1040A0000F270F2770B500F580550446B5F8CC3DB5
:1040B00020480133002154F8333023F07F43584027
:1040C0000AF0BEFD02282BD8B5F8D03D1A4903F2FC
:1040D0006D1292B2B2F5F07F24BF733B9AB201F138
:1040E000180C00200CE0C01A531D9BB26FF4ED7643
:1040F000B3F5F07F32442CBF92B21A468C450BD0F8
:1041000002F6045304EB430311F8016FB3F90430D2
:10411000002EE8D11844E7E7D5F8DC3D834201DB07
:10412000002070BD0023C5F8DC0DA5F8CE3D0120B0
:1041300070BD00BF50765500D779010070B500F50D
:1041400080550446B5F8CC3D027837480133022A41
:1041500054F8333023F07F4380EA03004FF000012E
:104160000CBF022600260AF06BFDB0422CD8B5F831
:10417000D0CD2E490CF26D1292B2B2F5F07F24BF71
:10418000ACF1730292B2002001F1180E0CE0C01ADB
:10419000531D9BB26FF4ED76B3F5F07F32442CBF24
:1041A00092B21A4671450BD002F6045304EB430356
:1041B00011F8016FB3F90430002EE8D11844E7E795
:1041C000D5F8E03D834201DB002070BD0CF1050312
:1041D0009BB20022B3F5F07FA5F8E42D24BF6FF465
:1041E000ED720CEB0203A5F8D23D0CF101039BB27A
:1041F000B3F5F07F24BF6FF4EF736344A5F8D83DA7
:104200000CF2DF139BB2B3F5F07FA5F8D4CD28BF35
:104210000CF1FF3CC5F8E00D34BFA5F8D63DA5F87C
:10422000D6CD012070BD00BF68B4AA00BF790100DF
:1042300038B504460D46FFF735FFB8B104F5805296
:104240000521B2F8CE3D82F8E61D03F1180004F511
:104250000051013324F81050A2F8CE3D0020012374
:10426000C1F8C800A1F8CC00237038BD2046FFF784
:1042700065FF0028F9D0074907480AF019FB0748ED
:10428000012104F049FA0548012104F051FA022302
:10429000237038BD6871010020E6FF1FD096FF1F14
:1042A0002DE9F04F00F580540546B4F8CC3D744834
:1042B0000133002655F8333087B0584031460AF0B4
:1042C000BFFC012871D9B4F8D63DB4F8D82DB4F8A4
:1042D000D01D93420AD38B4248D98A4246D2B4F8C1
:1042E000E43D952B49D807B0BDE8F08F8B42F4D957
:1042F000B4F8E42D952A40D8B4F8D8EDB4F8D03D00
:104300007345F0D1B4F8D28D5E4FDFF8909105F58A
:10431000D05C0CF10C0C4146002302AE14E016F800
:104320000BB0385C00EA0B0006F80A00481D80B2AA
:104330006FF4ED7A0133B0F5F07F51449BB22CBF9E
:1043400089B20146602B47D03CF911004FEAD30BEC
:104350000028DA4603F00700E1DA16F80BA019F896
:10436000000040EA0A0006F80B00DFE72846FFF7E6
:10437000E5FEB4F8E42D952ABED9434943480AF036
:1043800097FA4348002104F0C7F90021404804F09F
:10439000CFF93E4809F0CCFE0023C4F8DC3DC4F858
:1043A000E03D2B7007B0BDE8F08F384839490AF07E
:1043B0007FFA3146364804F0AFF93146344804F00C
:1043C000B7F9324809F0D4FEC4F8DC6DC4F8E06DEA
:1043D0002E7007B0BDE8F08F02EB021303EB8313DE
:1043E00002EB8303C3EB830302EB83039BB2B3F5BE
:1043F000436F29D872B305F50055B5F8CC20B2B992
:1044000022480C22314609F05DFE0023C5F8C83071
:10441000A5F8CC30B4F8E43D00220133A4F8E43D23
:10442000C4F8DC2DC4F8E02D07B0BDE8F08FD5F856
:10443000C8301648B3FBF2F331465BBA0E22ADF832
:10444000143009F03FFEE0E710480C22314609F035
:1044500039FEDFE70FFA8EF30093B4F9D61DB4F9F5
:10446000D43D019155218DF8111041F22D61ADF827
:104470001210064808490FFA88F20AF02BFBBAE737
:104480005E13AAAA2C740100AC71010020E6FF1F84
:10449000D096FF1F8C710100D471010034740100AB
:1044A00000F580532DE9F0470C68D3F8EC7D0E69D8
:1044B000D3F8E82D07EB040ED3F8F44D2644B645A7
:1044C0004FEAD2087546A8BF3546B64508F27E7653
:1044D00000EB860602F0070CD6F804E0AA4655DA8F
:1044E000394E16F80C6006EA0E0600EB880000F55F
:1044F0008050C0F8FC6D4E6837444E693444A74282
:104500003E46A8BF2646A74256DA2F4CD0F8A47ED6
:1045100014F80C403C40C0F8A44E8C68D3F8F07DF1
:104520008D6907EB0409D3F8F84D04EB0508C14584
:10453000CE46A8BFC646C14535DADFF88C80D0F834
:104540004C5F18F80C8008EA0508C0F84C8FCD685D
:10455000C9692F4421448F423C46A8BF0C468F4274
:104560001ADA1949D0F8F47F11F80C103940C0F864
:10457000F41F0132C3F8ECADC3F8F06DC3F8F4EDED
:10458000C3F8F84DC3F8E82DBDE8F0870F4E16F8D4
:104590000C6046EA0E06A8E70C49D0F8F47F11F843
:1045A0000C103943E3E7DFF82480D0F84C5F18F8AB
:1045B0000C8048EA0508C8E7044CD0F8A47E14F83B
:1045C0000C403C43A7E700BF1C74010024740100A9
:1045D00010B54A680B6888B0D11883F0010C82F0DE
:1045E0000104234462446444009105916946CDE985
:1045F0000232CDE9062301940494FFF751FF08B07D
:1046000010BD00BF2DE9F0414F4A504C7F27402597
:1046100040F249164FF0000C42F29C030FE000EB11
:10462000DC05013EE95C3940E954751C0CF1010CD4
:104630004BD006F007050CF00701555D675CF110E3
:1046400001F27E7100EB810149680D42E7D000EB79
:10465000DC0E751E1EF8031039400EF803100CF125
:10466000010C96B3E91001F2D27100EB810105F063
:1046700007064968965D0E4252D000EBDC010CF053
:10468000070611F803E0A75D07EA0E07CF546E1E78
:10469000DDB1AC44F11001F2FC7106F0070500EB4E
:1046A000810112F805E04D68ACEB06011EEA050F2A
:1046B00000EBD10701F0070809D0FD5C12F80810E3
:1046C000013E2943F954711CE4D1BDE8F08100EBAF
:1046D000D10701F0070517F803E0555D01F1010C62
:1046E00045EA0E01F954771E002EEED0F91001F5BF
:1046F000F56100EB810107F007054968555D0D4242
:1047000000EBDC050CF00701EE5C515C41EA0601B0
:10471000E9540CF1010C11D07D1E002FA2D1D4E779
:1047200000EBDC060CF00701F75C615C3940F154EA
:104730000CF1010C6F1E002DD8D1C6E77E1E002F94
:104740007FF477AFC1E700BF247401001C7401003F
:10475000FF2310B54A1E114C01F1260E184601E048
:10476000180ADBB212F801CF83EA0C03964534F83D
:10477000133083EA0003F3D1DB4391F82700DAB268
:1047800090429BB201D0002010BD91F82820B2EBDE
:10479000132F0CBF0120002010BD00BF1C720100B0
:1047A0002DE9F0438B4C0F46154699B04A1E06463C
:1047B00004F15201702301E014F8013B12F8010FDB
:1047C000A14283EA00031370F6D10021542203A80A
:1047D0000FF0BEFADFF800C2002180240CEB410389
:1047E00048E0CA10BA5CD0070DD593F800E05878BD
:1047F0000EF1600EEE4424FA00F01EF8548C40EAEC
:1048000008000EF8540C90070DD593F802E0D87804
:104810000EF1600EEE4424FA00F01EF8548C40EACB
:1048200008000EF8540C50070DD593F804E05879A1
:104830000EF1600EEE4424FA00F01EF8548C40EAAB
:1048400008000EF8540C10070DD593F806E0D8793F
:104850000EF1600EEE4424FA00F01EF8548C40EA8B
:1048600008000EF8540C081DB0F5257F03F108036D
:1048700064DB0146B1F5257FB3DB06F580530024E8
:10488000C3F8EC4DC3F8F04DC3F8F44DC3F8F84D40
:10489000C3F8E84D4FF08008402718AB03EBE40263
:1048A00004F0070312F8542C28FA03F1114227FAF6
:1048B00003F314BF4FF0010C4FF0000C134214BF70
:1048C0000123002301A930460234CDF808C001932A
:1048D000FFF77EFEB4F5257FDFD13046FFF792FE6D
:1048E0002922002128460FF033FA40F24911DFF85F
:1048F000EC8040220F4642F29C0E4FF0010C01E08A
:1049000018F8042006EBE1047B1A14F80E90D8087E
:10491000013903F0070312EA090F01F007040CFA4A
:1049200003F302D02A5C13432B544B1CE8D12946D5
:10493000304619B0BDE8F043FFF70ABFD3060FD5E4
:104940001CF810E00CEB40000EF160030DEB030EC1
:1049500043781EF8540C24FA03F303430EF8543C36
:10496000930610D54B1D0CEB430E1CF813009EF85C
:1049700001306030684424FA03F310F854EC43EA41
:104980000E0300F8543C500612D412060ED5CB1D6F
:104990000CEB43001CF81320437860326A4424FA7D
:1049A00003F312F8540C034302F8543C083115E7A2
:1049B0008B1D0CEB430E1CF813009EF80130603089
:1049C000684424FA03F310F854EC43EA0E0300F8A9
:1049D000543CDAE73D74010098740100247401002E
:1049E0002DE9F04700F58055A2B095F8E63D044664
:1049F0000E46A3B9B5F8CE3D03F11802013324F8F1
:104A000012609BB240F6E9429342A5F8CE3D2DD00C
:104A100040F6EE4293420AD022B0BDE8F087FFF79D
:104A200041FB95F8E63D013B85F8E63DE2E70022D3
:104A3000A5F8E42D4FF0EE72C5F8D02D4FF4EC73CD
:104A40003F49C5F8D41D4FF4EB72A5F8D83D3D4958
:104A5000019200933C4840F2D7134FF4EE720AF0F3
:104A600039F80223237022B0BDE8F087DFF8E08038
:104A7000DFF8E09004F13007002305220DA940F68D
:104A8000E34E17E003F0070011F80CC018F800001F
:104A900000EA0C00885502F1050C1FFA8CFC01336A
:104AA000F445A2F6DF429BB28CBF92B26246B3F5E8
:104AB000257F10D037F912004FEAD30C002803F0FD
:104AC000070A6646DEDA11F80C6019F80A0030436E
:104AD00001F80C00DFE702AA2046FFF761FE38B9B3
:104AE0002070C5F8DC0DC5F8E00DB5F8CE3D8FE7B8
:104AF0001648012104F5005603F00EFE134801216B
:104B000003F016FEB6F8CC2052B90F48292202A9AC
:104B100009F0A2FA0023C6F8C830A6F8CC30E4E7C2
:104B2000D6F8C8300848B3FBF2F302A98DF832304A
:104B30002B22C3F307238DF8313009F08DFAE9E712
:104B4000D701D601F871010020E6FF1FD096FF1FA4
:104B50002C74010034740100002B5BD02DE9F84364
:104B600000F580545E1E8146B6B2B4F8CC3DB4F870
:104B7000D00DA1F1020802EB4606971E09F500557B
:104B800017E04846FFF754FBB4F8D00DB4F8CC3D1D
:104B9000013080B201339BB2B0F5F07F28BF002016
:104BA000052B28BF0023BE42A4F8D00DA4F8CC3DAD
:104BB0002ED037F802CFD5F8C820B5F8CC1009EBC5
:104BC000C30362440131A5F8CC10C5F8C8209A6827
:104BD000D3F80CC038F9021F92184CEB0C0C0029CA
:104BE000B8BF42F00102C3E9022C00F6045099F864
:104BF000003009EB4000012B818005D0022BC0D191
:104C00004846FFF74DFBBFE74846FFF7E9FEBBE725
:104C1000BDE8F883704700BF70B5044600254FF427
:104C2000B970258120806581657325730DF04CF87E
:104C3000294660604FF4167204F144000FF088F8C2
:104C400004F11C063C23A4F8A032C4F89C5228228C
:104C5000294630460FF07CF8034A044B2261636119
:104C6000A661204670BD00BF05000300E00CFF1FD9
:104C7000292A01D004207047428938B5038992B2AD
:104C80009BB29A426CD04289038992B29BB29A42FB
:104C90000DD34389048902881B1B9BB29A420FD211
:104CA00000223349334809F033FE052038BD04891A
:104CB0000288438912FA83F31B1B9BB29A42EFD3FB
:104CC000292B98BF1AB2ECD9037B03F0FF04002B09
:104CD0004BD1426803899BB2D454038901339BB200
:104CE00003810289038892B29BB29A4228BF048151
:104CF0000289438992B29BB29A4204BF0123037393
:104D00004A1E4FF0010E28311DE0456803899BB211
:104D100005F803C0038901339BB20381B0F808C0D2
:104D200003881FFA8CFC9BB29C4528BF0481B0F815
:104D300008C043891FFA8CFC9BB29C4508BF80F8D1
:104D40000CE08A420AD0037B12F801CF03F0FF0483
:104D5000002BDAD08A4280F80DE0F4D1002038BD73
:104D6000037B002B9CD10388AAE701234373C7E789
:104D7000F079010020E6FF1F0C2A01D004207047C3
:104D8000428938B5038992B29BB29A426DD042896A
:104D9000038992B29BB29A420DD343890489028857
:104DA0001B1B9BB29A420FD200223449344809F0AF
:104DB000AFFD052038BD04890288438912FA83F3C8
:104DC0001B1B9BB29A42EFD30C2B98BF1AB2ECD9A3
:104DD000037B03F0FF04002B4CD1426803899BB294
:104DE0000125D55403892B449BB203810289038892
:104DF00092B29BB29A4228BF04810289438992B23F
:104E00009BB29A4204BF012303734A1E4FF0010E66
:104E10000B311DE0456803899BB205F803C0038987
:104E200001339BB20381B0F808C003881FFA8CFCE1
:104E30009BB29C4528BF0481B0F808C043891FFA83
:104E40008CFC9BB29C4508BF80F80CE08A420AD0DB
:104E5000037B12F801CF03F0FF04002BDAD08A4263
:104E600080F80DE0F4D1002038BD037B002B9BD1EE
:104E70000388A9E701234373C7E700BF107A010045
:104E800020E6FF1F428908B5038992B29BB29A427D
:104E90003ED04289038992B29BB29A420DD3438994
:104EA000018902885B1A9BB29A420FD21D491E48A3
:104EB000002209F02DFD052008BD018902884389E3
:104EC00012FA83F35B1A9BB29A42EFD3002BEDD018
:104ED000037B03F0FF0103BB426803899BB24FF0E1
:104EE000020C02F803C0038901339BB203810289DB
:104EF000038892B29BB29A4228BF018102894389FA
:104F000092B29BB29A4204BF01230373002008BDF2
:104F1000037B002BCAD10388D8E701234373002009
:104F200008BD00BF307A010020E6FF1F2DE9F04FD9
:104F30009BB015460C4603920021532205A80EF0A3
:104F400007FF5322284600210EF002FFDFF8B8B118
:104F50000023621E019302921D469E464FF0010AF5
:104F6000029A019912F8019F02922B46002475467D
:104F70000AFA04F219EA020F14BF4FF0010E4FF0C3
:104F8000000EEE184A1C1AA8764400EBD10C00EB78
:104F9000D20716F0010F0EEB030001F0070802F034
:104FA000070204F1010400F001002B4601F10201A7
:104FB00007D01CF8546C1BF8088048EA06060CF869
:104FC000546C30B117F8540C1BF80220024307F858
:104FD000542C082C01D07546CAE7019B1033B3F559
:104FE000287F0193BCD1464D03980022012405EB94
:104FF000420339E01AA901EBD20111F9546C11F8FE
:10500000541C002E08DA1F785E7810F807C004FAE6
:1050100006F646EA0C06C6554E0608D59F78DE7899
:1050200010F807C004FA06F646EA0C06C6558F06C5
:1050300008D51F795E7910F807C004FA06F646EA2B
:105040000C06C655CE0608D59F79DE7910F807C044
:1050500004FA06F646EA0C06C655161DB6F5257F77
:1050600003F1080317D33246B2F5257FC2D3039B61
:1050700024480022591E00F15204134601E010F8A2
:10508000013B11F8012FA04283EA02030B70F6D115
:105090001BB0BDE8F08F0B0709D505EB460315F8EB
:1050A00016605B78875D04FA03F33B4383554F0733
:1050B0000AD5531D05EB430715F813607B78875D10
:1050C00004FA03F33B4383558E070AD5931D05EB82
:1050D000430715F813607B78875D04FA03F33B43BD
:1050E0008355CB070AD5D31D05EB430615F81310DE
:1050F0007378465C04FA03F333434354083276E78B
:10510000B47A0100597A0100507A010030B59BB0A1
:105110000DF1080C06AC012340F2493E4FF6B745AD
:1051200033EA01020CBFACF80050ACF800E00CF11F
:10513000020C5B006445DBB2F2D108230DEB0301E6
:10514000224610300CF0C6FF0023009303482823AA
:105150002246012103F0F6F91BB030BDD096FF1FA7
:105160002DE9F0414289038992B29BB29A42A2B0E2
:10517000044600F09F804289038992B29BB29A4212
:1051800028D2038942899B1A9BB263B36289616802
:10519000B4F89C3292B28A5C002A49D163BBA44A1B
:1051A0001278002A40F0D080B4F8A022002A00F043
:1051B0003C81AA20E11801339BB29A4281F8440055
:1051C000F8D10023A4F89C22A4F89E32A2B922B000
:1051D000BDE8F08142890188038911FA83F39B1AA3
:1051E0009BB2002BD2D1B4F89C32002BEFD0628955
:1051F000616892B28A5CDAB98E4803F065FA0546B6
:1052000012E0B4F89E325A1C2344A4F89E2293F86C
:105210004410FFF77BFFB4F89E22B4F89C32283D7F
:105220009A42ADB280F0C880282D2046E9D8CEE75A
:10523000012A44D1002BDFD12189628989B292B23F
:10524000914200F0E88000206268628920736289E0
:10525000013292B262816189228889B292B291420E
:1052600028BF6081002514E06168628992B28A5C7F
:1052700080F8442025736289013292B2628161898B
:10528000228889B292B2914228BF65810C2B00F02E
:1052900099802189628903F1010C89B292B2E018E8
:1052A00091421FFA8CF3A4F89C32DDD1227B002AB4
:1052B000DAD1EBE7037B002B95D0038865E7022A60
:1052C00018BF1A4682D1002B96D12189628989B2F2
:1052D00092B2914200F0A48000206268628920733B
:1052E0006289013292B262816189228889B292B266
:1052F000914228BF60815522C8277A2603F1010E0A
:1053000003F1020CDD1C181D591D04EB03080633C4
:1053100014FA8EFE14FA8CFC14FA85F514FA80F057
:1053200014FA81F19BB2122B88F844208EF84420A5
:105330008CF8442085F8442080F8447081F844605B
:10534000DCD1C4F89C3257E72289638992B29BB2C0
:105350009A425CD0002163686389217363890133B9
:105360009BB263816289238892B29BB29A4228BF22
:10537000618101A90DF12D05002013E062686389A8
:105380009BB2D25C207363890A7001339BB2638144
:105390006289238892B29BB29A4228BF6081013110
:1053A0008D4213D02289638992B29BB29A42E5D191
:1053B000237B002BE2D1F2E70023C4F89C3222B019
:1053C000BDE8F0810023A4F89E3215E70DF132020A
:1053D00001A92046FFF7AAFDB4F89CC24AF2EA638D
:1053E0000DF13102ADF830300DF18505EA21ACEB5D
:1053F000020001E012F8011B831814FA83F3AA4299
:1054000083F84410F6D10CF1550292B2D9E6237B11
:10541000002B9FD1ADE7227B002A7FF414AF21E758
:10542000227B002A7FF458AF65E7A4F89E22CEE6DF
:105430000AA7FF1FD096FF1F01EB4101490001F5AC
:105440009671B1F5167F28BF4FF41671A0F8A0121F
:10545000704700BF4289038992B29BB29A421DD025
:105460004289038992B29BB29A4208D34389018947
:105470000288581A80B282420AD2002070470288FD
:105480000389408912FA80F0C01A80B28242F4D3B4
:10549000074BA3FB0030C0F387007047037B002B52
:1054A000EBD10088024BA3FB0030C0F387007047AC
:1054B0004FECC44E38B500F678450446284602F055
:1054C000AFFD00B938BD284602F0B0FD0028F9D084
:1054D0000849094809F0ECF9002384F84C3C2846B7
:1054E00002F092FD04F6584002F08EFD012384F88C
:1054F000983C38BDDC7F010020E6FF1F2DE9F84312
:10550000044602F019FB04F5806002F015FB04F577
:10551000006002F011FB04F5406002F055F904F55B
:10552000426002F0FFF904F62840002502F072FC08
:1055300004F5446002F008FDC4F84C5C04F54560D5
:1055400002F046FD04F6584002F042FD04F54660C4
:1055500002F03EFD04F6684002F03AFD04F54760B3
:1055600002F036FD04F6784002F032FD04F6884978
:1055700004F5486002F02CFD04F54968484602F045
:1055800027FD404602F024FD4FF43573C4F8AC3CCF
:10559000C4F8B43C5E4BC4F8B83C45F26833C4F878
:1055A000BC3C4FF40043C4F8D03CC4F8F43CC4F80D
:1055B000FC3C584BC4F8003D47F6E423C4F8043DD6
:1055C000554BC4F8D83C554BC4F8DC3C544BC4F89C
:1055D000F83C4FF4B563C4F8B03C44F66C23C4F80F
:1055E000E03C84F8985CC4F8A45CC4F89C5CC4F803
:1055F000A85CC4F8A05CC4F8D45CC4F8C85CC4F867
:10560000C05CC4F8CC5CC4F8C45CC4F8EC5CC4F8FE
:10561000E45CC4F8F05CC4F8E85C04F6085002F0FE
:1056200071F801264FF001134FF4C871C4F81C3D06
:10563000C4F8186D04F5526002F0D0F940F6611319
:10564000A4F8403DA4F8485D84F83C5DA4F84A5DA8
:10565000A4F83E6D84F84C5D84F84D5D41F2C220A3
:105660000CF032FB4FF41667A4F8585DC4F8440DF3
:10567000A4F85A5D84F85D5D84F85C5DA4F8507D03
:105680004FF496500CF020FBC4F8540D04F556600E
:1056900002F0D6FC48462A463146A4F8805D02F066
:1056A0009BFC96222946404602F096FC3A4622E0B0
:1056B000D4F8441DB4F8483D9BB221F81300B4F867
:1056C000483D01339BB2A4F8483DB4F8481DB4F8F6
:1056D000403D89B29BB2994228BFA4F8480DB4F866
:1056E000481DB4F84A3D89B29BB2994208BF84F87C
:1056F0004C6D013A09D094F84C3D03F0FF00002BAB
:10570000D6D0013A84F84D6DF5D12046BDE8F88336
:10571000F96BFFFFB505FFFF0080FFFF5D3BFFFF5B
:105720000000FFFFF0B50446BFB0484802F0CCFFD0
:10573000B4F85A1DB4F8582D89B292B2914266D08D
:10574000B4F85A2DB4F8583D92B29BB29A4257D34E
:10575000B4F85A2DB4F8501DB4F8583D11FA83F33B
:105760009B1A9BB20A2846D9632B44D9831E9BB24D
:10577000642B28BF64235A1E02AF92B20DF10A01B6
:105780003D4601EB420600201CE0D4F8541DB4F85D
:105790005A2D92B231F912C084F85C0DB4F85A2D2A
:1057A00025F802CB013292B2A4F85A2DB4F85A1D52
:1057B000B4F8502D89B292B2914228BFA4F85A0D84
:1057C000B54211D0B4F8581DB4F85A2D89B292B22E
:1057D0009142DAD194F85C2D02F0FF0C002AD4D16A
:1057E00025F802CBB542EDD10022009217483A4687
:1057F0000A2102F0A7FE94F83C3D7BB93FB0F0BD12
:10580000B4F8583DB4F85A2D9B1A9BB2AAE794F805
:105810005C3D002BEFD0B4F8503DA3E704F5526592
:10582000284602F063F94F28E8D902AF3C463EAE65
:1058300021462846033402F02FF9B442F8D1044837
:10584000F022394608F000FF3FB0F0BDD096FF1FB0
:1058500020E6FF1F38B50446002500F5456084F8B2
:105860004C5C02F0D1FB04F6584002F0CDFB04F68C
:10587000684002F0C9FB04F5476002F0C5FB04F67E
:10588000784002F0C1FB04F5486002F0BDFB04F66D
:10589000884002F0B9FB04F5496002F0B5FB04F55D
:1058A000406002F039F804F5806002F099FA04F5DE
:1058B000006002F095FA204602F092FA04F5446086
:1058C00002F082FBA4F8585D04F55660A4F85A5D16
:1058D00084F85D5D84F85C5D02F0CAFB04F55260FB
:1058E00002F026F904F6284002F028FB84F8985CC0
:1058F000A4F8805D38BD00BF2DE9F04F83B090461D
:105900009DF834409DF8402080F84D2CC4EB0414E1
:105910009DF8442080F84E2CA4009DF848209DF866
:10592000306080F84F2CA4B200F5466B054600228B
:1059300058460F46214601939DF838909DF83CA0AB
:1059400002F04AFBC6EB0611890089B2002205F578
:10595000456002F041FB019B5CB94246394628464E
:10596000CDF834A0CDF8309003B0BDE8F04F02F090
:10597000FBB8584602F042FB019BEEE72DE9F041EF
:1059800082B004469DF8208001930D461646002102
:10599000BDF82420009200F678409DF8287002F0AF
:1059A0001BFBDDE90023B8F1000F0AD1324629467E
:1059B00004F580600997089702B0BDE8F04102F055
:1059C000D3B8414604F54760009302F005FB009B05
:1059D000ECE700BF2DE9F04F85B09A469DF84C30BA
:1059E00080F8183D9DF8503080F8193D9DF85430EE
:1059F00080F81A3D9DF8583080F81B3D9DF86430C2
:105A0000A0F81C3D9DF83C309DF844B002939DF8F1
:105A10005C309DF840C09DF84890009304469DF886
:105A20006C300193154600F658400022CDF80CC0AA
:105A30009DF838709DF860609DF8688002F0CCFA9F
:105A40005946002204F6684002F0C6FA0022494690
:105A500004F5486002F0C0FA294604F5446002F0FB
:105A60007BFA2A46414604F6085001F055FE01989B
:105A70000099A4F83E0D324604F6284002F0D2F90F
:105A8000029B3A46514604F5406001F0ADFE10B16C
:105A900005B0BDE8F08F039A514604F5426005B0A9
:105AA000BDE8F04F01F042BF10B484469DF80840B5
:105AB000BDF80400ACF81E2D0294019401241A468E
:105AC0008CF83C4D03465DF8044B0CF5006002F089
:105AD0004BB800BF70B504460D4600F5456002F0B6
:105AE00097FA294604F6584002F092FA294604F53E
:105AF000466002F08DFA294604F6684002F088FA02
:105B0000294604F5476002F083FA294604F67840F6
:105B100002F07EFA04F68846294604F5486002F051
:105B200077FA3046294602F073FA04F549602946AF
:105B300002F06EFA304602F073FA00B970BD3046DA
:105B400002F074FA0028F9D094F84C1C034808F0CD
:105B5000C1FD3046BDE8704002F050BA20E6FF1F9C
:105B600010B5044600294CD102B910BD2D482E496C
:105B700008F09EFE072384F84C3C4FF49662012007
:105B800022E0D4F8541DB4F8583D9BB221F813C05C
:105B9000B4F8583D01339BB2A4F8583DB4F8581DF1
:105BA000B4F8503D89B29BB2994228BFA4F858CDB1
:105BB000B4F8581DB4F85A3D89B29BB2994208BF57
:105BC00084F85C0D013A09D094F85C3D03F0FF0CB9
:105BD000002BD6D0013A84F85D0DF5D104F658407B
:105BE00002F00CFA04F5496002F00EFA04F688405F
:105BF00002F004FA94F84C1C0A48BDE8104008F082
:105C000069BD0A49074808F053FE0223084884F892
:105C10004C3C012102F080FD0548012102F088FD85
:105C2000DCE700BF20E6FF1F08800100F07F0100D5
:105C3000D096FF1F38B5044631B100F658452846C6
:105C400002F0EEF9E0B938BD17480D4602F064FDE8
:105C50001548294602F06CFD1449154808F028FE45
:105C6000032384F84C3C04F6784002F0C7F994F81A
:105C70003C3D002BE7D0BDE838400D4808F04EBD54
:105C8000284602F0D3F90028DDD00A49084808F078
:105C90000FFE042384F84C3C284602F0B5F994F832
:105CA0003C3D002BE7D138BDD096FF1F348001006A
:105CB00020E6FF1F2080010070B50446A1B11848FE
:105CC000012102F029FD1648012102F031FD15489D
:105CD000154908F0EDFD022384F84C3C04F67840A9
:105CE000BDE8704002F090B900F6784630460D46A7
:105CF00002F096F900B970BD304602F097F900281D
:105D0000F9D00A49074808F0D3FD304684F84C5CC6
:105D100002F07AF904F65840BDE8704002F074B918
:105D2000D096FF1F20E6FF1FF07F0100DC7F0100FF
:105D300038B5044631B100F65845284602F070F9EE
:105D400068B938BD0E480F4908F0B2FD082384F841
:105D50004C3C04F67840BDE8384002F04FB9284684
:105D600002F064F90028ECD00548074908F0A0FDCE
:105D7000092384F84C3C2846BDE8384002F044B979
:105D800020E6FF1F688001005080010038B590F8C0
:105D90004C3C04460D460A2B09D8DFE803F04B08BB
:105DA0005109060608575D2B3B00002D63D038BD16
:105DB0002946FFF781FF94F84C3C002BF7D104F5FE
:105DC0004965284602F02CF918B994F8983C002B44
:105DD00067D1284602F024F90028E8D0284602F0CE
:105DE00025F90028E3D0284602F00EF9002384F8B4
:105DF000983C38BD002ADAD13149324808F058FDC4
:105E00000A2384F84C3C04F6784002F0F7F894F842
:105E10004C3CD2E7002A48D02B492A4808F048FDDC
:105E2000092384F84C3C04F6784002F0EDF894F82D
:105E30004C3CC2E72946FFF793FE94F84C3CBCE784
:105E40002946FFF7F7FE94F84C3CB6E71146FFF7FA
:105E50006FFF94F84C3CB0E762B31C49194808F056
:105E600027FD072384F84C3C04F6784002F0CCF878
:105E700094F84C3CA1E71648294602F04DFC144822
:105E8000294602F055FC13490E4808F011FD052380
:105E900084F84C3C04F6784002F0B0F894F84C3C9E
:105EA0008BE7284602F0AAF893E7FFF703FB94F884
:105EB0004C3C82E7FFF7FEFA94F84C3C7DE700BFCC
:105EC000A080010020E6FF1F508001000880010033
:105ED000D096FF1F8480010070B5044616460D461B
:105EE000002947D090F8803D002B7ED090F8813D6E
:105EF000002E78D0002B3CD194F8803D002B00F090
:105F000089804FF49660012122E0D4F8542DB4F832
:105F1000583D9BB222F813C0B4F8583D01339BB2F0
:105F2000A4F8583DB4F8582DB4F8503D92B29BB245
:105F30009A4228BFA4F858CDB4F8582DB4F85A3D69
:105F400092B29BB29A4208BF84F85C1D013809D016
:105F500094F85C3D03F0FF0C002BD6D0013884F898
:105F60005D1DF5D1012384F8813D15B994F8803D7C
:105F70001BBB70BD42B190F8813D002BF6D194F867
:105F8000803D002BBDD145E090F8803DABB990F845
:105F9000813D002BEDD03B483B4908F089FC0023B4
:105FA00084F84C3C04F6884002F02EF801220023CD
:105FB00084F8982C84F8813D70BD3448002102F0AB
:105FC000ABFB3248002102F0B3FB94F8815D002D59
:105FD0004DD094F83C3D002284F8802D5BBB002E10
:105FE000C7D194F8813D83B970BD2848012102F0E2
:105FF00093FB2648012102F09BFB94F8813DF3B10D
:10600000012384F8803D002EB3D194F8803D002B0D
:10601000CCD1C0E71E491B4808F04AFC072304F610
:10602000884084F84C3C01F0E9FF94F84C1C15487A
:1060300008F050FB65E7134808F070FBCFE71549FF
:10604000104808F035FC022384F84C3C04F68840E4
:1060500001F0D4FF94F84C1C0A4808F03BFB0122E5
:1060600094F8813D84F8802D002EBCD042E705488D
:10607000054908F01DFC84F84C5C04F6884001F0EA
:10608000C3FFA6E720E6FF1FDC7F0100D096FF1FBD
:1060900008800100F07F010038B500F54665044630
:1060A000284601F0BDFF20B1284601F0BFFF48B9E6
:1060B00038BD0A480A4908F0FBFB2046BDE83840D5
:1060C00001F07ABE0649054808F0F2FB204601F0CF
:1060D00073FE2846BDE8384001F090BF20E6FF1F60
:1060E000BC80010038B5044631B100F66845284649
:1060F00001F09CFF70BB38BD0D46244802F00CFB3C
:106100002248294602F014FB2149224808F0D0FB1E
:1061100004F6684084F84C5C01F076FF04F65840C1
:1061200001F072FF04F5476001F06EFF04F5456071
:1061300001F06AFF04F6884001F066FF94F83C3DE8
:10614000012284F8982C002BD5D0BDE838401148A6
:1061500008F0E4BA10490F4808F0AAFB022384F8BB
:106160004C3C284601F050FF94F84D3C002BC2D027
:1061700094F84F3C002BBED02046FFF78DFF04F56E
:106180004560BDE8384001F039BF00BFD096FF1F21
:10619000DC7F010020E6FF1FF07F010038B50446D8
:1061A000D1B100F65845284601F03AFF002835D114
:1061B00004F54565284601F033FF00B938BD28468F
:1061C00001F034FF0028F9D02046FFF765FF28468C
:1061D000BDE8384001F012BF1E480D4602F09CFA9F
:1061E0001C48294602F0A4FA1B491C4808F060FB31
:1061F000032384F84C3C04F6784001F0FFFE94F849
:106200003C3D002BD4D0154804F5456508F086FACE
:10621000284601F005FF0028D0D0D0E7284601F03D
:1062200005FF0028C4D00E490C4808F041FB0423A8
:1062300084F84C3C04F5476001F0E6FE284601F086
:10624000E3FE04F5446001F0B9FE94F83C3D002BF8
:10625000AED0D8E7D096FF1F3480010020E6FF1FA4
:106260002080010070B5044631B32E48012102F0B0
:1062700053FA2C48012102F05BFA2B482B4908F015
:1062800017FB022384F84C3C04F6784001F0BCFE76
:1062900004F54565284601F0C3FE00B970BD2846E7
:1062A00001F0C4FE0028F9D02046FFF7F5FE28468D
:1062B000BDE8704001F0A2BE00F67845284601F026
:1062C000AFFE0028E4D0284601F0B0FE0028DFD061
:1062D0001548174908F0ECFA04F547660B2384F8D3
:1062E0004C3C304601F09CFEB0B912490E4808F013
:1062F000DFFA04F5806001F05FFD304601F084FEB6
:10630000284601F081FE04F6584001F07DFE04F5B8
:10631000486001F073FEBBE7304601F087FE0028BD
:10632000EED0E2E7D096FF1F20E6FF1FF07F0100CE
:10633000CC800100DC80010038B5044631B100F6A4
:106340006845284601F072FEF8B938BD1C480D4674
:106350001C4908F0ADFA04F6684084F84C5C01F082
:1063600053FE04F6584001F04FFE04F5476001F07B
:106370004BFE04F5456001F047FE04F6884001F04D
:1063800043FE012384F8983C38BD0F490C4808F0BF
:106390008FFA072384F84C3C284601F035FE94F828
:1063A0004D3C002BD1D094F84F3C002BCDD0204653
:1063B000FFF772FE04F54560BDE8384001F01EBEEF
:1063C00020E6FF1FDC7F01000880010038B504468D
:1063D000C9B100F65845284601F022FE30BB04F54D
:1063E0004565284601F01CFE00B938BD284601F07D
:1063F0001DFE0028F9D02046FFF74EFE2846BDE8D6
:10640000384001F0FBBD1548154908F051FA082342
:1064100004F6784084F84C3C04F5456501F0EEFD47
:10642000284601F0FDFD0028DFD0DFE7284601F017
:10643000FDFD0028D3D00B49084808F039FA09239C
:1064400084F84C3C04F5476001F0DEFD284601F07D
:10645000DBFD04F5446001F0B1FDC0E720E6FF1F5D
:10646000688001005080010070B50446F1B12A48EF
:106470002A4908F01DFA072384F84C3C04F67840BA
:1064800001F0C2FD04F54565284601F0C9FD00B9DB
:1064900070BD284601F0CAFD0028F9D02046FFF75C
:1064A000FBFD2846BDE8704001F0A8BD00F6784528
:1064B000284601F0B5FD0028E4D0284601F0B6FDDD
:1064C0000028DFD01448164908F0F2F904F54766B1
:1064D0000B2384F84C3C304601F0A2FDB0B91149C1
:1064E0000D4808F0E5F904F5006001F065FC304660
:1064F00001F08AFD284601F087FD04F6584001F0BE
:1065000083FD04F5486001F079FDBBE7304601F0FA
:106510008DFD0028EED0E2E720E6FF1F0880010095
:10652000CC800100E880010038B5044699B104F53B
:106530004565284601F074FD00B938BD284601F0D4
:1065400075FD0028F9D02046FFF7A6FD2846BDE8D6
:10655000384001F053BD0D480D4602F0DDF80B4800
:10656000294602F0E5F80A490A4808F0A1F994F82A
:106570004E3C052284F84C2C23B904F6784001F0F7
:106580003DFDD4E72046FFF787FDF6E7D096FF1FD5
:106590008480010020E6FF1F38B5044631B32B4844
:1065A000012102F0B9F82948012102F0C1F8284878
:1065B000284908F07DF9042384F84C3C04F678401F
:1065C00001F022FD04F54565284601F029FD00B9DA
:1065D00038BD284601F02AFD0028F9D02046FFF7F3
:1065E0005BFD2846BDE8384001F008BD00F678455F
:1065F000284601F015FD0028E4D0284601F016FDDC
:106600000028DFD01449124808F052F90B2384F80F
:106610004C3C04F5446001F0D7FC10490C4808F0EC
:1066200047F904F5806001F0C7FB284601F0ECFC57
:1066300004F5476001F0E8FC04F6584001F0E4FC82
:1066400004F5486001F0DAFCBCE700BFD096FF1FFC
:1066500020E6FF1F20800100CC800100DC800100CB
:1066600038B5044699B104F54565284601F0D8FCD3
:1066700000B938BD284601F0D9FC0028F9D02046E1
:10668000FFF70AFD2846BDE8384001F0B7BC0648D0
:10669000064908F00DF90A2384F84C3C04F67840CA
:1066A00001F0ACFCDFE700BF20E6FF1FA080010087
:1066B00038B50446F1B12748274908F0F9F809230D
:1066C00084F84C3C04F6784001F09EFC04F54565E6
:1066D000284601F0A5FC00B938BD284601F0A6FC0B
:1066E0000028F9D02046FFF7D7FC2846BDE83840FF
:1066F00001F084BC00F67845284601F091FC0028A2
:10670000E4D0284601F092FC0028DFD0134911485C
:1067100008F0CEF80B2384F84C3C04F5446001F0FB
:1067200053FC0F490B4808F0C3F804F5006001F072
:1067300043FB284601F068FC04F5476001F064FC67
:1067400004F6584001F060FC04F5486001F056FC86
:10675000BCE700BF20E6FF1F50800100CC80010095
:10676000E880010070B50446002938D115466AB9A1
:1067700000F54866304601F053FC00283DD104F591
:106780004565284601F04CFCE0B970BD2C492D4808
:1067900008F08EF807232C4984F84C3C294808F06F
:1067A00087F804F5806001F01BFB04F5006001F040
:1067B00017FB04F6584001F021FC04F5476001F096
:1067C0001DFCDCE7284601F031FC0028DDD0204626
:1067D000FFF762FC2846BDE8704001F00FBC1B4883
:1067E000012101F099FF1948012101F0A1FF184989
:1067F000144808F05DF80223CDE7304601F016FC9E
:106800000028BCD013490F4808F052F8304684F8ED
:106810004C5C01F0F9FB04F6884001F0F5FB94F8BC
:106820004E3C43B904F54565284601F0EDFB0123D4
:1068300084F8983CA5E72046FFF72EFCF2E700BF5E
:106840000880010020E6FF1FF8800100D096FF1F9E
:10685000F07F0100DC7F010038B50446002946D1F5
:1068600002B938BD00F66845284601F0BFFB002894
:1068700040F0BA807449754808F01AF894F84D3C15
:10688000072284F84C2C002B40F0C5804FF4966210
:10689000012023E0D4F8541DB4F8583D9BB221F8F0
:1068A00013C0B4F8583D01339BB2A4F8583DB4F876
:1068B000581DB4F8503D89B29BB2994228BFA4F844
:1068C00058CDB4F8581DB4F85A3D89B29BB29942DC
:1068D00008BF84F85C0D013A00F0A18094F85C3D9B
:1068E00003F0FF0C002BD5D084F85D0DF3E700F624
:1068F0006845284601F07AFB00285FD15449534887
:1069000007F0D6FF94F84D3C022284F84C2C002B63
:1069100040F096804FF49662012022E0D4F8541D96
:10692000B4F8583D9BB221F813C0B4F8583D013378
:106930009BB2A4F8583DB4F8581DB4F8503D89B244
:106940009BB2994228BFA4F858CDB4F8581DB4F8AA
:106950005A3D89B29BB2994208BF84F85C0D013A56
:1069600009D094F85C3D03F0FF0C002BD6D0013A1F
:1069700084F85D0DF5D104F6584001F03FFB04F5B5
:10698000476001F03BFB04F5456001F037FB04F57F
:10699000496001F039FB2F48012101F0BDFE2D486F
:1069A000012101F0C5FE04F6884001F027FB94F8B0
:1069B0004C1C2648BDE8384007F08CBE26492348C9
:1069C00007F076FF012384F84C3C284601F016FBC3
:1069D00094F84D3C13B194F84F3C8BB394F84C3C75
:1069E000013B012B96D938BD1C49184807F060FFC0
:1069F000062384F84C3C284601F000FB94F84D3CFB
:106A000013B194F84F3C33B194F84C3C063B012B46
:106A10007FF63CAF38BD2046FFF73EFBF4E704F6B7
:106A2000584001F0EBFA04F5476001F0E7FA04F58D
:106A3000456001F0E3FA04F5496001F0E5FAB2E7D8
:106A40002046FFF729FBC9E70880010020E6FF1F69
:106A5000F07F0100D096FF1F048101001C8101001E
:106A600038B5044690F84C0C0B460B2819D8DFE8D3
:106A700000F01920272E353C434A51585F0619462D
:106A80002046FFF76FFE94F84C3C53B904F5806044
:106A900001F0B0F928B904F5006001F0ABF9002865
:106AA0004DD038BD19462046FFF7D6FE94F84C3C31
:106AB000EBE719462046FFF715FB94F84C3CE4E75A
:106AC00019462046FFF76AFB94F84C3CDDE719466F
:106AD0002046FFF7C7FB94F84C3CD6E71946204602
:106AE000FFF722FD94F84C3CCFE719462046FFF70C
:106AF00053FD94F84C3CC8E711462046FFF71CFCB8
:106B000094F84C3CC1E711462046FFF75FFC94F82F
:106B10004C3CBAE711462046FFF7A6FC94F84C3CE3
:106B2000B3E711462046FFF79BFD94F84C3CACE7D9
:106B300011462046FFF7BCFD94F84C3CA5E72046E3
:106B400001F058F90028ACD104F54965284601F058
:106B500067FA10B994F8983C83B9284601F060FAB6
:106B600000289ED0284601F061FA002899D02846D6
:106B700001F04AFA002384F8983C38BD284601F019
:106B80003DFAEAE72DE9F04F2DED028B044690F82F
:106B90001A0D85B00F4616461D4608B181F0010753
:106BA00029462046FEF796FF002D00F01E8105F1D4
:106BB000FF3804F628435FFA88F8DFF8C89308EE38
:106BC000103A06EB480804F5566A023E04F5406B9D
:106BD00036F9025F94F81B2DB4F93E1D2D0295FB8A
:106BE000F1F52DB2002A40F03D810DF10E01504625
:106BF00001F0BCFA002800F0128194F83C2D002A24
:106C000000F00D8194F8181D012900F0338102294C
:106C100000F0BF81002900F0F38029465846019218
:106C200000F008FE99F80010019A0A2900F0E880A7
:106C300008B10246384694F8191D002940F00D812C
:106C4000CF4B1978002900F0BA8101462046FFF7A2
:106C500007FF94F84C2C002A00F0C48099F800201B
:106C60000A2A40F0BF8094F8802D22B194F83C2D80
:106C7000002A40F0B68194F8812D002A00F0B280FD
:106C8000BDF80E20B4F81E1DD4F8A45CD4F8AC0CEA
:106C900011FB02F1D4F8B02C09B205FB02F200FBA3
:106CA0000122C4F8A41CD4F89C0CD4F8B41CC4F879
:106CB0009C5C00FB0122D4F8A81CD4F8B80CD4F8D2
:106CC000C85C00FB1122D4F8A00CC4F8A01CD4F8B6
:106CD000BC1C00FB1122D4F8D41CD4F8D00C05FB4A
:106CE00001F1D21302F30E0212B2C4F8A82CC4F8B8
:106CF000C82C00FB0212D4F8C00CD4F8D81CC4F87D
:106D0000C05C00FB0122D4F8CC1CD4F8DC0CD4F815
:106D1000EC5C00FB1122D4F8C40CC4F8C41CD4F8F9
:106D2000E01C00FB1122D4F8F81CD4F8F40C05FB8D
:106D300001F1D21302F30E0212B200FB0211C4F8E9
:106D4000CC2CD4F8F00CC4F8EC2CD4F8E42CD4F807
:106D5000FC3CC4F8E45C02FB0311D4F8002D02FBF8
:106D60001015D4F8E81CD4F8042DC4F8E80C01FB85
:106D70001255ED1305F30E052AB2C4F8F02C04F5F4
:106D8000496001F04DF9014604F5426000F010FE43
:106D900094F85C2D02F0FF01002A40F01E81284487
:106DA000D4F8545DB4F8582D92B225F81200B4F816
:106DB000582D013292B2A4F8582DB4F8580DB4F8F9
:106DC000502D80B292B2904228BFA4F8581DB4F85A
:106DD000581DB4F85A2D89B292B2914204BF0122D3
:106DE00084F85C2D46457FF4F3AE05B0BDEC028B14
:106DF000BDE8F08F27B999F800200A2AF2D10022C5
:106E000094F8191D002940F0BF805D4B19780029C6
:106E100000F0B18039462046FFF722FE1EE794F8C5
:106E2000182D012A25D0022A00F08F80002AE1D0F7
:106E30002946584600F0FEFC0246002800F0DC809F
:106E4000002FDCD099F800200A2AD8D0384600223A
:106E500094F8191D00293FF4F3AE01462046FFF7D0
:106E60003BF8F6E618EE100A294600F0DFFF074669
:106E7000BBE6002229465846019200F0DBFC94F85C
:106E80004C1D019A01F0FF0C002940F09D80D4F8C0
:106E9000443DB4F8481D89B223F81150B4F8481D98
:106EA000013189B2A4F8481DB4F848EDB4F8401D8A
:106EB0001FFA8EFE89B28E4528BFA4F848CDB4F8DB
:106EC00048CDB4F84A1D1FFA8CFC89B28C4504BF2A
:106ED000012184F84C1DB4F848CDB4F84A1D1FFABE
:106EE0008CFC89B28C4573D0D4F8445DB4F84A1D4B
:106EF00089B235F91150002184F84C1DB4F84ACDFF
:106F00000CF1010C1FFA8CFCA4F84ACDB4F84AED40
:106F1000B4F840CD1FFA8EFE1FFA8CFCE64528BF60
:106F2000A4F84A1D99F8001012BB08BB0A297FF487
:106F300059AF94F8191DB1B9114B1978002939D0FE
:106F400001462046FFF78CFD88E62946584600F0AA
:106F500071FC002856D0002F5BD13A4694F8191DD9
:106F600000200029E8D001462046FEF7B5FF75E66F
:106F70000A29DED05FE639462046FEF707FF6DE6B8
:106F8000550EFF1F09A7FF1F39462046FEF7A4FF35
:106F900064E629465846019200F04CFC99F800102E
:106FA000019A0A297FF444AE0028C2D0C7B33A46FA
:106FB0003846BEE701462046FEF7E8FE4EE60146AB
:106FC0002046FEF7E3FE44E6012184F84D1D82E7EA
:106FD00094F84C1D002987D1A4E7012284F85D2D87
:106FE00000E7294604F6085000F09EFB014604F530
:106FF000526000F007FD3EE699F800100A293FF4C0
:10700000FFAEEFE699F800200A2A7FF4EBAE0022EB
:107010008FE799F800200A2A3846F8D0002217E7AF
:1070200002469BE72DE9F04F2DED028B044690F8C8
:107030001A0D85B00E4615461F4608B181F00106AF
:1070400039462046FEF746FD002F00F06581013FDE
:10705000FFB205EB4703019304F62843DFF82083D2
:1070600008EE103A04F55669023D04F5406AA3465D
:1070700035F9027F9BF81B2DBBF93E1D3F0297FBA4
:10708000F1F73FB2002A40F072810DF10E0148463F
:1070900001F06CF8002800F044819BF83C4D002C76
:1070A00000F03F819BF8182D012A00F06C81022A24
:1070B00000F05A8252B33946504600F0BBFB98F8B4
:1070C00000200A2A014621D009B10C4631469BF81E
:1070D000192D002A40F04681A84B1A78002A40F06A
:1070E000A28222465846FEF751FE9BF84C2C002AFD
:1070F00000F00E8198F800100A2920D008E12EB97E
:1071000098F800200A2A40F0038100249BF8192DEA
:10711000002A40F02382994B1A78002A00F0188246
:10712000224631465846FFF79BFC98F800200A2A71
:1071300040F0EE809BF84C2C002A00F0FF81911F5C
:10714000C9B20129BBF91C4D8C4B40F2AE811978B4
:10715000002900F03C82013AD2B2012A00F24782B3
:1071600039460BF6085000F0DFFA9BF83C2D074635
:107170002AB19BF84C2C013A012A40F2978217FB66
:1071800004F73FB2584600F037FE002800F09E8119
:107190000BF58064584600F02FFE002800F0AA810D
:1071A000204600F029FE002800F0B681DBF8A41C80
:1071B000DBF8B02CDBF8AC0CCBF8A47C01FB02F2C2
:1071C00000FB0722DBF89C0CCBF89C1CDBF8B41C02
:1071D000DBF8D07CDBF8E43C00FB0122DBF8A81CE8
:1071E000DBF8B80C00FB1122DBF8A00CCBF8A01CDC
:1071F000DBF8BC1C00FB1122DBF8C80CDBF8D41C4C
:10720000D21300FB01F102F30E0212B2CBF8A82C4C
:10721000CBF8C82C07FB0212DBF8C07CDBF8D81CCB
:10722000CBF8C00C07FB0122DBF8DC0CDBF8CC1C34
:10723000DBF8EC7C00FB1122DBF8C40CCBF8C41C9F
:10724000DBF8E01C00FB1122DBF8F81CDBF8F40C87
:1072500001FB07FCD21302F30E0212B200FB02CCB8
:10726000DBF8FC0CDBF8F01CCBF8CC2C03FB00CCDF
:10727000DBF8000DCBF8E47CCBF8EC2C00FB11C75D
:10728000DBF8042DDBF8E80CCBF8E81C00FB1277E8
:10729000FF1307F30E073AB2CBF8F02C584600F074
:1072A000ABFD002800F076810BF5496000F0B8FED8
:1072B00001460BF5426000F07BFB9BF85C2DBFB2F2
:1072C00002F0FF01002A40F061810744DBF8540D11
:1072D000BBF8582D92B220F81270BBF8582D01322D
:1072E00092B2ABF8582DBBF8580DBBF8502D80B2B8
:1072F00092B2904228BFABF8581DBBF8581DBBF89E
:107300005A2D89B292B2914204BF01228BF85C2DB2
:10731000019B9D427FF4ACAE05B0BDEC028BBDE895
:10732000F08F9BF8184D012C2CD0022C00F094808B
:10733000002C3FF4E4AE3946504600F07BFA044698
:10734000002800F06A81002E3FF4DFAE98F800209C
:107350000A2A3FF4DAAE314600249BF8192D002AA0
:107360003FF4BAAE22465846FEF7B6FDBDE618EE2B
:10737000100A394600F05AFD064686E6550EFF1FF4
:1073800009A7FF1F00243946504600F053FA9BF826
:107390004C2D02F0FF01002A40F01581DBF8443D3E
:1073A000BBF8482D92B223F81270BBF8482D013279
:1073B00092B2ABF8482DBBF848CDBBF8402D1FFA70
:1073C0008CFC92B2944528BFABF8481DBBF8481D11
:1073D000BBF84A2D89B292B2914204BF01228BF8C8
:1073E0004C2DBBF8481DBBF84A2D89B292B2914290
:1073F00000F0E380DBF8441DBBF84A2D92B231F96E
:10740000127000218BF84C1DBBF84A2D013292B24C
:10741000ABF84A2DBBF84ACDBBF8402D1FFA8CFCC7
:1074200092B2944528BFABF84A1D98F8002054BB8F
:1074300048BB0A2A7FF46CAF9BF8192D002A40F054
:107440000A819E4B1A78002A00F0F28001462246FB
:107450005846FFF705FB68E63946504600F0EAF962
:107460000146002800F0C580002E40F0E780344639
:107470009BF8192D0021002A00F0C68022465846AC
:10748000FEF72AFD51E60A2AD6D09BF8192D002ACC
:1074900040F0DB80894B1A78002A00F0FC8001461E
:1074A00022465846FFF7DCFA1FE61A78BDF90E703F
:1074B000BBF91E4D002A7FF453AE17FB04F4584667
:1074C00027B200F099FC00287FF462AE0BF5006053
:1074D00000F092FC0BF5806400287FF45BAE204640
:1074E00000F0E2FB384407B2584600F085FC002863
:1074F0007FF456AE204600F07FFC00287FF450AEAB
:107500000BF5006000F0D0FB384407B2204600F0D5
:1075100073FC00287FF44AAE0BF5006000F06CFCB1
:1075200000287FF443AE9BF84C2C5846002A40F0CC
:10753000B88000F0B9FB384407B237E60BF580603D
:1075400000F058FC002800F08C809BF84C2CF6E5ED
:10755000224631465846FEF719FCE6E522463146FA
:107560005846FEF7B9FCE0E53946504600F062F9AE
:1075700098F800200A2A01467FF4A6AD00283ED0E4
:10758000002E00F099803446314638E001228BF815
:107590005D2DBDE6204600F02FFC00287FF484AE70
:1075A0000BF5006000F028FC00287FF47DAE0BF5A1
:1075B000446000F0D5FC074476E69BF84C2D002A89
:1075C0007FF418AF31E701228BF84D2D09E79BF8C6
:1075D0003C1D00293FF49CAE013AD2B2012A3FF68D
:1075E00097AE39460BF5526000F00CFA90E6002792
:1075F000C8E598F800200A2A7FF48AAE00249BF898
:10760000192D002A7FF43AAF2C4B1A78002A3DD06E
:1076100022465846FFF724FA87E598F800200A2A00
:107620003FF474AD74E622465846FFF719FA5CE55C
:10763000014622465846FEF7A9FB76E598F8002059
:107640000A2A3146DAD0002487E601462246584607
:10765000FEF742FC49E5014622465846FEF73CFC4F
:1076600063E50BF5006000F0C5FB00287FF46DAF0B
:10767000584600F0BFFB00287FF467AF0BF5496068
:1076800000F0CEFC00287FF460AF41E62246584669
:10769000FEF77CFB49E5014622465846FEF776FB9D
:1076A00023E500F045FB384407B27FE501460BF5C2
:1076B000526000F0A7F962E50446D9E6550EFF1FB7
:1076C00010B490F8194D1CB15DF8044BFFF75ABA8D
:1076D0005DF8044BFFF7A6BC08B500F5566000F056
:1076E000ADFD034BA3FB0030C0F3C71008BD00BFC6
:1076F0008988888808B500F5566000F0C3FC002032
:1077000008BD00BF00224FF4804102608180827179
:1077100082600273704700BFC9014B42D2010180F1
:1077200043808280704700BFB0F9002092B30346C7
:10773000807910B498B98A422EDC214AB3F904103A
:107740001068012200FB01F1C9139A7101F30F01C6
:107750001A7308B214469C605DF8044B70479A682F
:10776000B2F5166F02F101041ED81A7B1448B3F962
:10777000041050F822000132D2B200FB01F10B2AB2
:107780004FEAE1311A7301F30F0108B2E3D9002285
:107790001A73E0E708467047B3F902208A42CCDA50
:1077A00008465DF8044B704742F6DF6294429C60E5
:1077B00003D9002199710846F3E70020CCE700BF08
:1077C00034810100FFFFFFFF9FED057B002280ED6C
:1077D000007BC0E902220282426182610277704727
:1077E000000000000000000030B500240025C0E9C2
:1077F00000450F4D4FF0000C2C464FF0430E06E0B5
:107800000CF1010CBCF1320F0FD014F810EF7145E0
:10781000F6D105EB0C15D5E90214C0E9001421439B
:1078200003D0C0E90223002030BD042030BD00BFDA
:10783000888101002DE9F041D0E90067456983693D
:1078400085610446EA17008A05FB07FC01EB610825
:1078500006FB02CCA5FB06218C440130D20F80B27E
:1078600041F2707E42EA4C0202F31E02C3EB420177
:1078700041447045208282B0207F616102D002B015
:10788000BDE8F08185FB01C24FEADC7C4CEA420C8A
:1078900081FB0112C90F41EA420101F31E0285FB7F
:1078A0000551ED0F0CF31E0C45EA41050CFB07FEDC
:1078B0004FEAEC7106FB01EEACFB06C6B6444FEA9C
:1078C000DC7C05F31E052A444CEA4E0CA3680CF33D
:1078D0001E0CA2EB4C0200B1E3689342CCBF002522
:1078E00001258542257706D1002323826361A361A8
:1078F00002B0BDE8F0810648064900951BB212B2FD
:1079000007F06CF80023207F23826361A361EFE717
:1079100020E6FF1F64810100002343618361037738
:107920000382704700220260426070472DE9F041F7
:107930000023074615461D48432404E00133322B3B
:1079400031D010F83340A142F8D1184E386806EB18
:10795000C3067388BB8010B10AF0B8F9BB88580021
:107960000AF0B2F9BB883860D3B105EB45030024B7
:1079700005EB8305A04640460BF0C6FEA1B23A686F
:1079800080FB0530DB0F43EA400303F30F0322F8CB
:1079900011300134BA887168A3B29A428844EAD897
:1079A0000020BDE8F0810420BDE8F081A88401003A
:1079B000C288B0F804C0531C10B49BB20468C380E2
:1079C0009C4598BF002334F91220C38009B152426C
:1079D00012B210465DF8044B704700BF38B5002561
:1079E00004460581018045814573057301EB410023
:1079F0000AF06AF904F1100325766060256163617D
:107A0000204638BD037E01F50061002B3BD0032BDF
:107A100031D130B504694269214301611578547848
:107A200092F802E0027B02F0FF0C002A31D141689B
:107A3000028992B202EB42028D540A44547082F8D9
:107A400002E00289013292B202810189028889B280
:107A500092B2914228BFA0F808C00189428989B238
:107A600092B2914204BF0122027301330021DBB2C2
:107A70000161037630BD0133DBB2062B037628BFEC
:107A800000230376704701330903DBB201610376FB
:107A9000704701224273E8E70289438992B29BB2A0
:107AA0009A4210B50446084619D0616863899BB2B2
:107AB00003EB43031944032207F082FE00212173E4
:107AC000638901339BB263816289238892B29BB23E
:107AD0009A424FF0010328BF6181184610BD227BF6
:107AE00002F0FF03002AE0D1184610BD4289038945
:107AF00092B29BB29A4212D04289038992B29BB24F
:107B00009A4204D203894289981A80B27047438905
:107B10000288008912FA80F0C01A80B27047027B96
:107B200002F0FF030AB1008870471846704700BF93
:107B300000230376704700BF38B50446002500F8DF
:107B4000015B4FF47A7229460CF002F9A4F8EA536B
:107B5000C4F8EC53A4F8F053C4F8F453C4F8F85341
:107B6000C4F8FC53204638BD2DE9F04F002685B0FF
:107B7000A0F8EA6391F800C002939DF83C309DF8AC
:107B800038A0019204460393BCF1000F4DD0444845
:107B9000DFF8109140F2E238002341221F4603E053
:107BA00010F825201F46CAB30133DBB2624503EB50
:107BB0004305F5D107EB470700EB87073B7A6BB32B
:107BC00003F1FF3CB4F8EA33D7F804E05A1C52FA48
:107BD0008CFC4FF000471FFA8CFC11E06A7819F812
:107BE0000BB022EA0B0203F1010B43456A701FFA46
:107BF0008BF34FEA57074CD86345A4F8EA330DD00E
:107C000037EA0E0204EBD30503F0070BE6D119F8AF
:107C10000B2095F801B042EA0B02E4E70136F6B218
:107C200011F806C0BCF1000FB6D1D4F8F413039BD1
:107C30000298A4F8FE3345F6C052019BB2FBF0F067
:107C4000B2FBF3F3A4F8FCA3A4F8EE33A4F8F80312
:107C500021B108460AF03AF8B4F8F8030AF034F80B
:107C6000B4F8F853C4F8F4037DB1002203466C085D
:107C700011461646012001328C4291B28CBF187019
:107C80001E70A94203F10103F5D3002005B0BDE841
:107C9000F08F00230420A4F8EA3305B0BDE8F08F8C
:107CA00038860100488801000346007890B3B3F895
:107CB000ECC31E4803EBDC010CF007024978825C40
:107CC00011EA0200B3F8FA2305D0D3F8F413895C63
:107CD00009B3B3F9FC03B3F8F813013292B291423D
:107CE00098BF0022B3F8F013A3F8FA234A1CB3F8A4
:107CF000EE1392B29142A3F8F0230BD80CF10102DB
:107D0000B3F8EAC392B200219445A3F8F013A3F8A4
:107D1000EC2305D97047B3F8FC03404200B2DAE720
:107D20001970A3F8EC13A3F8FA1370474888010000
:107D30000346007890B3B3F8ECC31E4803EBDC01B4
:107D40000CF007024978825C11EA0200B3F8FA23CA
:107D500005D0D3F8F413895C09B3B3F9FE03B3F883
:107D6000F813013292B2914298BF0022B3F8F01397
:107D7000A3F8FA234A1CB3F8EE1392B29142A3F887
:107D8000F0230BD80CF10102B3F8EAC392B2002140
:107D90009445A3F8F013A3F8EC2305D97047B3F882
:107DA000FE03404200B2DAE71970A3F8EC13A3F81F
:107DB000FA13704748880100B0F8EC3313B9B0F8F3
:107DC000F03303B17047B0F8FA33002BFAD1012237
:107DD0000270A0F8EC33A0F8F033A0F8FA33704743
:107DE00000230370A0F8EC33A0F8F033A0F8FA33C6
:107DF000704700BF00787047B0F8EC3313B9B0F8A3
:107E0000F0330BB101207047B0F8FA03003818BF07
:107E1000012070470022026042600281C26002615C
:107E200082827047C0E90012704700BF70B5C56814
:107E30003E4E036905610446008906FB05F24FEAE0
:107E4000E27C0130D20F80B242EA4C0202F31E0201
:107E5000C3EB420303EB81113C2882B02081E16037
:107E600002D0207D02B070BD81FB0123D20F42EA17
:107E7000430281FB0513C90F41EA430101F31E03CD
:107E800006FB03F3D917DB0F43EA410385FB0551DA
:107E9000ED0F207D02F31E0245EA410505F31E05A4
:107EA0002A4403F31E032568A2EB430208BBAA423F
:107EB00030DA637D0133DBB2092B63752BD9A37DE7
:107EC000092B28D8012323751846194900902BB295
:107ED000184812B206F082FD1648A37D627D16494D
:107EE00006F01CFD207D00232381E360236102B0A6
:107EF00070BD6568AA4211DBA37D617D0133DBB2F1
:107F00000929A37501D9092B0DD900232375A37560
:107F10001846DAE7607500232375E4E70023A375AC
:107F2000637D092BF1D901232375DCE74DC5FB30B7
:107F30005088010020E6FF1F788801000023C360FD
:107F4000036103750381704700224FF48041018073
:107F5000827042600272704701EB810101807047BC
:107F60000246807870B1516842F6DF6399420AD8C0
:107F70000020013145F6BF53994201D85160704746
:107F8000002353607047107A0B4BB2F800C033F8EF
:107F90001030013013FB0CF35FFA80FCBCF13B0F97
:107FA0004FEAE33303F30F0318B28ABF002382F8CA
:107FB00008C01372DDE700BF94880100002301228E
:107FC000827043600372704700238370704700BF64
:107FD000002202604260704702EB420245F6C05345
:107FE000D20003FB01220260704700BF024B006811
:107FF000A3FB003000097047ABAAAAAA03680BB123
:1080000001234360704700BF00234360704700BFF7
:1080100043681BB102680AB119444160704700BF50
:108020004068003818BF0120704700BF03682BB1BB
:10803000406883422CBF00200120704718467047DB
:1080400038B500254FF46163044685820570C5820A
:108050004560856083810576457642F6302009F0DB
:1080600033FE231D20612577A360204638BD00BF65
:10807000002383820370C3824360037643760377D1
:10808000704700BF384BA3FB023C4FEA5C0C0CEB83
:108090004C0C8C4461452DE9F04136D0CB1C4FF09F
:1080A000010E21E00569828A92B202EB4202AC180D
:1080B00005F802806770A670828A013292B28282CD
:1080C000848A8289A4B292B2944228BF8182818A32
:1080D000C28A89B292B2914208BF80F818E0634523
:1080E00003F1030211D01346027E13F8038C13F838
:1080F000027C13F8016C02F0FF01002AD2D0634524
:1081000080F819E003F10302EDD1037F0BB1BDE864
:10811000F081C28A838A92B29BB29A4217D0C28AF5
:10812000838A92B29BB29A420ED3C28A8189838A91
:1081300011FA83F39B1A9BB2B3F5967F94BF002389
:1081400001230377BDE8F081838AC28AF2E7027EC9
:1081500002F0FF03002AF4D08389B3F5967F94BF21
:10816000002301230377EDE7ABAAAAAA0346007F09
:10817000002859D0F0B51A78CAB1032A0BD15C682F
:10818000C4F30B0CACF5006C0FFA8CFC0132A1F8B7
:1081900000C01A70F0BD0132D2B24FF0000C052AB7
:1081A000A1F800C088BF83F800C0F2D9F0BDB3F8D1
:1081B00014E0B3F816C01FFA8EFE1FFA8CFCE645D9
:1081C00033D01C69B3F816C01FFA8CFC0CEB4C0CB6
:1081D00004EB0C0514F80C706E78AD7800241C7656
:1081E000B3F816C00CF1010C1FFA8CFCA3F816C0F2
:1081F000B3F816E0B3F80CC01FFA8EFE1FFA8CFC21
:10820000E64528BFDC821C464FF0000C44F804CF42
:108210001F715E719D719C605C684FEA143CACF507
:10822000006C0FFA8CFCB1E770471D7E05F0FF046F
:10823000002DC6D11C772046F0BD00BFC28A838ABC
:1082400092B29BB29A421BD0C28A838A92B29BB2EC
:108250009A4208D3C38A818A8289581A80B290428E
:108260000AD9002070478289838AC08A12FA80F076
:10827000C01A80B29042F4D800EB400080B2704740
:10828000037E002BEDD1808900EB400080B2704767
:1082900070B504460626002585F0010529462046CE
:1082A00000F0D4FF2946204600F0D8FF294620469A
:1082B00000F0D8FF2946204600F0D8FF2946204686
:1082C00000F0D8FF2946204600F0D8FF2946204676
:1082D00000F0D8FF013EFA21204600F0FBFF16F027
:1082E000FF06D9D13146204600F0BCFF314620467A
:1082F00000F0BCFF3146204600F0BCFF314620466E
:1083000000F0BCFF3146204600F0BCFF20460121B2
:1083100000F0A8FF2046FA2100F0DCFF20460121F2
:1083200000F0A4FF2046FA2100F0D4FF20460121EE
:1083300000F0A0FF2046FA2100F0CCFF20460121EA
:1083400000F09CFF2046FA2100F0C4FF20460121E6
:1083500000F098FF2046FA2100F0BCFF314620468D
:1083600000F090FF2046FA2100F0B4FF314620468D
:1083700000F084FF2046FA2100F0ACFF3146204691
:1083800000F078FF2046FA2100F0A4FF3146204695
:1083900000F06CFF2046FA2100F09CFF3146204699
:1083A000BDE8704000F05EBF2DE9F84F00254FF4A6
:1083B0001676044685810570C581868005744574EE
:1083C0004FF4166009F080FC4FF4FA73A583A38282
:1083D000E583A06084F8205084F821504FF4FA60BF
:1083E00009F072FCA585A061E585A68484F830506B
:1083F00084F831504FF4966009F066FC4FF040234A
:10840000C4F82033C4F82433C4F82833C4F82C3318
:10841000C4F830334FF4804304F144074FF00108AF
:10842000A4F81E334FF00823A0626563A563E563DB
:10843000256484F81C5384F83853C4F83C53A4F8DA
:108440004453C4F8485384F84C53C4F84083C4F8E8
:1084500034332946102238460BF07AFC04F16006CA
:10846000324BC4F834804FF05008A763E3634246B0
:10847000294630460BF06CFC2D4BE36504F1BC0A39
:108480000C238C27A4F85430DFF8B490A66504F5CB
:10849000AA7B2A263A46294650460BF059FCC4F8D6
:1084A000B4A03A4604F5F67A2946A4F8B060C4F8B8
:1084B000B89058460BF04CFC2946C4F84CB1C4F8AF
:1084C0005091A4F848613C2250460BF041FC1949F8
:1084D000C4F8E81104F50D7306214246A4F8E01132
:1084E000C4F8E4A1294618460BF032FC124BC4F83C
:1084F0003032294604F524730A25C4F82C023A4682
:108500001846A4F828520BF023FC0C4AC4F8880241
:10851000C4F88C222046A4F8846200F02FFD204687
:10852000FFF7B6FE2046BDE8F88F00BFE00DFF1F45
:10853000C80DFF1F000DFF1FB40DFF1F600DFF1FB3
:108540000C0DFF1F2DE9F04F057885B00E9F002D13
:1085500072D01E4690F84C330446002B6CD1574B1A
:1085600091461A7888465AB990F81C13012281F076
:1085700001011A7000F06EFE5149524806F098F958
:1085800008F1FF310A2907D8DFE801F05C5F626576
:10859000686B6E0606715900B4F92083002E4BD02B
:1085A000013EB6B209EB4606A9F10205B4F83693CE
:1085B000BB4635F8021F11FB08F1C91301F30F0187
:1085C000494489B2B1F5805F04D3B4F84433013330
:1085D000A4F84433002F52D09BF80030ADF80810B7
:1085E0008DF80A3094F82020029B039302F0FF0AD2
:1085F000002A3FD1A069A28B92B200EB820003A9AE
:10860000042207F0DDF8A28B013292B2A283A18B83
:10861000A28A89B292B2914228BFA4F81CA0A28B70
:10862000E38B92B29BB29A4204BF012384F82030BC
:10863000AE420BF1010BBCD105B0BDE8F08FB4F92F
:108640003283ABE7B4F92283A8E7B4F92483A5E722
:10865000B4F92683A2E7B4F928839FE7B4F92A8303
:108660009CE7B4F92E8399E7B4F92C8396E7B4F923
:10867000308393E74FF0010384F82130D8E7ADF859
:1086800004108DF8067094F82030019A0392002BA4
:10869000F0D1A069A38B9BB200EB8300042203A955
:1086A00007F08EF8A38B01339BB2A383A28BA38A1E
:1086B00092B29BB29A42B2D3A783B0E70AA7FF1F38
:1086C0000C89010020E6FF1FC28B838B92B29BB204
:1086D0009A4219D0C28B838B92B29BB29A4208D332
:1086E000C38B818B828A581A80B2904288BF002047
:1086F0007047828A838BC08B12FA80F0C01A80B2D6
:10870000904288BF0020704790F820300BB10020C5
:108710007047808A704700BF38B5044D2B788B4274
:108720000C4601D000F09AFD2C7038BD08A7FF1F41
:1087300080F84113704700BF30B5354D2B788B4220
:1087400083B01DD0013B0C46092B0BD8DFE803F0AA
:10875000051E242A30363C0A0A420021019000F00E
:1087600081FD0198631E092B09D8DFE803F0053964
:108770003D4145494D08080B012100F073FD2C7067
:1087800003B030BD012100F099FDF8E70021019010
:1087900000F06CFD0198E5E70021019000F06AFD12
:1087A0000198DFE70021019000F068FD0198D9E70A
:1087B0000021019000F066FD0198D3E700210190AF
:1087C00000F070FD0198CDE70021019000F05EFD02
:1087D0000198C7E70021019000F070FD0198C1E702
:1087E000012100F043FDCAE7012100F043FDC6E787
:1087F000012100F043FDC2E7012100F043FDBEE787
:10880000012100F04FFDBAE7012100F03FFDB6E77E
:1088100009A7FF1F38B5057805B138BD044600F03B
:10882000D5FB0123237029462046BDE83840FFF7D9
:1088300083BF00BF2DE9F04FD0F83C3302780133FD
:108840008FB00446C0F83C33002A00F0EB80D0F82B
:1088500048134BF67F32914215D98E4A1278511E39
:10886000042900F27381022A04D18B4B1B78002B60
:1088700040F0BA8200212046FFF75EFFD4F83C3377
:108880000022C4F8482345F6BF52934200F2B88054
:1088900094F83833002B40F0AD80E28BA38B92B27A
:1088A0009BB29A4200F08E80E28BA38B92B29BB275
:1088B0009A4280F0D680A38BE28B9B1A9BB2002B4E
:1088C00000F08780E289A38992B29BB29A4200F0BD
:1088D000C380E289A38992B29BB29A4280F0C98098
:1088E000A389E2899B1A9BB2012B68D9B4F91E9324
:1088F00094F8413303930DF1140B4B4607ADB4F8D4
:1089000034A3D94606AEA84600279B46A189E28932
:1089100089B292B2914200F09A80A168E28992B243
:1089200001EB82010CA8042206F04AFF2774E289B9
:10893000013292B2E281E189A28889B292B2914277
:1089400028BFE7819DF8322009F8012BA18DE28D27
:1089500089B292B2914275D0A16AE28D92B231F899
:10896000122084F830702A80E28D013292B2E285C2
:10897000E18DA28C89B292B2914228BFE785039B18
:108980004BB1BDF8302092B2002A7AD1B4F842231C
:108990000132A4F84223BDF8302092B2A2EB0A02C1
:1089A00012FB0BF2D21302F30F0226F8022B4645FC
:1089B00005F10205AAD194F84C33002B74D00FB006
:1089C000BDE8F08F94F820301BB1A38A002B7FF410
:1089D00079AF314B1A78002A3FF474AF94F81C1326
:1089E000204600221A7000F035FC2C492C4805F076
:1089F0005FFF67E7204600F01FFC84F84C034CE75C
:108A000094F84013002381F00101C4F83C3384F84A
:108A10004013204600F01AFC94F83833002B3FF442
:108A20003CAFE7E71F498B42C9D990F84013C0F823
:108A30003C2381F0010180F840130FB0BDE8F04FF6
:108A400000F004BC94F83020002A85D197E7227CFE
:108A5000002A7FF462AF75E7237C002BAFD0A38898
:108A600042E7E28BA18AA38B11FA83F39B1A9BB294
:108A700025E7E289A188A38911FA83F39B1A9BB2A7
:108A800032E7BDF8302040F6FF7192B28A4282D1BF
:108A90007CE700BF09A7FF1F0AA7FF1F1489010079
:108AA00020E6FF1F7FA9030002220AA906A809F0F9
:108AB0007FFA0AA902230CAA04F134000AF0BCFCD4
:108AC000DDE90C321344BDF81810AB4A03EBD37345
:108AD0005B1403F30F039BB2C91AADF82010BDF865
:108AE0001A101278CB1AADF82230002A33D1A34BDA
:108AF0001B78002B40F03281A14B1B78002B40F0FB
:108B00006581A04B1B78002B40F01A819E4B1B788F
:108B1000002B40F004819D4B1B78002B40F0F1802E
:108B20009B4B1B78002B40F0DE809A4B1B78002B70
:108B300040F0CF80984B1B78002B3FF440AF08AC3F
:108B4000964802222146F7F7D1FF38E7063A012A74
:108B50003FF696AE8EE60A2A1AD8013A092A3FF65F
:108B60002EAF01A353F822F0AD8C00006F8C0000F3
:108B7000498C0000238C0000FD8B0000BF890000A1
:108B8000D78B0000BF890000BF890000B78B0000B1
:108B9000602A00F03581632A7FF411AF09AA06A983
:108BA00004F15400022309F07FFF7D48022209A945
:108BB000F8F76EFD03E7204600F03EFB08AC0146E7
:108BC000022378482246FEF77BFD734B1B78002B6F
:108BD0003FF4F5AEB4E76E4B1B78002B3FF4EFAEDD
:108BE00009AA08A904F52170022309F05DFF6E4867
:108BF000022307AA09A900F05FFFE0E6614B1B789A
:108C0000002B3FF4DCAE09AA08A904F50A70022380
:108C100009F04AFF6548022307AA09A901F050FE9E
:108C2000CDE6574B1B78002B3FF4C9AE09AA08A923
:108C300004F5F070022309F037FF5D48022307AA0C
:108C400009A902F045FDBAE6504B1B78002B3FF412
:108C5000B6AE09AA08A904F5A470022309F024FFFE
:108C60005448022307AA09A906F070FBA7E6464B61
:108C70001B78002B3FF4A3AE022306A904F1B00039
:108C800009AA09F011FF4C4B1B78002B00F0C4809F
:108C90004A4B1B78002B00F0B98002230093484810
:108CA00005AB07AA09A9F9F7F9FF88E6334B1B784A
:108CB000002B3FF484AE09AA08A904F15400022352
:108CC00009F0F2FE3F48022307AA09A9FBF744FF77
:108CD00075E6204600F0B0FA0223014608AA3148A2
:108CE000FEF7EEFC26E709AA08A904F52170022385
:108CF00009F0DAFE2C48022307AA09A900F0DCFEDD
:108D000013E709AA08A904F5A470022309F0CCFE10
:108D10002848022307AA09A906F018FB00E7022346
:108D200006A909AA04F1B00009F0BEFE224B1B7887
:108D3000002B5ED02448022209A9F9F78DFFEAE64C
:108D400009AA08A904F50A70022309F0ADFE174824
:108D5000022309A907AA01F0B3FDD7E609AA08A9C9
:108D600004F15400022309F09FFE1648022309A9CA
:108D700007AAFBF7F1FEBFE609A7FF1F540EFF1F6E
:108D8000590EFF1F580EFF1F530EFF1F5B0EFF1FD4
:108D9000570EFF1F560EFF1F520EFF1FC016FF1F5C
:108DA000DC22FF1F4889FF1F209AFF1F0CA7FF1F0F
:108DB0001CBCFF1F50E8FF1F550EFF1F0AA7FF1F17
:108DC0003C48FF1FD065FF1FEC42FF1F09AA08A9FE
:108DD00004F5F070022309F067FE1348022309A985
:108DE00007AA02F075FC8CE610480021FAF7D0FDC6
:108DF00040E50F48022307AA09A9F9F7ABFB8AE669
:108E00000C48022207A9F8F767FFD8E50A480222B2
:108E100009A9F9F721FFD2E50548022307AA09A904
:108E2000F9F798FBCBE500BF1CBCFF1FE464FF1FF4
:108E30003C27FF1F4023FF1FEC42FF1F2DE9F0439B
:108E40009DF8409080F81C334FEAC919A0F8309380
:108E50009DF844909DF820309DF81C809DF824706A
:108E60009DF828609DF82C509DF830409DF834E026
:108E70009DF838C04FEAC919A0F83293BDF948905F
:108E800009F50069DB01A0F83693BDF94C90A0F814
:108E900020339DF83C3009F500694FEAC818FF01FE
:108EA000F601ED01E4014FEACE1E4FEACC1CDB01D6
:108EB000A0F834939DF85090A0F81E83A0F8227378
:108EC000A0F82463A0F82653A0F82843A0F82AE3CA
:108ED000A0F82CC3A0F82E3380F8389319B1C8F14C
:108EE0000008A0F81E83B2B17F4276426D42644210
:108EF000CEF1000ECCF1000C5B42A0F82273A0F87A
:108F00002463A0F82653A0F82843A0F82AE3A0F889
:108F10002CC3A0F82E33BDE8F08300BFB0F842C3E5
:108F2000B0F84433BCF1000C18BF4FF0010C003B0B
:108F300081F800C018BF012300211370A0F842136C
:108F4000A0F84413704700BF0346002290F82100A8
:108F500083F82120704700BF03460022407C5A74EA
:108F6000704700BF0023C0F848337047D0F848036B
:108F7000704700BF90F84C03704700BF08B501214F
:108F8000052006F001FE0121062006F0FDFD01216D
:108F9000032006F0F9FD0021042006F0F5FD012173
:108FA000092006F0F1FD01210A2006F0EDFD012166
:108FB0000B2006F0E9FD01210C2006F0E5FDBDE8DF
:108FC00008400121182006F0DFBD00BF414B424997
:108FD000DA6A70B542F48052C024DA6281F8214026
:108FE000D96B3E4A41F000613524D9639460042373
:108FF00012244021D46011625362536A43F080030B
:109000005362536A13F08003FBD1916BD46B166CDF
:1090100021443144566C3144966C3144D66C314411
:10902000C1F34E01452441F400414FF0E025D162E7
:109030001460284C8022C5F80421216B284A41F095
:1090400000612163122135249460D16004211362F0
:109050005162536A43F080035362546A14F08004EF
:10906000FBD1936BD16B1B4D0B4490F81C13106C10
:109070000344506C0344906C0344D06C0344C3F32A
:109080004E0343F40043D362164B8E22AA614FF481
:1090900040725A61AA6BA3F5304342F00102AA6301
:1090A000042040F2F3121C6058609A6022221A6079
:1090B0001A6842F0010205201A6006F02DFD2146D3
:1090C000062006F029FDBDE870400121032006F0CE
:1090D00023BD00BF0080044000C00C4000B003402E
:1090E00000B00B4000B0044030B583B04FF40062D4
:1090F0000023ADF800208DF80230828BC38B92B232
:109100009BB29A4204465BD0A169E38B9BB201EB10
:1091100083010422684606F053FB002184F82010E6
:10912000E38B01339BB2E383E28BA38A92B29BB2BF
:109130009A4228BFE1833A4BBDF8000039491A68CA
:109140000880110641D4384B1A6812060CD51A69EA
:1091500094F8303003F0FF01002B2DD1A06AA38DCD
:109160009BB220F8132009E094F8303003F0FF019F
:1091700013BBA26AA38D9BB222F81310A38D0133F7
:109180009BB2A385A28DA38C92B29BB29A4228BFB8
:10919000A185A28DE38D92B29BB29A4204BF0123B6
:1091A00084F83030204B04221A60D4F8483301335D
:1091B000C4F8483303B030BD012384F83130F1E7FF
:1091C00090F82030002B9FD1B5E71B699BB2ADF81A
:1091D0000030237C009A019203F0FF05EBB9A068F0
:1091E000A38904229BB200EB83000DEB020106F081
:1091F000E7FAA38901339BB2A381A289A38892B223
:109200009BB29A4228BFA581A289E38992B29BB200
:109210009A4204BF0123237495E70123637492E704
:1092200000B0034000C00C4000B00B400148FFF705
:109230005BBF00BFD096FF1F08B5042006F096FC68
:10924000A0F10100B0FA80F0400908BD032006F04B
:1092500063BC00BF052006F05FBC00BF062006F01F
:109260005BBC00BF092006F057BC00BF0A2006F017
:1092700053BC00BF0B2006F04FBC00BF0C2006F013
:109280004BBC00BF182006F047BC00BF10B509203A
:109290000C4606F041FC21460C20BDE8104006F0CB
:1092A0003BBC00BF10B509200C4606F035FC21463A
:1092B0000A20BDE8104006F02FBC00BF10B5092001
:1092C0000C4606F029FC21460B20BDE8104006F0B4
:1092D00023BC00BF084606F093BC00BF01207047C6
:1092E0000846102244F2580106F06ABA38B503461F
:1092F000002503F8015B0446457029465D709D70AA
:10930000DD701D714FF4F06206300AF021FD134B41
:109310001349C4F88C37C4F89037C4F88817202252
:109320002946A4F88657C4F89457C4F8985704F20D
:109330009C700AF00DFDA4F8BC572022294604F2C7
:10934000BE700AF005FD632384F8E037A4F8DE5709
:10935000C4F8E457A4F8E857204638BD0F270F2774
:1093600000000F2700230E4A0E4903704FF0630CD4
:1093700080F8E0C7A0F8BC37A0F8DE37A0F8863741
:10938000C0F88817C0F88C27C0F89027C0F8943729
:10939000C0F89837C0F8E437A0F8E837704700BF46
:1093A0000F270F2700000F2770B5044682B0002A50
:1093B00077D03E4E4FF47A5C0020E646354614E006
:1093C0009D42B8BF1D469E45A8BF9E464B1D9BB201
:1093D000B3F5707F00F10100A1F2BB3138BF19462F
:1093E00083B228BF89B29A420CD904EB4103B3F986
:1093F0000630002BE4DC9C45A8BF9C469E42B8BFCB
:109400001E46E3E70CEB060305EB0E025B1003EBD5
:1094100062065510A5EB660542F34F021BB246F3F8
:109420004F062DB2224923480195009605F052FBC4
:1094300094F8E037632B26D004EB43020133DBB210
:109440000F2BA2F89C67A2F8BE5704F29A7184F819
:10945000E03704F2BA7E20D800221346A4F8BC27D5
:10946000A4F8DE2731F802CF488C624403448E45CD
:1094700012B21BB2F6D112111B11A4F8BC27A4F82A
:10948000DE3702B070BD04F29A710B4604F2BA7E68
:1094900023F8026F9E455D84FAD1002384F8E037FB
:1094A000DAE7154616461346BCE700BF80C1FFFF4A
:1094B0001C89010020E6FF1F2DE9F047BDF8204080
:1094C000BDF92470BDF92890002A00F0888002348C
:1094D000444EBFB2A4B2C9F1000800252DE04FEA06
:1094E000DC0E0CF0070C16F80CA013F80EC02CEADA
:1094F0000A0C03F80EC004F1FF3CCCF3CC0E0CF0C8
:10950000070C13F80EA016F80CC04CEA0A0C03F86E
:109510000EC001F1050C1FFA8CFCBCF5707F05F143
:1095200001052CBFA1F2BB3161461FFA85FC28BFA3
:1095300089B202346245A4B251D900EB410EA4F1C4
:10954000020CBEF806E0AEEB070E0FFA8EFEC64523
:109550001FFA8CFCC3DBBEF1000F1CDBCE454FEACB
:10956000DC0E0CF0070C13F80EA016F80CC04CEA39
:109570000A0C03F80EC004F1FF3CCCF3CC0E0CF047
:10958000070C23DA16F80CA013F80EC02CEA0A0C0C
:1095900003F80EC0BDE74FEADC0E0CF0070C16F81E
:1095A0000CA013F80EC02CEA0A0C03F80EC004F14C
:1095B000FF3CCCF3CC0E0CF0070C16F80CA013F803
:1095C0000EC02CEA0A0C03F80EC0A2E713F80EA096
:1095D00016F80CC04CEA0A0C03F80EC099E7BDE877
:1095E000F08700BFF08901002DE9F04F1F46B0F869
:1095F000863703440546587887B048409DF8404078
:109600009DF84480164605F0FFFAA04247D8B5F809
:10961000883703F29D391FFA89F9B9F5707F24BFA5
:10962000233B1FFA83F9741EF21D454BCC460026DE
:109630004FF47A514FF6FD7A032012E0BBF1FF3F61
:1096400027D01EFB00660CF1050E1FFA8EFEBEF53C
:10965000707F26BFACF2BB3C1FFA8CFCF4469442F0
:1096600019D005EB4C0E14F901BFBEF906E07345A5
:10967000B8BF73467145A8BF7146BBF1010F05D055
:10968000BBF1030FDAD11EFB0A66DCE7A6EB0E0680
:10969000D9E77644D7E7D5F89427B24203DB002018
:1096A00007B0BDE8F08F95F8E027632A38D0B5F908
:1096B000BC17B5F9DE37029300240822019105ABEF
:1096C000494628460094FFF7F7FE3B789DF81400C2
:1096D000584005F099FA7B7807469DF815005840E8
:1096E00005F092FA0744FFB2B845D8D3B5F88837E9
:1096F000A5F88E3703F2973292B2B2F5707F4FF031
:10970000040128BF293BC5F89467A5F89817A5F868
:109710008A9734BFA5F88C27A5F88C370120BFE7BE
:109720001944A3EB610344F63E1202FB03F341F339
:109730004F0143F3CF33A5F8BC17A5F8DE37BAE7DE
:1097400080C1FFFF70B582B00025384B384A0195C3
:109750000095F2210446FFF747FF364B019500952F
:10976000354A05460D212046FFF73EFF94F89A370B
:10977000064645BB00283DD0002B3FD0013BDBB265
:10978000012B84F89A371CD1B4F88E3703F2BF321C
:1097900092B2B2F5707F28BF03F1FF32A4F8902790
:1097A0005A1C92B2B2F5707F2ABFA3F2BF33A4F85D
:1097B0009227A4F8923794F89B2722700023A4F8EC
:1097C0009A3702B070BD002BD8D1C4F8E437A4F8A2
:1097D000E8371A480121FEF79FFF18480121FEF7DC
:1097E000A7FF632240F2051384F8E027A4F89A3714
:1097F0009EB915E0002BC1D102B070BDC4F8E437AA
:10980000A4F8E8370D480121FEF786FF0B48012137
:10981000FEF78EFF632384F8E037022384F89B373A
:10982000042384F89A3702B070BD00BF008A01009B
:10983000148A0100FC8901000C8A0100D096FF1FE8
:1098400070B5B0F89027B0F89217B0F888378A4210
:1098500092B0044611D29A4205D9B4F88C279A42A4
:109860002AD012B070BD9942F7D302260125CDE966
:109870000056874B874A0D210BE09A4201D9994245
:10988000EBD302260125CDE90056814B814A0D21FB
:109890002046FFF7A9FECDE900567F4B7F4A0546DB
:1098A000FD212046FFF7A0FE05B12670002840F0FC
:1098B0008980B4F88837D0E7B4F89837042B16D1EC
:1098C000B4F88E3703F2BF3292B2B2F5707F28BF80
:1098D00003F1FF32A4F890275A1C92B2B2F5707FC0
:1098E0002ABFA3F2BF33A4F89227A4F89237B4F8A2
:1098F0008A17C0222046FFF757FD2378012B00F07E
:109900008780022B29D0B4F9DE17B4F9BC27019265
:1099100008230291B4F88A170093C02205AB2046B1
:10992000FFF7CAFDB4F89857013DADB2A4F89857B7
:10993000002D79D02378A5F10305B5FA85F56D09D9
:10994000012B8DF8145029D0022B12D00023C4F81B
:10995000943784F89B3712B070BDB4F9DE07B4F9C0
:10996000BC37B4F98E274E4900904E4805F036F8C2
:10997000C9E7B4F8E827002A00F08380D4F8E43778
:10998000B3FBF2F3C3F307218DF8451045488DF87A
:109990004630332205A904F0DFFD08E0B4F8E827DB
:1099A000002A5ED13F48312205A904F09DFD002325
:1099B000C4F8E437A4F8E8370023C4F8943784F8EF
:1099C0009B37C8E7B4F9DE07B4F9BC37B4F98E2782
:1099D00035490090334805F001F834480021FEF77E
:1099E0009BFE00213148FEF7A3FE2E4804F0ECFD5B
:1099F000002142F20F726320B4F888372170A4F876
:109A00008C2784F8E007A4F89A17C4F8941726E77F
:109A1000B4F9DE07B4F9BC37B4F98E2724490090B5
:109A2000204804F0DBFF6EE71E48224904F040FFA7
:109A300029461E48FEF770FE29461C48FEF778FEB0
:109A4000184804F0E1FD42F20F7263232570A4F878
:109A50008C2784F8E037A4F89A57C4F8945712B0CA
:109A600070BDD4F8E437B3FBF2F3C3F307218DF8EC
:109A700045100C488DF84630332205A904F034FD1A
:109A800095E70848312205A904F066FD8FE700BF7D
:109A9000FC8901000C8A0100F8890100048A010098
:109AA0009C89010020E6FF1F3C890100D096FF1F22
:109AB00068890100CC890100002B46D0F8B55D1EF5
:109AC000EDB2971EB0F88637B0F88827044601EB50
:109AD00045058E1E16E0FFF735FEB4F88827B4F86A
:109AE0008637013292B201339BB2B2F5707F28BF44
:109AF0000022052B28BF0023B542A4F88827A4F82C
:109B0000863721D037F802CFD4F8E417B4F8E80745
:109B100023448C44013036F9021FC4F8E4C7A4F88A
:109B2000E80758784000C0B20029B8BF40F00100F3
:109B30005870237804EB4202013B012BD180204670
:109B4000C9D8FFF77DFEC8E7F8BD704770B5044679
:109B500000254FF47A602581208065816573257327
:109B600008F0B2F8294660604FF4966204F13C00B8
:109B70000AF0EEF804F11C064FF49653F022A4F814
:109B8000F024C4F8F434C4F8EC54C4F8F854202297
:109B9000294630460AF0DCF8034A044B226163612F
:109BA000A661204670BD00BF05000900F80DFF1F2B
:109BB000312A01D0042070474289038992B29BB2B6
:109BC0009A4230B544D04289038992B29BB29A42FC
:109BD00008D34389048902881B1B9BB29A420AD28C
:109BE000052030BD04890288438912FA83F31B1BC8
:109BF0009BB29A42F4D32F2BF2D901F1300C4FF0E3
:109C0000010E18E0456803899BB2EA5403890133C9
:109C10009BB203810289038892B29BB29A4228BF09
:109C200004810289438992B29BB29A4208BF80F8AC
:109C30000CE061450AD0037B11F8012F03F0FF040B
:109C4000002BDFD0614580F80DE0F4D1002030BD5D
:109C5000037B002BC4D10388CDE700BF70B58EB065
:109C600002AB04AD4FF4F77640F2C95E4FF6372CE5
:109C70004FF6126201F0C004802C1ED0C02C19D007
:109C8000B4B1A3F800C0023389009D42C9B2F1D13A
:109C90002A4602A90423103008F01CFA002300937E
:109CA000074814232A460721FEF74CFC0EB070BD6E
:109CB0001A80E8E7A3F800E0E5E71E80E3E700BFCD
:109CC000D096FF1FF0B5B0F8EC348FB0044613B354
:109CD0005848594EFEF7F8FC054617E0B4F8EE3444
:109CE0005A1C2344A4F8EE2493F83C10FFF7B6FF67
:109CF0003378143DADB21BB1D4F8F434C4F8F83461
:109D0000B4F8EE24B4F8EC349A4274D2142D204600
:109D1000E4D80FB0F0BD4189028989B292B2914274
:109D20006ED04189028989B292B2914231D20289C0
:109D30004189521A92B2002A34D0404A1278002A3D
:109D400063D0002019E06168628992B28D5C207353
:109D50006289013292B262816189228889B292B2AB
:109D6000914228BF60815A1C92B22344302AA4F841
:109D7000EC2483F83C5055D013462189628989B27E
:109D800092B29142DFD1227B02F0FF05002ADAD1A4
:109D9000E9E741890088228910FA82F2521A92B2C8
:109DA000002ACAD1D4F8F834002BB2D02148214F70
:109DB000FEF78AFC0026054613E0CDE9026608F0AE
:109DC00089F91423009604AA07213846FEF7BAFB46
:109DD000D4F8F834143D013BADB2C4F8F834002B8C
:109DE00097D0142D4FF0040304AA02A904F1100027
:109DF000E3D80FB0F0BD0023C4F8EC340FB0F0BDD1
:109E0000027B002ACED0028895E7B4F8F01469B13D
:109E10007720E21801339BB28B4282F83C00F8D1E4
:109E2000A4F8EC340023A4F8EE3451E7A4F8EE14BF
:109E3000B8E700BFD096FF1F550EFF1F0AA7FF1FF0
:109E400001EB4101890001F51671B1F5966F28BF4C
:109E50004FF49661A0F8F014704700BF428903895F
:109E600092B29BB29A421DD04289038992B29BB2B0
:109E70009A4208D3438901890288581A80B28242E3
:109E80000AD20020704702880389408912FA80F0C4
:109E9000C01A80B28242F4D3084BA3FB0030C0F357
:109EA00047107047037B002BEBD10088A3F155339B
:109EB000A3FB0030C0F34710704700BFABAAAAAAAB
:109EC0004FF4966303FB01F1C0F8F414704700BF30
:109ED000014803F0C5B900BF20E6FF1F10B5664872
:109EE000664C03F067FF6648FEF7A4FC654B1B78E1
:109EF000002B00F09D802378012B00F09680624AB1
:109F0000127812B1022B00F09580604A127812B1DB
:109F1000032B00F097805E4A127812B1042B00F0F8
:109F200096805C4A127812B1052B00F095805A4A4F
:109F3000127812B1072B00F09480584A12784AB177
:109F4000062B03D0564801F07BFE10B1544801F0B7
:109F500047FF2378534A1278F2B1CBB10A2B17D0BE
:109F6000632B25D0A3F15C02D2B2062A29D86FF068
:109F70004D0141FA02F2D2074AD55D2B2BD05B2B63
:109F80002FD06C2B33D0652B37D0002B3BD010BD9E
:109F90004548F7F711F82378444A1278002ADFD0B1
:109FA0000A2BDDD14248FBF7BDFB2378632BD9D1C7
:109FB0004048F7F7A7FB2378A3F15C02D2B2062A48
:109FC000D5D9A3F16602052AD9D83B48F7F714FD85
:109FD00023785D2BD3D13948F7F710FE23785B2B1C
:109FE000CFD13748F7F7C6FD23786C2BCBD1354856
:109FF000F7F794FD2378652BC7D13348F7F742FE76
:10A000002378002BC3D1BDE810403048F7F75EB885
:10A010002F48F7F761FA2378A3F16602052AACD836
:10A020002548F7F7E9FC2378D3E72A48FBF798F8A7
:10A03000237864E7284B1B78C3B12848F9F72AFF37
:10A04000237862E7264805F0B3FA237863E72548CA
:10A0500001F0BEFC237864E7234800F06BFD237811
:10A0600065E72248FFF72EFE237866E72048F8F7D9
:10A0700045FB237849E700BF20E6FF1F09A7FF1F24
:10A08000D096FF1F540EFF1F530EFF1F5B0EFF1FC6
:10A09000590EFF1F580EFF1F570EFF1F5A0EFF1FAE
:10A0A000E0E3FF1F520EFF1F4C20FF1F560EFF1F45
:10A0B0004889FF1F1C23FF1F2023FF1F3823FF1F7A
:10A0C0003423FF1F3023FF1F3C23FF1F4C23FF1FA0
:10A0D000B022FF1FA086FF1F550EFF1FE464FF1F65
:10A0E00090FBFF1F60DEFF1F88B6FF1F0CA2FF1F43
:10A0F000F83DFF1F08B52F48F9F746FF2E48FAF73D
:10A100008BFD2E48F7F72CFA2D48F7F7F7FA2D4874
:10A11000F8F7C6FB2C48F8F7B5FD2C48F9F7BAFA62
:10A120002B48F7F71BFE2B48F8F732FA2A48F7F7C7
:10A13000B5F82A4804F0B2FD294805F057F9294836
:10A1400000F0FCFD284801F021FB2848F7F752FDFC
:10A15000274800F06DF8274800F0FCFB2648F7F789
:10A1600003FD2648FFF7C2F82548FFF7EFFC254816
:10A17000F7F7D0FC244801F039FD2448F7F77EFDBD
:10A180002348FBF7BBF92348F7F72EFC2248F6F7E4
:10A1900071FC2248F6F7BAFD2148F7F795FD2148F2
:10A1A000F6F784FF204801F0F5FFBDE808401F489E
:10A1B000FEF7FAB8D065FF1FA086FF1FDC22FF1F45
:10A1C0001C23FF1FEC42FF1F3C48FF1FE464FF1FDE
:10A1D0003C27FF1FF83DFF1FB022FF1F50E8FF1F65
:10A1E00090FBFF1F1CBCFF1F60DEFF1F3823FF1FFB
:10A1F0000CA7FF1F88B6FF1F3423FF1F209AFF1FE5
:10A200000CA2FF1F3023FF1FE0E3FF1F3C23FF1FB3
:10A210004889FF1F2023FF1FC016FF1F4C20FF1F70
:10A220004023FF1F4C23FF1F20E6FF1FD096FF1F78
:10A2300038B500250446294600F8025B142209F0CF
:10A2400087FD29464FF4706204F1160009F080FD85
:10A25000144B1549C4F81C3FC4F8203FC4F8181F1C
:10A2600020222946A4F8165FC4F8245FA4F8285FCA
:10A2700084F82A5F04F62C7009F06AFDA4F84C5F9C
:10A280002022294604F64E7009F062FD632384F80B
:10A29000703FA4F86E5FC4F8745FA4F8785F20463E
:10A2A00038BD00BF0F270F2700000F2700230F4ADC
:10A2B0000F4903704FF0630C80F870CFA0F84C3F4B
:10A2C000A0F86E3FA0F8163FC0F8181FC0F81C2F6A
:10A2D000C0F8202FC0F8243FA0F8283F80F82A3F7C
:10A2E000C0F8743FA0F8783F704700BF0F270F27D2
:10A2F00000000F2770B5044682B0002A78D03E4E89
:10A300004FF47A5C0020E646354615E09D42B8BF22
:10A310001D469E45A8BF9E4601F10A039BB2B3F5B8
:10A32000F06F00F10100A1F2767138BF194683B2D7
:10A3300028BF89B29A420CD904EB4103B3F9163015
:10A34000002BE3DC9C45A8BF9C469E42B8BF1E463E
:10A35000E2E70CEB060305EB0E025B1003EB620673
:10A360005510A5EB660542F34F021BB246F34F06AC
:10A370002DB2224922480195009604F0ABFB94F8D7
:10A38000703F632B26D004EB43020133DBB20F2B6B
:10A39000A2F82C6FA2F84E5F04F62A7184F8703F81
:10A3A00004F64A7E20D800221346A4F84C2FA4F8C5
:10A3B0006E2F31F802CF488C624403448E4512B2AE
:10A3C0001BB2F6D112111B11A4F84C2FA4F86E3F4A
:10A3D00002B070BD04F62A710B4604F64A7E23F8DB
:10A3E000026F9E455D84FAD1002384F8703FDAE75E
:10A3F000154616461346BCE780C1FFFF1C8A0100C4
:10A4000020E6FF1F2DE9F047BDF82040BDF924707C
:10A41000BDF92890002A00F088800234444EBFB273
:10A42000A4B2C9F1000800252DE04FEADC0E0CF0C3
:10A43000070C16F80CA013F80EC02CEA0A0C03F84F
:10A440000EC004F1FF3CCCF3CC0E0CF0070C13F85B
:10A450000EA016F80CC04CEA0A0C03F80EC001F16D
:10A460000A0C1FFA8CFCBCF5F06F05F101052CBF3E
:10A47000A1F2767161461FFA85FC28BF89B20234C9
:10A480006245A4B251D900EB410EA4F1020CBEF812
:10A4900016E0AEEB070E0FFA8EFEC6451FFA8CFCD7
:10A4A000C3DBBEF1000F1CDBCE454FEADC0E0CF027
:10A4B000070C13F80EA016F80CC04CEA0A0C03F8AF
:10A4C0000EC004F1FF3CCCF3CC0E0CF0070C23DAE9
:10A4D00016F80CA013F80EC02CEA0A0C03F80EC0F4
:10A4E000BDE74FEADC0E0CF0070C16F80CA013F8D1
:10A4F0000EC02CEA0A0C03F80EC004F1FF3CCCF3AA
:10A50000CC0E0CF0070C16F80CA013F80EC02CEAB9
:10A510000A0C03F80EC0A2E713F80EA016F80CC040
:10A520004CEA0A0C03F80EC099E7BDE8F08700BFBB
:10A530008C8A0100B0F8183F56492DE9F04703F224
:10A540002677BFB2B7F5F06F534C24BF5A3B9FB28A
:10A55000064686B0B94604F1090C6FF002020025E8
:10A560004FF47A504FF6FD784FF0030E11E00132B0
:10A5700022D013FB0E5509F10A039BB2B3F5F06F1D
:10A5800024BFA9F276739BB2644517D014F9012F4A
:10A59000994606EB4903B3F916309942B8BF1946FC
:10A5A0009842A8BF1846012A04D0032ADFD113FB22
:10A5B0000855E0E7ED1ADEE71D44DCE7D6F8243F56
:10A5C000AB4235DA96F8703F632B52D0B6F94C2F78
:10A5D000B6F96E3F02934FF000083946019205AB81
:10A5E0000A223046CDF80080FFF70CFF33789DF843
:10A5F0001400434580F0CD000CBF4FF0010A4FF02E
:10A60000030A04F001FB04469DF8150080F0F500F4
:10A6100004F0FAFA81469DF8160020F00F0080F051
:10A62000900004F0F1FA48440444E4B2544503D9DC
:10A63000002006B0BDE8F087B6F8182FA6F81E2F48
:10A6400002F21B739BB2B3F5F06F4FF0060128BF07
:10A65000653A4FF00100C6F8245FA6F8281FA6F857
:10A660001A7F34BFA6F81C3FA6F81C2F06B0BDE821
:10A67000F0874218A1EB620344F63E1101FB03F39D
:10A6800042F34F0243F3CF33A6F84C2FA6F86E3FA8
:10A69000A0E700BF80C1FFFF948A0100B0F8163F19
:10A6A00000EB430310B504465888C0F3090080F45A
:10A6B000A67080F0010004F0ADFA022829D82046E7
:10A6C000FFF738FF28B394F82A3F3BB3013BDBB2D6
:10A6D000012B84F82A3F1BD1B4F81E3F03F27F728E
:10A6E00092B2B2F5F06F28BF03F1FF32A4F8202F29
:10A6F0005A1C92B2B2F5F06F2ABFA3F27F73A4F88E
:10A70000222FA4F8223F01220023227084F82A3F3E
:10A7100010BD94F82A3F002BD8D110BDC4F8743F67
:10A72000A4F8783F07480121FDF7F6FF054801210D
:10A73000FDF7FEFF6322042384F8702F84F82A3F7C
:10A7400010BD00BFD096FF1F30B5B0F8202FB0F875
:10A75000221FB0F8183F8A4293B0044607D29A42AB
:10A7600007D9B4F81C2F9A421DD013B030BD9A42BD
:10A7700001D99942F5D3B4F8163F04EB4303588846
:10A78000C0F3090080F4A67080F0010004F042FAE2
:10A79000022802D82046FFF7CDFEB4F8183FB4F8DF
:10A7A0001C2F9A42E1D1B4F8283F062B16D1B4F8F9
:10A7B0001E3F03F27F7292B2B2F5F06F28BF03F131
:10A7C000FF32A4F8202F5A1C92B2B2F5F06F2ABFC4
:10A7D000A3F27F73A4F8222FA4F8223FB4F81A1F23
:10A7E000C0222046FFF786FDB4F96E0FB4F94C3F46
:10A7F000B4F91E2F2E4900902E4804F0EFF8B4F95A
:10A800006E1FB4F94C2F019208230291B4F81A1F5D
:10A810000093C02205AB2046FFF7F4FDB4F8285F93
:10A82000013DADB2A4F8285F45B3A5F10505B5FA21
:10A8300085F5B4F8783F6D098DF8145073B91D484B
:10A84000312205A903F0F8FD0023C4F8743FA4F8F1
:10A85000783F0023C4F8243F13B030BDD4F8742FE0
:10A86000B2FBF3F3C3F307218DF8451011488DF8BF
:10A870004630332205A903F0DFFDE5E70D480E4918
:10A8800004F016F80D482946FDF746FF0B48294607
:10A89000FDF74EFF074803F007FE42F20F726323F5
:10A8A0002570A4F81C2F84F8703F84F82A5FD0E745
:10A8B000408A010020E6FF1F688A0100D096FF1F32
:10A8C000002B46D0F8B55D1EEDB2971EB0F8163FCE
:10A8D000B0F8182F044601EB45058E1E16E0FFF771
:10A8E000DDFEB4F8182FB4F8163F013292B20133EE
:10A8F0009BB2B2F5F06F28BF00220A2B28BF0023BD
:10A90000B542A4F8182FA4F8163F21D037F802CF8B
:10A91000D4F8741FB4F8780F04EB43038C4401306F
:10A9200036F9021FC4F874CFA4F8780F5888400095
:10A9300080B20029B8BF40F001005880237804EBB2
:10A940004202012BD1822046C9D1FFF7FDFEC8E7A4
:10A95000F8BD7047F8B5044600254FF47A602581AC
:10A96000208065816573257307F0AEF92946606024
:10A970004FF4966204F1D40009F0EAF904F12807D3
:10A9800040F6B833F022C4F88C3504F14806A4F838
:10A9900088252946C4F884552022C4F890553846A5
:10A9A00009F0D6F98C222946304609F0D1F9064A39
:10A9B000064B226163611622054BA761A2832662C2
:10A9C00063622046F8BD00BF0A0009005C0EFF1F4D
:10A9D000100FFF1F312A01D00420704742890389DC
:10A9E00092B29BB29A4230B544D04289038992B266
:10A9F0009BB29A4208D34389048902881B1B9BB2ED
:10AA00009A420AD2052030BD04890288438912FA8D
:10AA100083F31B1B9BB29A42F4D32F2BF2D901F183
:10AA2000300C4FF0010E18E0456803899BB2EA54E0
:10AA3000038901339BB203810289038892B29BB2DE
:10AA40009A4228BF04810289438992B29BB29A42FA
:10AA500008BF80F80CE061450AD0037B11F8012F94
:10AA600003F0FF04002BDFD0614580F80DE0F4D146
:10AA7000002030BD037B002BC4D10388CDE700BF8D
:10AA800070B5ACB0054602AB04ACF52640F2DF2E43
:10AA90004FF6215C4FF60B7001F0C002802A26D0E1
:10AAA000C02A21D0F2B1A3F800C0023389009C4231
:10AAB000C9B2F1D1224602A905F11000042307F022
:10AAC00009FB18AA214605F11C00282307F0ECFF1A
:10AAD000002300930748282318AA0521FDF732FD1B
:10AAE0002CB070BD1880E0E7A3F800E0DDE71E8021
:10AAF000DBE700BFD096FF1F30B5ADB004460025A0
:10AB000002A904AA04231030CDE9025507F0E2FAA5
:10AB100004A904F11C0018AA282307F0C5FF044863
:10AB20000095282318AA0521FDF70CFD2DB030BD96
:10AB3000D096FF1FB0F8843570B504460BB3584863
:10AB4000584EFDF7C1FD054617E0B4F886355A1C8E
:10AB50002344A4F8862593F8D410FFF791FF3378A7
:10AB6000283DADB21BB1D4F88C35C4F89035B4F89B
:10AB70008625B4F884359A4262D2282D2046E4D83E
:10AB800070BD4189028989B292B291425CD04189FB
:10AB9000028989B292B2914231D202894189521A14
:10ABA00092B2002A34D0404A1278002A51D00020B4
:10ABB00019E06168628992B28D5C2073628901320A
:10ABC00092B262816189228889B292B2914228BF91
:10ABD00060815A1C92B22344302AA4F8842583F859
:10ABE000D45058D013462189628989B292B29142D9
:10ABF000DFD1227B02F0FF05002ADAD1E9E74189A3
:10AC00000088228910FA82F2521A92B2002ACAD11E
:10AC1000D4F89035002BB3D02148FDF755FD0546FB
:10AC20000AE0FFF769FFD4F89035283D013BADB24B
:10AC3000C4F89035002BA3D0282D2046F1D870BD44
:10AC40000023C4F8843570BD027B002AE0D002885E
:10AC5000A7E7B4F8881539B15F20E21801339BB239
:10AC60008B4282F8D400F8D160184A1C8B1C14FA6D
:10AC700082F2572580F8D45014FA83F3752082F8B5
:10AC8000D4000331FD200022A4F8841583F8D400F9
:10AC9000A4F8862553E70023A4F886354FE700BFC4
:10ACA000D096FF1F550EFF1F0AA7FF1F01EB4101A2
:10ACB000490001F59671B1F5966F28BF4FF4966182
:10ACC000A0F88815704700BF4289038992B29BB2F1
:10ACD0009A421DD04289038992B29BB29A4208D30C
:10ACE000438901890288581A80B282420AD2002020
:10ACF000704702880389408912FA80F0C01A80B236
:10AD00008242F4D3084BA3FB0030C0F347107047D6
:10AD1000037B002BEBD10088A3F15533A3FB00305C
:10AD2000C0F34710704700BFABAAAAAA4FF416732E
:10AD300003FB01F1C0F88C15704700BF70B500250A
:10AD40000646294600F8045B142206F5005408F074
:10AD5000FFFF29464FF4075206F1180008F0F8FFEC
:10AD6000174BC4F8DC3142F20F7206F50750C4F8F5
:10AD7000E031C4F8E431A4F8E8212946C4F8D851F8
:10AD80002022C4F8EC51A4F8F05184F8F251343088
:10AD900008F0DEFF06F50850A4F8145220222946D8
:10ADA000163008F0D5FF632384F8383284F8425215
:10ADB000A4F83652C4F83C52A4F84052304670BD54
:10ADC0000F270F2700F50053002202701049C3F827
:10ADD000EC214FF0630C42F20F7083F838C2C3F8D5
:10ADE000D821C3F8DC11C3F8E011C3F8E411A3F8CB
:10ADF000E801A3F81422A3F83622A3F8F02183F87F
:10AE0000F221C3F83C22A3F8402283F84222704783
:10AE10000F270F2770B5044682B0002A00F0848007
:10AE2000434E4FF47A5E00207546B44616E09C45CA
:10AE3000B8BF9C469D42A8BF1D464B1D9BB2B3F5B3
:10AE4000875FA1F5865100F10100A1F11B0138BF18
:10AE5000194683B228BF89B29A420CD901F10C037A
:10AE600034F91330002BE2DC9E45A8BF9E469E427B
:10AE7000B8BF1E46E1E70EEB06030CEB05025B10C4
:10AE800003EB62065510A5EB660542F34F021BB2B9
:10AE900046F34F062DB2274927480195009603F047
:10AEA00019FE04F5005E9EF83832632B2CD004EBBB
:10AEB000430202F500520133DBB2A2F8F461A2F8BA
:10AEC00016520F2B8EF8383204F5075304F5085448
:10AED00003F1320304F1120422D800210A46AEF82D
:10AEE0001412AEF8361233F802CF588C6144024483
:10AEF0009C4209B212B2F6D109111211AEF8141225
:10AF0000AEF8362202B070BD04F50753323304F5B3
:10AF1000085412341A4622F8026F94425584FAD12A
:10AF200000228EF83822D8E7154616461346B2E7B7
:10AF300080C1FFFFA08A010020E6FF1F2DE9F04736
:10AF4000BDF82040BDF92470BDF92890002A00F01A
:10AF50008A800234454EBFB2A4B2C9F10008002570
:10AF60002FE04FEADC0E0CF0070C16F80CA013F8DB
:10AF70000EC02CEA0A0C03F80EC004F1FF3CCCF31F
:10AF8000CC0E0CF0070C13F80EA016F80CC04CEA0F
:10AF90000A0C03F80EC001F1050C1FFA8CFCBCF57D
:10AFA000875F28BFA1F5865105F101052CBF1B392C
:10AFB00061461FFA85FC28BF89B202346245A4B2FB
:10AFC00051D901F10C0EA4F1020C30F81EE0AEEBE9
:10AFD000070E0FFA8EFEC6451FFA8CFCC1DBBEF1D0
:10AFE000000F1CDBCE454FEADC0E0CF0070C13F80B
:10AFF0000EA016F80CC04CEA0A0C03F80EC004F1BF
:10B00000FF3CCCF3CC0E0CF0070C23DA16F80CA0A6
:10B0100013F80EC02CEA0A0C03F80EC0BBE74FEA87
:10B02000DC0E0CF0070C16F80CA013F80EC02CEA7E
:10B030000A0C03F80EC004F1FF3CCCF3CC0E0CF06C
:10B04000070C16F80CA013F80EC02CEA0A0C03F833
:10B050000EC0A0E713F80EA016F80CC04CEA0A0CBC
:10B0600003F80EC097E7BDE8F08700BF048C01002D
:10B070002DE9F04F00F500576049B7F8DA3103F5D4
:10B0800083560D36B6B2B6F5875F24BF733B9EB2CA
:10B090000322054689B05A4801F1170EB246002432
:10B0A0004FF47A5C4FF6FD79904612E0013221D0E0
:10B0B00013FB08440AF105039BB2B3F5875F03D382
:10B0C000AAF586531B3B9BB2714517D011F9012F8E
:10B0D0009A460AF10C0335F913309842B8BF184666
:10B0E0009C45A8BF9C46012A06D0032ADED113FB4B
:10B0F0000944DFE71C44DDE7E41ADBE7D7F8EC316D
:10B10000A3422EDA97F83832632B65D0B7F91422B0
:10B11000B7F9363202930023019200939846182221
:10B1200006AB31462846FFF709FF2A78DFF8D490AE
:10B1300042459B460CBF0223042305930DF11E0AD2
:10B14000552201E019F8012F1BF8010B504003F0C4
:10B150005BFDD34540445FFA80F8F3D1059B9845E9
:10B1600003D9002009B0BDE8F08FB7F8DA21C7F89D
:10B17000EC410523A7F8F03102F5835307339BB266
:10B18000B3F5875F28BFA2F17903A7F8E0312B78E8
:10B19000A7F8E821A7F8DE61D3B902F2BB739BB22E
:10B1A000B3F5875F28BFA2F62513A7F8E23102F2B4
:10B1B000BD739BB2B3F5875FA7F8E62128BFA2F65F
:10B1C0002312A7F8DC6134BFA7F8E431A7F8E42123
:10B1D000012009B0BDE8F08F0CEB0002A0EB620388
:10B1E00044F63E1101FB03F342F34F0243F3CF3326
:10B1F000A7F81422A7F836328CE700BF148C0100A0
:10B2000080C1FFFF0C8C010038B500F500550446E5
:10B21000B5F8D831264804EB83035B6823F07F43FD
:10B22000584003F0F7FC02282AD82046FFF720FFF9
:10B2300030B395F8F23143B3013BDBB2012B85F813
:10B24000F2311CD1B5F8E63103F2BB7292B2B2F51D
:10B25000875F28BFA3F62512A5F8E22103F2BD728D
:10B2600092B2B2F5875F2ABFA3F62313A5F8E421B3
:10B27000A5F8E43101220023227085F8F23138BDAF
:10B2800095F8F231002BD7D138BDC5F83C32A5F87E
:10B29000403208480121FDF73FFA06480121FDF739
:10B2A00047FA6322092385F8382285F8F23138BD40
:10B2B000A030FB00D096FF1F30B500F500549FB0C2
:10B2C000B4F8E221B4F8E431B4F8DA119A42054650
:10B2D00005D28A4219D88B4203D21FB030BD8A42B0
:10B2E000F9D8B4F8D831904805EB83035B6823F0B4
:10B2F0007F43584003F08EFC022802D82846FFF70F
:10B30000B7FEB4F8DA11B4F8E4318B42E5D1B4F801
:10B31000DC3103F1780189B2B1F5875F03D3A3F57E
:10B320008353083B99B2B4F91432B4F9362201932D
:10B33000002302920093082204AB2846FFF7FEFD8B
:10B340009DF8113003F00F0384F842320F2B31D8EF
:10B35000DFE803F0BF3030963030307930303030B5
:10B3600008303050B4F8E611B422FFF753FDB4F9B9
:10B370003612B4F91432B4F9E6216C4800916C49E4
:10B3800003F02CFBB4F91432B4F9362201930823EC
:10B3900002920093B4F8E61105ABB4222846FFF7F9
:10B3A000CDFD4FF0010C61488DF814C02E221946D6
:10B3B00002F0B2FFB4F8E82102F586531F339BB2C6
:10B3C000B3F5875F28BF02F1FF33A4F8E231531CC5
:10B3D0009BB2B3F5875F25BFA2F586521F3AA4F84A
:10B3E000E431A4F8E421002302222A70C4F8EC31ED
:10B3F0001FB030BDB4F8DC11D822FFF70BFDB4F953
:10B400003612B4F91432B4F9E6214848009149499A
:10B4100003F0E4FAB4F91432B4F9362201930823A4
:10B4200002920093B4F8DC1105AB2846D822FFF74E
:10B4300085FD4FF0010C3D488DF814C037221946A8
:10B4400002F06AFFB6E7B4F8DC11B422FFF7E2FCC1
:10B45000B4F93612B4F91432B4F9E6213348009144
:10B46000354903F0BBFAB4F91432B4F9362201932A
:10B47000082302920093B4F8DC1105ABB4228DE7E7
:10B48000B4F8DC114822FFF7C5FCB4F93612B4F960
:10B490001432B4F9E62125480091284903F09EFAB8
:10B4A000B4F91432B4F936220193082302920093BE
:10B4B000B4F8DC1105AB28464822FFF73FFD4FF0FA
:10B4C000010C1A488DF814C01322194602F024FF0B
:10B4D00070E7B4F8DC114FF4C672FFF79BFCB4F9C7
:10B4E0003612B4F91432B4F9E62110480091144927
:10B4F00003F074FAB4F91432B4F936220193082334
:10B5000002920093B4F8DC1105AB28464FF4C672E2
:10B51000FFF714FD4FF0010C04488DF814C06422AD
:10B52000194602F0F9FE45E7A030FB0020E6FF1FB8
:10B53000F08A0100808B0100208B0100508B0100FC
:10B54000C08A010070B500F50054BCB0B4F8E22127
:10B55000B4F8E411B4F8DA318A42054607D29A42C7
:10B5600007D9B4F8E0219A421BD03CB070BD9A4292
:10B5700001D99942F5D3B4F8D831504805EB83038B
:10B580005B6823F07F43584003F044FB022802D855
:10B590002846FFF76DFDB4F8DA31B4F8E0219A429D
:10B5A000E3D1B4F8F031052B18D1B4F8E82102F555
:10B5B00086531F339BB2B3F5875F28BF02F1FF3379
:10B5C000A4F8E231531C9BB2B3F5875F25BFA2F507
:10B5D00086521F3AA4F8E431A4F8E421B4F8DE114D
:10B5E0004FF458722846FFF715FCB4F93612B4F937
:10B5F0001432B4F9E82132480091324903F0EEF9EF
:10B60000B4F91432B4F9362201930823029200935C
:10B61000B4F8DE1105AB4FF458722846FFF78EFCE4
:10B62000B4F8F061013EB6B2A4F8F0613EB3A6F101
:10B630000406B6FA86F6B4F8403276098DF814603E
:10B640006BB91F48D92205A902F09EFE0023C4F859
:10B650003C32A4F84032C4F8EC313CB070BDD4F8B0
:10B660003C22B2FBF3F3C3F307218DF8ED1014482D
:10B670008DF8EE30DB2205A902F086FEE6E71048E1
:10B68000114903F015F931461048FDF745F83146E8
:10B690000E48FDF74DF80A4802F0AEFE42F20F7276
:10B6A00063232E70A4F8E02184F8383284F8F26124
:10B6B000C4F8EC6184F842623CB070BDA030FB007D
:10B6C00020E6FF1FB08B0100E08B0100D096FF1F2A
:10B6D000002B5AD02DE9F8435D1E00F50054EDB261
:10B6E000B4F8D8318146A2F1020801EB45058F1E5E
:10B6F00000261DE04846FFF787FDB4F8DA31013334
:10B700009BB2B3F5875F38BFA4F8DA31B4F8D8310B
:10B7100028BFA4F8DA6103F101039BB228BF84F8C3
:10B720004262052B28BF0023BD42A4F8D8312AD09D
:10B7300038F8020FD4F83C12B4F8402209EB830326
:10B740000844013237F9021FC4F83C02A4F8402231
:10B750005A6800294FEA4202B8BF42F001025A601B
:10B76000B4F8DA3199F800200C33012A29F81310C3
:10B7700005D0022ABED14846FFF7E4FEBDE74846A1
:10B78000FFF79AFDB9E7BDE8F88370472DE9F0416E
:10B79000044600254FF47A60258120806581657319
:10B7A000257306F091FA294660604FF4966204F121
:10B7B000C00008F0CDFAF02304F128082027A4F8EF
:10B7C000743541F27073C4F8783504F148063A468E
:10B7D0002946C4F87055C4F87C55404608F0B8FABC
:10B7E00029467822304608F0B3FA064B2361064B0F
:10B7F0006361064BC4F81880A78326626362204603
:10B80000BDE8F081050008003C0FFF1F8C0FFF1FF3
:10B81000122A73D970B544890389A4B29BB29C42A1
:10B8200010D044890389A4B29BB29C4268D2058996
:10B830000488438914FA83F35B1B9BB29C4205D2B4
:10B84000052070BD037B002BFAD103889A42F7D8FC
:10B85000037B03F0FF05002B5BD1446803899BB297
:10B86000013AE254038901339BB2038104890388BE
:10B87000A4B29BB29C4228BF058104894389A4B22B
:10B880009BB29C4242D000239C464FF0010E24E024
:10B8900046680489A4B2013306F804C0B0F808C0B1
:10B8A0000CF1010C1FFA8CFCA0F808C0B0F808C01D
:10B8B00004881FFA8CFCA4B2A44528BF0581B0F807
:10B8C00008C044891FFA8CFCA4B2A445DBB208BFAF
:10B8D00080F80CE093429C460ED2047B8C4404F02A
:10B8E000FF059CF801C0002CD2D00133DBB293429B
:10B8F00080F80DE09C46F0D3002070BD0420704716
:10B90000438904891B1B9BB2048897E701230373B7
:10B91000B9E701234373013AB5E700BF70B598B0AA
:10B92000054602AB04AC4FF4D27640F2EC4E4FF633
:10B93000143C4FF65C6001F0C002802A26D0C02A79
:10B9400021D0F2B1A3F800C0023389009C42C9B2F1
:10B95000F1D1224602A905F11000042306F0BAFB3A
:10B960000EAA214605F11C00142307F09DF80023C0
:10B970000093074814230EAA0421FCF7E3FD18B036
:10B9800070BD1880E0E7A3F800E0DDE71E80DBE78C
:10B99000D096FF1F30B599B00446002502A904AA2D
:10B9A00004231030CDE9025506F094FB04A904F1FC
:10B9B0001C000EAA142307F077F8044800951423FE
:10B9C0000EAA0421FCF7BEFD19B030BDD096FF1FB2
:10B9D000B0F8703570B504460BB35E485E4EFCF7A8
:10B9E00073FE054617E0B4F872355A1C2344A4F8D8
:10B9F000722593F8C010FFF791FF3378143DADB274
:10BA00001BB1D4F87835C4F87C35B4F87225B4F895
:10BA100070359A424BD2142D2046E4D870BD41892E
:10BA2000028989B292B2914245D04189028989B294
:10BA300092B291421AD202894189521A92B2F2B15B
:10BA4000464A1278002A3BD1B4F8741500297CD0FC
:10BA50007720E21801339BB28B4282F8C000F8D104
:10BA6000A4F870350023A4F87235B6E74189008840
:10BA7000228910FA82F2521A92B2002AE0D1D4F846
:10BA80007C35002BCAD03348FCF71EFE05460AE081
:10BA9000FFF780FFD4F87C35143D013BADB2C4F80C
:10BAA0007C35002BBAD0142D2046F1D870BD002370
:10BAB000C4F8703570BD027B002AE0D00288BEE772
:10BAC0002189628989B292B291423BD061686289D0
:10BAD00092B200208D5C20736289013292B2628141
:10BAE0006189228889B292B2914228BF6081002D7B
:10BAF0002BD0ADB2002019E06168628992B28E5CF1
:10BB000020736289013292B262816189228889B28E
:10BB100092B2914228BF60815A1C92B22344AA4239
:10BB2000A4F8702583F8C0609CD0134621896289EF
:10BB300089B292B29142DFD1227B02F0FF06002A45
:10BB4000DAD1E9E7227B002AC0D10023A4F87235BC
:10BB500095E700BFD096FF1F550EFF1F0AA7FF1FD6
:10BB600001EB4101890001F51671B1F5966F28BF0F
:10BB70004FF49661A0F87415704700BF428903899D
:10BB800092B29BB29A421DD04289038992B29BB273
:10BB90009A4208D3438901890288581A80B28242A6
:10BBA0000AD20020704702880389408912FA80F087
:10BBB000C01A80B28242F4D3074BC008A3FB003006
:10BBC000C0B27047037B002BEBD10088024BC0084A
:10BBD000A3FB0030C0B270475F427B094FF496630D
:10BBE00003FB01F1C0F87815704700BF70B504463B
:10BBF00000254FF47A602581208065816573257367
:10BC000006F062F829466060C82204F5B87008F0B2
:10BC10009FF804F11C064823A4F83C32C4F83852BB
:10BC20004FF4AA722946304608F092F8034B666139
:10BC300006222282A361204670BD00BFCC0FFF1FE9
:10BC4000B0F8382203460AB10120704741890289C1
:10BC500089B292B2914218D04189028989B292B2D6
:10BC600091420AD342890188008911FA80F0801A32
:10BC700080B2003818BF0120704700895B89C01A64
:10BC800080B2003818BF01207047027B02F0FF002D
:10BC9000002ADAD01888ECE7442A01D00420704743
:10BCA0004289038992B29BB29A4230B549D0428907
:10BCB000038992B29BB29A4208D3438904890288CD
:10BCC0001B1B9BB293420AD9052030BD0489028810
:10BCD000438912FA83F31B1B9BB29342F4D8432B84
:10BCE000F2D94A1E4FF0010E43311DE04568038929
:10BCF0009BB205F803C0038901339BB20381B0F8FE
:10BD000008C003881FFA8CFC9BB29C4528BF0481A5
:10BD1000B0F808C043891FFA8CFC9BB29C4508BF51
:10BD200080F80CE08A420AD0037B12F801CF03F0BE
:10BD3000FF04002BDAD08A4280F80DE0F4D1002015
:10BD400030BD037B002BBFD10388C8E72DE9F0414C
:10BD50008046ADF5227D0E4614270EE00FCCACE8F0
:10BD60000F000FCCACE80F0094E803001437760006
:10BD7000B42F8CE80300F6B218D002AB03EB470CEB
:10BD8000ACF1280C3306134C134DE646E6D50FCD27
:10BD9000AEE80F000FCDAEE80F0095E803001437B2
:10BDA0007600B42F8EE80300F6B2E6D152AA02A9BB
:10BDB00008F11000A02306F077FE00230093074847
:10BDC000A02352AA0621FCF7BDFB0DF5227DBDE89C
:10BDD000F08100BF2C8C0100548C0100D096FF1F15
:10BDE00038B54289038992B29BB29A42044663D025
:10BDF0004289038992B29BB29A4236D20389428920
:10BE00009B1A9BB2002B39D0B4F83822002A38D1C3
:10BE1000384B1B78002B54D010461AE061686389B8
:10BE20009BB211F803C02073638901339BB2638115
:10BE30006189238889B29BB2994228BF6081531CD3
:10BE40009BB22244442BA4F8383282F870C145D00A
:10BE50001A462189638989B29BB29942DED1237B3C
:10BE600003F0FF0C002BD9D1E9E74289018803894F
:10BE700011FA83F39B1A9BB2002BC5D1B4F8383268
:10BE8000CBB11D48FCF720FC054611E0B4F83A326E
:10BE90005A1C2344A4F83A2293F87011FFF756FF76
:10BEA000B4F83A22B4F83832A03D9A42ADB219D271
:10BEB000A02D2046EAD838BD037B002BDED00388B6
:10BEC000A0E7B4F83C1289B1AA20A318013292B2BB
:10BED0008A4283F87001F8D1A4F838220023A4F82C
:10BEE0003A32CEE70023C4F8383238BDA4F83A120B
:10BEF00038BD00BF0AA7FF1FD096FF1F01EB41010D
:10BF000049084831962928BF9621A0F83C1270476D
:10BF10004289038992B29BB29A421DD04289038919
:10BF200092B29BB29A4208D3438901890288581A77
:10BF300080B282420AD20020704702880389408979
:10BF400012FA80F0C01A80B28242F4D3084BA3FBED
:10BF50000030C0F387107047037B002BEBD10088C3
:10BF6000A3F10F33A3FB0030C0F38710704700BF6D
:10BF7000F1F0F0F0022905D0032907D0012903D000
:10BF80000020704704F0B6B905F0ECBB04F068BDC2
:10BF9000022905D0032907D0012903D000207047CA
:10BFA00004F090B905F078BC04F042BD022908B550
:10BFB00005D003290BD0012905D0002008BD04F0CD
:10BFC000ADF9C0B208BD05F0A9FBC0B208BD04F0D0
:10BFD0005BFDC0B208BD00BF10B58C46BCF1020FBE
:10BFE0009DF808401046194616D0BCF1030F0BD03F
:10BFF000BCF1010F00D010BD05F0CAFB002CFAD037
:10C00000BDE8104005F06CBC04F0F2FC002CF2D04E
:10C01000BDE8104004F000BD04F0C0F8002CEAD0E8
:10C02000BDE8104004F042B9022907D003292DE9E8
:10C03000F8432AD0012905D0BDE8F88316481146F7
:10C0400005F0CABC154D164C2E68164FDFF85C90F3
:10C0500040F2EE2804E0B3F5FA6FEDD805F03CFEAF
:10C0600005F03AFE237843B13B78DB0705D52B6812
:10C07000D9F800209B1A0E2BDED82B6822789B1B48
:10C08000002AE8D14345E9D9D6E7BDE8F843064898
:10C09000114605F059BD00BF6810FF1F8C0000203D
:10C0A00084020020A80200207C10FF1FAC020020A8
:10C0B00030B58FB08579C47A027A017843790395D7
:10C0C0000D94847A029303790193C3780093837863
:10C0D0000C94447A0B94447B0A94047B0994C2F335
:10C0E00080140894C2F34015D40907940695C579C5
:10C0F00002F00F0401EB8101427803480594049596
:10C10000F9F768FC0FB030BD4889FF1F30B5A5B006
:10C11000E0230C788DF80C30F2238DF80E308CB3C0
:10C120004FF0030CACF102030CF190050DEB050E82
:10C13000DBB20EF8844CCC5C0CF10103E6465FFAEE
:10C1400083FC002CEED10EF10303DCB20EF1020EE3
:10C150005FFA8EFE23460CF190010DEB010C0EF1FF
:10C1600090010DEB010EC2F30725012100910CF89F
:10C17000845C0EF8842C03AA8DF80D40FFF72CFF89
:10C1800025B030BD05234FF0040E1C464FF0030CC4
:10C19000E1E700BF70B5044600254FF4B9764FF4CF
:10C1A0000072294607F0D4FDA4F81052C4F80052DA
:10C1B000A4F8125284F80452A4F8086284F81452C5
:10C1C00084F81552304605F07FFDA4F82852C4F8D3
:10C1D0000C02A4F82A52C4F81852A4F81C52A4F86D
:10C1E000206284F82C5284F82D52304605F06CFD04
:10C1F000C4F82402204670BD30B504468DB07648A0
:10C20000FCF7B0FE754A764B12781B788DF8132038
:10C210004FF4A751ADF8101001218DF812106E489F
:10C220008DF814300DF10F020DF10E01FCF776FEC2
:10C230009DF80E302BB19DF8143043F002038DF8B9
:10C2400014306548FCF788FE28B19DF8143043F09F
:10C2500004038DF814306048FCF776FE28B19DF891
:10C26000143043F008038DF814305B48FCF782FE6D
:10C270009DF8143008B143F010039DF80F200AB167
:10C2800043F02003574A58491278087843EA82134A
:10C2900000228DF814308DF81520002840F097808A
:10C2A000524B8DF816001B78002B4FD0504B1B784B
:10C2B000002B00F084804F48F7F7B8FB03464D4849
:10C2C0008DF81730F7F7E0FB4B4A034610788DF8EE
:10C2D0001830002842D0494803F036FA484B8DF810
:10C2E0001900187800283FD04648FFF747FC464B16
:10C2F0008DF81A00187800283CD04448FEF7E4FC7A
:10C30000434B8DF81B001878002839D04148FDF7C1
:10C31000A5FD414B8DF81C001878002836D03F4809
:10C32000FBF7DAF93E4B8DF81D001878002833D062
:10C330003C48FFF7EDFD3C4B8DF81E0019780029B5
:10C3400030D03A48F4F780FE01462BE08DF81730E4
:10C35000294A8DF8183010780028BCD1284B8DF868
:10C36000190018780028BFD1274B8DF81A001878CB
:10C370000028C2D1264B8DF81B0018780028C5D1A3
:10C38000254B8DF81C0018780028C8D1244B8DF857
:10C390001D0018780028CBD1234B8DF81E0019788A
:10C3A0000029CED100258DF81F100095142304AA72
:10C3B000204601210895FFF70FFE0DB030BD0A237E
:10C3C0001B488DF81730F6F72FFA0346C0E71948D7
:10C3D000F9F740F864E700BFD096FF1F09A7FF1FD9
:10C3E0000AA7FF1F08A7FF1F540EFF1F530EFF1FB2
:10C3F000550EFF1FE464FF1F5B0EFF1F90FBFF1F26
:10C40000590EFF1F60DEFF1F580EFF1F88B6FF1F6B
:10C41000570EFF1F0CA2FF1F560EFF1F4889FF1F5C
:10C420005A0EFF1FE0E3FF1F520EFF1F4C20FF1F9D
:10C43000F83DFF1FA086FF1F30B5B5B040F27F3337
:10C44000184AADF80C30044617480292FCF746FF34
:10C45000102200218DF80E000DF10F0007F078FC7E
:10C460000DF10F011048114DFCF73AFF4D21172334
:10C470008C4601E08C46A95C03F1D0006844A3F12E
:10C4800015020133D2B200F8C8CCDBB20029F1D1D9
:10C49000009102AA012120468DF80930FFF79CFD8A
:10C4A00035B030BDE0000002D096FF1FAC91010016
:10C4B000072A46D92DE9F04F8E794B788878CF78C6
:10C4C00091F8048091F8059099B0154603EB830329
:10C4D00006F0010AC6F3400B0A780890C6F38006FE
:10C4E00009965B002E464FF0070C00200D4600F128
:10C4F00060010CF1010E15F80C4069445FFA8EFCE6
:10C500000130B445C0B201F8344CF0DB00F16001F9
:10C510000DEB0104099E0899009100250696CDF8BF
:10C5200014B0CDF810A0CDF80C90CDF8088001978C
:10C530000BA904F8345C0448F9F7DEF919B0BDE83A
:10C54000F08F0420704700BF4889FF1F052A36D9A5
:10C550002DE9F04316464B78CA7891F8028091F89D
:10C56000049002EB820703EB83030A7893B05B002D
:10C570007F004FF0050C002000F148040CF101058C
:10C580000DEB040E11F80C400EF8344C5FFA85FCEC
:10C590000130B445C0B2EFDB00F148010DEB010CF6
:10C5A0000024CDF808900197CDF8008005A90CF87B
:10C5B000344C0448F9F7E2F913B0BDE8F0830420E5
:10C5C000704700BF4889FF1F032A32D92DE9F04187
:10C5D0008B7891F80380164603EB8307042E0A78C4
:10C5E0004B7890B04FEA470725D04FF0040C00205D
:10C5F00000F140040CF101050DEB040E11F80C40A4
:10C600000EF8344C5FFA85FC0130B445C0B2EFDB64
:10C6100000F140010DEB010C0024CDF804800097DF
:10C6200003A90CF8344C0548F9F73EFA10B0BDE800
:10C63000F081042070470020EAE700BF4889FF1F0F
:10C6400010B54B1EA4B00C466B2B6DD8DFE813F071
:10C650009003560320030403E802CC02B0026C00EE
:10C660006C0094026C006C006C006C006C006C0040
:10C670006C006C006C006C006C006C006C006C005A
:10C680006C006C006C006C006C006C006C006C004A
:10C690006C006C006C006C006C006C006C006C003A
:10C6A0006C006C006C006C006C006C006C006C002A
:10C6B0006C006C006C006C006C006C006C006C001A
:10C6C0006C006C006C006C006C006C006C006C000A
:10C6D0006C006C006C006C006C006C006C006C00FA
:10C6E0006C006C006C006C006C006C006C006C00EA
:10C6F0006C006C006C006C006C006C006C006C00DA
:10C700006C006C0078025C0240026C00240208029B
:10C710006C00EC01A5016C0089016D01510136012D
:10C720001B010001E500B200AA4B93F80432E3B10B
:10C73000E022F123A8488DF80C208DF80E304D2210
:10C74000032303F19001694401F8842C9A1ED2B2AC
:10C750000133825CDBB2002AF3D101219D480091B4
:10C7600003AA8DF80D30FFF737FC9C48F7F774FCEF
:10C770009B48F6F7B1F89B48F5F71EFB9A48F6F789
:10C78000E1FA9A4802F0CAFA042C40F0DE82984896
:10C79000FDF78CFD9748FCF7E5FD9748F9F75AF847
:10C7A0009648F4F773FD9648214624B0BDE8104042
:10C7B000FBF7C2BF874B93F80432E3B1E022F123C9
:10C7C00090488DF80C208DF80E304D22032303F194
:10C7D0009001694401F8842C9A1ED2B20133825C24
:10C7E000DBB2002AF3D101217A48009103AA8DF827
:10C7F0000D30FFF7F1FB7948F7F72EFC7848F6F794
:10C800006BF87848F5F7D8FA7748F6F79BFA032CD7
:10C81000B7D17D48FEF7D6FAB9E76E4B93F80432EC
:10C82000002BE8D0E022F12378488DF80C208DF819
:10C830000E304D22032303F19001694401F8842C4A
:10C840009A1ED2B20133825CDBB2002AF3D1CAE76E
:10C85000604B93F80432002BCDD0E022F1236C49D9
:10C860008DF80C208DF80E304D22032303F190003B
:10C87000684400F8842C9A1ED2B201338A5CDBB281
:10C88000002AF3D1AFE7534B93F80432002BB2D018
:10C89000E022F1235F488DF80C208DF80E304D22F8
:10C8A000032303F19001694401F8842C9A1ED2B24B
:10C8B0000133825CDBB2002AF3D194E7454B93F855
:10C8C0000432002B97D0E022F12353488DF80C203E
:10C8D0008DF80E304D22032303F19001694401F8D5
:10C8E000842C9A1ED2B20133825CDBB2002AF3D1CF
:10C8F00079E7384B93F80432002B3FF47CAFE02209
:10C90000F12346488DF80C208DF80E304D2203237C
:10C9100003F19001694401F8842C9A1ED2B20133CC
:10C92000825CDBB2002AF3D15DE72A4B93F8043234
:10C93000002B3FF460AFE022F12335498DF80C2045
:10C940008DF80E304D22032303F19000684400F867
:10C95000842C9A1ED2B201338A5CDBB2002AF3D156
:10C9600041E71C4B93F80432002B3FF444AFE02224
:10C97000F1232B488DF80C208DF80E304D22032327
:10C9800003F19001694401F8842C9A1ED2B201335C
:10C99000825CDBB2002AF3D125E70E4B93F8043218
:10C9A000002B3FF428AFE022F1231E488DF80C2025
:10C9B0008DF80E304D22032303F19001694401F8F4
:10C9C000842C9A1ED2B20133825CDBB2002AF3D1EE
:10C9D00009E700BF20E6FF1FD88E0100D065FF1FCA
:10C9E000EC42FF1F3C27FF1F3C48FF1F50E8FF1F82
:10C9F0000CA7FF1F209AFF1F4889FF1F4C23FF1F12
:10CA0000D096FF1FBC8E01001CBCFF1F0C8E0100C6
:10CA1000888D0100EC8D0100CC8D0100A88D0100F6
:10CA20009C8E0100148D0100A74B93F80432002B5B
:10CA30003FF4E1AEE022F123A4488DF80C208DF8FC
:10CA40000E304D22032303F19001694401F8842C38
:10CA50009A1ED2B20133825CDBB2002AF3D1C2E665
:10CA6000994B93F80432002B3FF4C5AEE022F1233A
:10CA700097488DF80C208DF80E304D22032303F1DA
:10CA80009001694401F8842C9A1ED2B20133825C71
:10CA9000DBB2002AF3D1A6E68B4B93F80432002BCD
:10CAA0003FF4A9AEE022F1238A488DF80C208DF8DE
:10CAB0000E304D22032303F19001694401F8842CC8
:10CAC0009A1ED2B20133825CDBB2002AF3D18AE62D
:10CAD0007D4B93F80432002B3FF48DAEE022F1231E
:10CAE0007D488DF80C208DF80E304D22032303F184
:10CAF0009001694401F8842C9A1ED2B20133825C01
:10CB0000DBB2002AF3D16EE66F4B93F80432002BB0
:10CB10003FF471AEE022F12370488DF80C208DF8BF
:10CB20000E304D22032303F19001694401F8842C57
:10CB30009A1ED2B20133825CDBB2002AF3D152E6F4
:10CB4000614B93F80432002B3FF455AEE022F12301
:10CB500063488DF80C208DF80E304D22032303F12D
:10CB60009001694401F8842C9A1ED2B20133825C90
:10CB7000DBB2002AF3D136E6534B93F80432002B94
:10CB80003FF439AEE022F12356488DF80C208DF8A1
:10CB90000E304D22032303F19001694401F8842CE7
:10CBA0009A1ED2B20133825CDBB2002AF3D11AE6BC
:10CBB000454B93F80432002B3FF41DAEE022F123E5
:10CBC00049488DF80C208DF80E304D22032303F1D7
:10CBD0009001694401F8842C9A1ED2B20133825C20
:10CBE000DBB2002AF3D1FEE5374B93F80432002B79
:10CBF0003FF401AEE022F1233C488DF80C208DF883
:10CC00000E304D22032303F19001694401F8842C76
:10CC10009A1ED2B20133825CDBB2002AF3D1E2E584
:10CC2000294B93F80432002B3FF4E5ADE022F123C9
:10CC30002F488DF80C208DF80E304D22032303F180
:10CC40009001694401F8842C9A1ED2B20133825CAF
:10CC5000DBB2002AF3D1C6E51B4B93F80432002B5C
:10CC60003FF4C9ADE022F12322488DF80C208DF865
:10CC70000E304D22032303F19001694401F8842C06
:10CC80009A1ED2B20133825CDBB2002AF3D1AAE54C
:10CC90000D4B93F80432002B3FF4ADADE022F123AD
:10CCA00015488DF80C208DF80E304D220B4603F1FF
:10CCB0009001694401F8842C9A1ED2B20133825C3F
:10CCC000DBB2002AF3D18EE520E6FF1F348D010090
:10CCD000508D01006C8D01002C8E0100508E0100E2
:10CCE000788E0100048D0100E08C0100F08C0100C1
:10CCF000CC8C0100BC8C0100A08C0100354B93F85A
:10CD00000432E3B1E022F12333488DF80C208DF892
:10CD10000E304D22032303F19001694401F8842C65
:10CD20009A1ED2B20133825CDBB2002AF3D1012118
:10CD30002848009103AA8DF80D30FFF74DF92748D8
:10CD4000F7F78AF9264801F0E9FF2648FEF73AF896
:10CD5000052C3FF41FAD2448FDF7A8FA072C3FF43B
:10CD60001CAD2248FCF7FEFA0A2C3FF419AD14E57D
:10CD7000184B93F80432E3B1E022F1231C488DF8FC
:10CD80000C208DF80E304D22032303F190016944ED
:10CD900001F8842C9A1ED2B20133825CDBB2002AE5
:10CDA000F3D101210B48009103AA8DF80D30FFF754
:10CDB00013F91048F5F790FD0F48F4F7FDFF0F4801
:10CDC000F5F7C0FF064801F0A9FF0648FDF7FAFF96
:10CDD000C1E700BF20E6FF1F908C0100D065FF1F58
:10CDE00050E8FF1F1CBCFF1F0CA7FF1F209AFF1F4E
:10CDF0007C8C0100EC42FF1F3C27FF1F3C48FF1FBB
:10CE0000242A40F27A812DE9F04F0D78C5F3001203
:10CE100080F804224C788A78CE78A9B0322E10920D
:10CE200004F02002119204F040020B4604F00207C5
:10CE300004F0040804F0080904F0100A0F9200F24C
:10CE400034810979052940F22B816C2900F22D816A
:10CE50005A2940F22E81B24AA1F15B0C5FFA8CFC98
:10CE600022FA0CF2D20740F1208193F806C0CDF8E7
:10CE700050C093F807C0CDF854C093F808C0CDF85F
:10CE800058C093F809C0CDF85CC093F80AC0CDF83B
:10CE900060C093F80BC0CDF864C093F80CC0CDF817
:10CEA00068C093F80DC0CDF86CC093F80EC0CDF8F3
:10CEB00070C093F80FC0CDF874C093F810C0CDF8CF
:10CEC00078C093F811C0CDF87CC093F814C093F8E3
:10CED0001AB0CDF880C093F815C05A79CDF884C047
:10CEE00093F816C01392BBF10F0FCDF888C093F8DA
:10CEF00017C0CDF88CC000F2D88093F81CC0CDF8D4
:10CF000048C0ACF17C0CDA7E2492BCF10E0F00F22A
:10CF1000CC8093F81DC0CDF894C093F81EC0DB7F81
:10CF2000CDF898C02793FFF78BFB7E497E4804F02D
:10CF300001040C70E943C1F3C011017031467B4814
:10CF4000F8F77AFA003F7A497A4818BF01270F703C
:10CF50003146F5F797FC59467748F6F7F3FF5946FF
:10CF60007648F5F7D7FE249A74481146F5F7DEFEA9
:10CF700059467348F5F708F959467248F5F77EFEA9
:10CF8000B8F10008704A714818BF4FF001083146E7
:10CF900082F8008002F0CAFB209A6C48C5F3C001F9
:10CFA00002F004FCB9F10009694A6A4818BF4FF061
:10CFB0000109314682F80090FEF7D2FD21996548BB
:10CFC000FEF70CFEBAF1000A634A644818BF4FF03E
:10CFD000010A314682F800A0FDF768FE22995F48F9
:10CFE000FDF7A4FE0F9F5E495E483A1E18BF01225E
:10CFF0000A703146FCF724FF23995A48FCF760FF7A
:10D000003146109E584A594806F001041470FEF744
:10D0100075FF57482599C6F3400202705548F4F74A
:10D020000DF8129B269A5448A3F1800149B2279B20
:10D03000F3F74AFE1C991B9B0791139A16991E9CA5
:10D040001D9806930191149B119909940890189CBE
:10D0500017981F9E0394803A02900B92081E159A0F
:10D06000464C0A96A3F1800318BF01200C9300924E
:10D07000C5F38003C5F3400205F001011A9F199E14
:10D080000597C5F3401504960D9520703C48FBF7B5
:10D09000D5FE3B48FBF7BEFB002029B0BDE8F08F72
:10D0A00001291DD1E2073FF5E0AE042029B0BDE81B
:10D0B000F08F072906D90A29F7D1119A002A7FF49F
:10D0C000D4AEF2E7032904D1B8F1000F7FF4CDAE5E
:10D0D000EBE704290AD1B9F1000F7FF4C6AEE4E70B
:10D0E0000229EFD1002F7FF4C0AEDEE7052906D17B
:10D0F000BAF1000F7FF4B9AED7E7042070470729D3
:10D1000004D10F9A002A7FF4B0AECEE7062904D1ED
:10D11000109AD2073FF5A9AEC7E70A29CDD0A4E6F9
:10D12000BFFD0300540EFF1F550EFF1FA086FF1FFB
:10D13000530EFF1FF83DFF1FE464FF1F3C48FF1F15
:10D140003C27FF1FEC42FF1F5B0EFF1F90FBFF1FE2
:10D15000590EFF1F60DEFF1F580EFF1F88B6FF1F0E
:10D16000570EFF1F0CA2FF1F5A0EFF1FE0E3FF1F09
:10D17000520EFF1F4C20FF1FC016FF1F560EFF1F31
:10D18000D096FF1F3AB308B52B4B09781B788B421A
:10D1900030D06C290FD85A2910D9284BA1F15B0245
:10D1A000D2B2D340DB0706D5012917D002291AD104
:10D1B000234B1B7853B90421084608BD0729F3D92E
:10D1C0000A29F8D11F4B1B78002BF4D0FFF738FA4F
:10D1D0000021084608BD0421084670471A4B1B78F9
:10D1E000002BF3D1E7E7032907D1184B1B78002B5D
:10D1F000ECD1E0E70021084608BD042904D1144B16
:10D200001B78002BE2D1D7E7052904D1114B1B78FD
:10D21000002BDBD1CFE7072904D10F4B1B78002B64
:10D22000D4D1C8E7062904D10C4B1B78002BCDD1F3
:10D23000C1E70A29C6D0C9E709A7FF1FBFFD030040
:10D24000530EFF1F560EFF1F540EFF1F5B0EFF1FD6
:10D25000590EFF1F580EFF1F570EFF1F5A0EFF1FBC
:10D2600010B54FF4E12204460121FEF7DDFE204611
:10D270004FF41652BDE810400321FEF7D5BE00BFA3
:10D28000F0B5044687B01546912900F2B980DFE871
:10D2900011F0B203AF03A80398038D03B700B700E2
:10D2A000B7001403B7000303B700B700B700B70017
:10D2B000B700EF02DB02B700C702B700B700B70044
:10D2C000B700AE02B7008A02B700790265025402C5
:10D2D000B7003D02B700B700B700B700B700B7000E
:10D2E000B700B700B700B700B700B700B700B70086
:10D2F000B70028021302B700B700B700B700B700A5
:10D30000B700B700B700B700B700B700B700B70065
:10D31000B700C201B700B700B700B700AB01940176
:10D32000B700B7007D01B700B700B700B700B7007E
:10D33000B7006601B700B700B700B7004F01B700EC
:10D34000B700B700B700B700B700B700B700B70025
:10D35000B7003C01290114010101B7009200B70098
:10D36000B700B700B700B700B700B700B700B70005
:10D37000B700B700B700B700B700B700B700B700F5
:10D38000B700B700B700B700B700B700B700B700E5
:10D39000B700CC00B700B700B700B700B700B700C0
:10D3A000B700B700B700B700B700B700B700B700C5
:10D3B000B700B200B200A34A12783AB1A24E327856
:10D3C000002A00F0AA830A2A00F0A7830222154649
:10D3D0009E4890F8043213B19D49FEF797FE9D498F
:10D3E000002300930491052304AA012120468DF80F
:10D3F0001450FEF7F1FD0023C4F8003207B0F0BD71
:10D400004FF4BC6001220023ADF810007F20009390
:10D410008DF812008DF813108DF814201146052395
:10D4200004AA2046FEF7D8FDE5E7002BE3D0013B38
:10D43000691E15FA83F3012521E0D4F80C62B4F8D3
:10D44000102292B2B054B4F81022013292B2A4F871
:10D450001022B4F81002B4F8082280B292B29042BE
:10D4600028BFA4F810C2B4F81002B4F8122280B297
:10D4700092B2904208BF84F814528B42BBD094F809
:10D48000142211F8010F02F0FF0C002AD5D084F805
:10D490001552F2E729461A46FFF796F80546002886
:10D4A00000F0EA82694890F804321BB16A492AB256
:10D4B000FEF72CFE6949002393E70D2B40F2D3823F
:10D4C0002846FEF7F5FD0546002800F0818302B2EC
:10D4D0005E4890F8043213B16149FEF717FE6149C6
:10D4E00000237EE729461A46FFF730F80546002854
:10D4F00000F0C782554890F804321BB15A492AB24D
:10D50000FEF704FE594900236BE729461A46FEF749
:10D51000CFFF0546002800F0B2824C4890F8043254
:10D520001BB153492AB2FEF7F1FD5249002358E7D7
:10D53000514A12783AB1444A1278002A00F00A831C
:10D540000A2A00F0078302221546404890F8043268
:10D5500013B14A49FEF7DAFD4949002341E7494A38
:10D5600012783AB1384E3278002A00F0FE82062A4C
:10D5700000F0FB8202221546344890F8043213B1C1
:10D580004149FEF7C3FD414900232AE7404A12788A
:10D590003AB12D4E3278002A00F0F282072A00F0CC
:10D5A000EF8202221546294890F8043213B1394916
:10D5B000FEF7ACFD3849002313E7354A12783AB13B
:10D5C000214E3278002A00F0F082072A00F0ED8226
:10D5D000022215461D4890F8043213B12F49FEF778
:10D5E00095FD2F490023FCE6294A12783AB1164EE0
:10D5F0003278002A00F09C82072A00F099820222E9
:10D600001546124890F8043213B12649FEF77EFD04
:10D6100025490023E5E6254A12783AB10A4E3278C8
:10D62000002A00F0B782052A00F0B48202221546D3
:10D63000064890F8043213B11D49FEF767FD1D49F5
:10D640000023CEE6560EFF1F09A7FF1F20E6FF1F8F
:10D6500074910100E0057F654C8F0100E0057F6358
:10D660002C8F0100E0057F620C8F0100E0057F61D7
:10D67000EC8E0100E0057F60520EFF1F90910100CB
:10D68000E0057F555A0EFF1F54910100E0057F50C1
:10D69000570EFF1F38910100E0057F4914910100EA
:10D6A000E0057F46EC900100E0057F45580EFF1F26
:10D6B000D0900100E0057F409B4A12782AB19B4E32
:10D6C000327812F0FB0F00F00D82022215469848C6
:10D6D00090F8043213B19749FEF718FD96490023DC
:10D6E0007FE6914A12782AB1904E327812F0FB0F01
:10D6F00000F00182022215468D4890F8043213B1E1
:10D700008E49FEF703FD8E4900236AE68D4A1278A2
:10D710003AB1864E3278002A00F0D981032A00F00F
:10D72000D68102221546824890F8043213B1864908
:10D73000FEF7ECFC8549002353E6854A1278002A5F
:10D7400040F0BA8102221546794890F8043213B1AC
:10D750008049FEF7DBFC8049002342E67C4A1278D0
:10D76000002A00F07D81012B00F05C820422154626
:10D770006F4890F8043213B17849FEF7C7FC784936
:10D7800000232EE6724A1278002A40F07C810222A1
:10D790001546674890F8043213B17249FEF7B6FC9B
:10D7A000714900231DE66A4A1278002A00F045817B
:10D7B0005E4E327812F0FD0F40F03F816B4A1278D6
:10D7C000002A00F04582294669481A46F6F71EF8F5
:10D7D0000546002D00F0F3812AB2554890F8043236
:10D7E00013B16449FEF792FC63490023F9E5584AF6
:10D7F00012784AB14D4E327812F0FD0F04D15B4AD7
:10D800001278002A40F0B38202221546484890F868
:10D81000043213B15749FEF779FC58490023E0E57B
:10D82000574B1B7823B1414E3378012B40F297823E
:10D83000022215463E4890F8043213B15149FEF7D2
:10D8400065FC51490023CCE54D4A127822B1374E90
:10D850003278012A40F2798202221546344890F843
:10D86000043213B14949FEF751FC49490023B8E598
:10D87000434A127822B12D4E3278012A40F2528268
:10D88000022215462A4890F8043213B14149FEF7A6
:10D890003DFC41490023A4E5244A1278002A00F007
:10D8A000008105221546224890F8043213B13B4905
:10D8B000FEF72CFC3A49002393E51C4E3278632A8C
:10D8C00000F088810227A2F15C01C9B2062900F2AA
:10D8D000CD806FF04D0040FA01F1C90740F195800D
:10D8E0005D2A00F081815B2A00F092816C2A00F0B1
:10D8F0008581652A00F08280002F00F0CF800C48DF
:10D9000090F804321BB127493AB2FEF7FFFB2649D3
:10D9100004910023009304AA0523012120468DF8D9
:10D920001470FEF759FB66E5590EFF1F09A7FF1F8C
:10D9300020E6FF1FB4900100E0057F3198900100C0
:10D94000E0057F305B0EFF1F74900100E0057F2033
:10D95000530EFF1F58900100E0057F1E1C90010030
:10D96000E0057F1D38900100E0057F1C550EFF1F6C
:10D97000E464FF1F00900100E0057F1AE0057F18B6
:10D98000540EFF1FE48F0100E0057F13C48F0100D8
:10D99000E0057F11A48F0100E0057F10908F01004A
:10D9A000E0057F0A6C8F0100E0057F080023AC488A
:10D9B00000930490042304AA01212046FEF70CFBE7
:10D9C00019E51A462946FFF7DDFB002845D1A54D8C
:10D9D0000090042304AA012120460495FEF7FCFAD6
:10D9E00009E51A462946FFF70BFA48BB9E4DEFE7BB
:10D9F000FEF702FCFFE4FEF71FFDFCE49B481A461D
:10DA00002946F4F753F9074676E71A462946984817
:10DA10000393F3F789FD3278039BA2F16601052990
:10DA200007463FF65DAF1A46924803932946F4F73E
:10DA300063F83278039B074652E702221546CCE68C
:10DA40008D490023009304918DF81400052304AA46
:10DA500001212046FEF7C0FACDE488490023F1E712
:10DA60000222154684E60422154631E5A2F166013C
:10DA700005293FF638AFD6E78148009599E78148F8
:10DA8000FBE78148F9E7294680481A46F5F728FF61
:10DA9000054600283FF4AFAC02B27AE67C48009716
:10DAA00087E729467B481A46F3F770FB05460028AE
:10DAB0003FF4A1AC02B2F6E6294674481A46F5F7DF
:10DAC0004FFF054600283FF496AC02B23CE62946DB
:10DAD00071481A4601F0BEFC0546002800F0FA80A5
:10DAE00002B220E629466D481A46FDF791FE05462A
:10DAF00050B102B2EBE5294668481A46FDF788FEA8
:10DB0000054608B102B2F7E53378002B7FF473AC19
:10DB100004212046FEF794FD6DE429466048DAB200
:10DB2000F9F7E8FD0546002800F0F28002B24FE464
:10DB300029465C48DAB2FCF73BF8054608B102B268
:10DB40005FE53378002B7FF456AC07212046FEF7C3
:10DB500077FD50E4294654481A46F3F7EDF8054698
:10DB600000283FF448AC02B2EFE429464F481A4679
:10DB7000FEF792F80546002800F0B68002B2FBE4FA
:10DB800029464848DAB2FCF713F805460028D8D0F1
:10DB900002B208E5294646481A46FCF71BFF05462F
:10DBA000002800F0AB8002B242E529463D48DAB2D7
:10DBB000FBF7FEFF05460028C3D002B20AE5337822
:10DBC000002B7FF418AC02212046FEF739FD12E449
:10DBD000384852E71A46384803932946F3F7E0FEDF
:10DBE0003278039B07466EE61A463448039329466B
:10DBF000F4F72EF83278039B074674E61A4630484D
:10DC000003932946F3F7A2FF3278039B074670E699
:10DC10001A462C4803932946F3F7D6FF3278039B24
:10DC2000074663E62978012900F0AC8000297FF4DB
:10DC30009DAD254B1B78022B7FF498AD234B1B78B1
:10DC4000002B3FF4D8AB1148F5F7A2FEFFF7D3BB8A
:10DC500029461F481A46F4F7C7FC0546B9E500BF38
:10DC6000E0047004E0047003E00470023C23FF1F32
:10DC7000B022FF1F2023FF1FE0057F02E0057F0386
:10DC8000E0047063E0047060E0047061E464FF1F0E
:10DC9000E00470084C23FF1F90FBFF1F60DEFF1F96
:10DCA0004889FF1F0CA2FF1F4C20FF1FE0E3FF1F4E
:10DCB00088B6FF1FE00470621C23FF1F3823FF1F7C
:10DCC0003023FF1F3423FF1F09A7FF1F0AA7FF1FD1
:10DCD000F83DFF1F3378002B7FF48DAB03212046E6
:10DCE000FEF7AEFCFFF787BB3378002B7FF483ABE6
:10DCF00006212046FEF7A4FCFFF77DBB3378002BFE
:10DD00007FF479AB05212046FEF79AFCFFF773BB41
:10DD10003378002B7FF46FAB0A212046FEF790FC8E
:10DD2000FFF769BB29461F481A46F6F7A1FF0546CB
:10DD300008B102B2A6E53378002B7FF45CAB012179
:10DD40002046FEF77DFCFFF756BB294615481A46CC
:10DD5000F7F712F805460028EDD002B27EE511482B
:10DD6000F7F790F805460028E5D002B262E52946AB
:10DD70000D481A46F5F7E0FC054600283FF41FAFB2
:10DD800002B243E5094A1278022A7FF4EFAC084A4E
:10DD90001278002A7FF42FAB03481946F5F7F8FDF7
:10DDA000FFF729BBA086FF1FE464FF1F09A7FF1F21
:10DDB0000AA7FF1F2DE9F0430446ADF5037D0125B9
:10DDC000C61C00F1040801212046FEF7D3F80746DF
:10DDD000B0B101212046FEF7E9F8B4F80032002B7B
:10DDE00040F08180E02806BF2070C4F80052A4F8FB
:10DDF000023201212046FEF7BDF807460028E8D18F
:10DE00009448FBF7B3F84BF67F339842B4F81222EC
:10DE1000B4F8103288BFC4F8007292B29BB29A4232
:10DE200000F0FA80B4F81222B4F8103292B29BB229
:10DE30009A4280F08C80B4F81092B4F81232A9EBB8
:10DE400003091FFA89F9B9F1000F40F0908003210E
:10DE50002046FEF78FF8B0F1000840F3D480D4F8E4
:10DE60001832434500F0E080B8F1F90F40F3CB8061
:10DE700003AD08EB05070DF583792E4601E04E450D
:10DE80000CD003212046FEF791F8D4F8183206F89A
:10DE9000010B013BBE42C4F81832F0D142AEE02281
:10DEA000A8EB0303327013F0FF034FF08002B2704F
:10DEB00000F0CC800333DAB2032315F8010BF054E1
:10DEC000591CCBB29A42F8D193B20025009501219A
:10DED000727020463246FEF77FF8A4F81C520DF50A
:10DEE000037DBDE8F083012B15D0022B1AD0E0543E
:10DEF0000133B4F802229BB29342A4F800327FF4BB
:10DF000062AFFF2B77D9043BE1789BB242462046B3
:10DF1000FFF7B6F957E702236070A4F80202A4F8ED
:10DF2000003250E7B4F80232A0700322A4F80022B5
:10DF30001BB9FF30A4F8020245E7032B7FF443AF7F
:10DF40000146002332462046FFF79AF93BE7B4F832
:10DF50001232B4F80822B4F8109212FA89F9A9EB37
:10DF600003091FFA89F9B9F1000F3FF470AF0321DB
:10DF70002046FEF70DF8814562DC4FF0000842AE06
:10DF8000474623E0D4F80CC2B4F81252ADB21CF8E4
:10DF900005C084F81472B4F8125286F800C0013536
:10DFA000ADB2A4F81252B4F812C2B4F808521FFA73
:10DFB0008CFCADB2AC4528BFA4F812720097FEF7F6
:10DFC0000BF81FFA88F399457FF641AFB4F810C2F9
:10DFD000B4F8125237701FFA8CFCADB20123AC4575
:10DFE00032464FF0030120469844CBD194F81452A6
:10DFF000002DC7D1E2E7033BA1789BB23246204611
:10E00000FFF73EF9DFE60023C4F81882A4F81C32BB
:10E010000DF5037DBDE8F08394F81432002B3FF436
:10E0200016AFB4F808920EE7B4F81C22632A3FF644
:10E030001FAFF92B3FF71CAF0132A4F81C224EE7AB
:10E040001FFA80F9B9F1000F97D100E703231A46B0
:10E050003BE700BFD096FF1F184B1B78012B29D838
:10E06000174B1B7833B300B591B04FF0E00C102381
:10E070008DF80CC08DF80E30EAB1033201395FFA29
:10E0800082FC032303F1400201336A44DBB211F83E
:10E0900001EF02F834EC6345F4D11FFA8CF300224F
:10E0A0000092012103AA8DF80DC0FDF795FF11B074
:10E0B0005DF804FB704703239C46F0E709A7FF1FA8
:10E0C000540EFF1F184B1B78012B29D8174B1B78B8
:10E0D00033B300B589B04FF0E00C11238DF80CC0BC
:10E0E0008DF80E30EAB1033201395FFA82FC032366
:10E0F00003F1200201336A44DBB211F801EF02F8A8
:10E1000014EC6345F4D11FFA8CF300220092012134
:10E1100003AA8DF80DC0FDF75FFF09B05DF804FBA1
:10E12000704703239C46F0E709A7FF1F540EFF1F0B
:10E130000D4B1B78012B02D80C4B1B7803B9704791
:10E1400000B585B0002312214FF4787C00938DF840
:10E150000E10032303AA0121ADF80CC0FDF73CFF0C
:10E1600005B05DF804FB00BF09A7FF1F540EFF1F99
:10E170000D4B1B78012B02D80C4B1B7803B9704751
:10E1800000B585B0002313214FF4787C00938DF8FF
:10E190000E10032303AA0121ADF80CC0FDF71CFFEC
:10E1A00005B05DF804FB00BF09A7FF1F540EFF1F59
:10E1B00010B51A4C94F800C01CF0FD0F8CB027D19C
:10E1C000174C247824B300294FF0E00414BF1A211F
:10E1D00018218DF808408DF80A10DBB103335FFA7F
:10E1E00083FC013A032303F1300101336944DBB2BC
:10E1F00012F801EF01F828EC6345F4D11FFA8CF313
:10E2000000220092012102AA8DF809C0FDF7E4FE68
:10E210000CB010BD03239C46F2E700BF09A7FF1F07
:10E22000530EFF1F0E4B1B7813F0FD0317D10D4A41
:10E230001278A2B100B5002985B014BF1B211921A5
:10E240004FF4787C00938DF80E10032303AA01216C
:10E25000ADF80CC0FDF7C0FE05B05DF804FB7047DB
:10E2600009A7FF1F530EFF1F194B1B78032B00D06C
:10E270004BBB184B1B7833B300B5A5B04FF0E00C87
:10E2800020238DF80CC08DF80E30EAB1033201392D
:10E290005FFA82FC032303F1900201336A44DBB28C
:10E2A00011F801EF02F884EC6345F4D11FFA8CF306
:10E2B00000220092012103AA8DF80DC0FDF78CFE0B
:10E2C00025B05DF804FB704703239C46F0E700BFD0
:10E2D00009A7FF1F5B0EFF1F0D4B1B78032B00D000
:10E2E00013B90C4B1B7803B9704700B585B00023F8
:10E2F00021214FF4787C00938DF80E10032303AA9C
:10E300000121ADF80CC0FDF767FE05B05DF804FB18
:10E3100009A7FF1F5B0EFF1F194B1B7813F0FB0FA4
:10E3200029D1184B1B7833B300B5A1B04FF0E00CE6
:10E3300030238DF808C08DF80A30EAB10332013974
:10E340005FFA82FC032303F1800201336A44DBB2EB
:10E3500011F801EF02F878EC6345F4D11FFA8CF361
:10E3600000220092012102AA8DF809C0FDF734FEB7
:10E3700021B05DF804FB704703239C46F0E700BF23
:10E3800009A7FF1F590EFF1F194B1B7813F0FB0F36
:10E3900029D1184B1B7833B300B5C3B04FF0E00C54
:10E3A00031238DF80CC08DF80E30EAB103320139FB
:10E3B0005FFA82FC032303F5847201336A44DBB203
:10E3C00011F801EF02F8FCEC6345F4D11FFA8CF36D
:10E3D00000220092012103AA8DF80DC0FDF7FCFD7B
:10E3E00043B05DF804FB704703239C46F0E700BF91
:10E3F00009A7FF1F590EFF1F0D4B1B7813F0FB03DE
:10E4000002D10C4A127802B9704700B585B03221AA
:10E410004FF4787C00938DF80E10032303AA01219A
:10E42000ADF80CC0FDF7D8FD05B05DF804FB00BFEA
:10E4300009A7FF1F590EFF1F194B1B78052B00D092
:10E440004BBB184B1B7833B300B5A5B04FF0E00CB5
:10E4500040238DF80CC08DF80E30EAB1033201393B
:10E460005FFA82FC032303F1900201336A44DBB2BA
:10E4700011F801EF02F884EC6345F4D11FFA8CF334
:10E4800000220092012103AA8DF80DC0FDF7A4FD22
:10E4900025B05DF804FB704703239C46F0E700BFFE
:10E4A00009A7FF1F580EFF1F0D4B1B78052B00D02F
:10E4B00013B90C4B1B7803B9704700B585B0002326
:10E4C00041214FF4787C00938DF80E10032303AAAA
:10E4D0000121ADF80CC0FDF77FFD05B05DF804FB30
:10E4E00009A7FF1F580EFF1F194B1B78072B00D0E1
:10E4F0004BBB184B1B7833B300B5A5B04FF0E00C05
:10E5000045238DF80CC08DF80E30EAB10332013985
:10E510005FFA82FC032303F1900201336A44DBB209
:10E5200011F801EF02F884EC6345F4D11FFA8CF383
:10E5300000220092012103AA8DF80DC0FDF74CFDC9
:10E5400025B05DF804FB704703239C46F0E700BF4D
:10E5500009A7FF1F570EFF1F194B1B78072B00D071
:10E560004BBB184B1B7833B300B5A5B04FF0E00C94
:10E5700046238DF80CC08DF80E30EAB10332013914
:10E580005FFA82FC032303F1900201336A44DBB299
:10E5900011F801EF02F884EC6345F4D11FFA8CF313
:10E5A00000220092012103AA8DF80DC0FDF714FD91
:10E5B00025B05DF804FB704703239C46F0E700BFDD
:10E5C00009A7FF1F570EFF1F0D4B1B78072B00D00D
:10E5D00013B90C4B1B7803B9704700B585B0002305
:10E5E00049214FF4787C00938DF80E10032303AA81
:10E5F0000121ADF80CC0FDF7EFFC05B05DF804FBA0
:10E6000009A7FF1F570EFF1F0D4B1B78072B00D0CC
:10E6100013B90C4B1B7803B9704700B585B00023C4
:10E6200048214FF4787C00938DF80E10032303AA41
:10E630000121ADF80CC0FDF7CFFC05B05DF804FB7F
:10E6400009A7FF1F570EFF1F70B5204B1B780A2B21
:10E65000ADF5027D0446164600D0DBB91C4B1B7895
:10E66000C3B1E023FC2E8DF8083016D8F51C6523C5
:10E670008DF809508DF80A3026B132460DF10B00A5
:10E6800001F09EF80023009302AAABB201212046BC
:10E69000FDF7A2FC0DF5027D70BD731D002532460D
:10E6A0008DF80A3003A865238DF80B308DF80950DA
:10E6B00001F086F8331D00959BB202AA0121204685
:10E6C000FDF78AFC0DF5027D70BD00BF09A7FF1F95
:10E6D000560EFF1F0F4B1B780A2B8C4600D013B928
:10E6E0000D4B1B7803B9704700B587B000234FF47A
:10E6F0009C6166220093ADF80C108DF80E20042367
:10E7000003AA01218DF80FC0FDF766FC07B05DF884
:10E7100004FB00BF09A7FF1F560EFF1F0D4B1B7800
:10E720000A2B00D013B90C4B1B7803B9704700B506
:10E7300087B0002367214FF4787C00938DF80E108A
:10E74000032303AA0121ADF80CC0FDF745FC07B077
:10E750005DF804FB09A7FF1F560EFF1F70B5204B85
:10E760001B780A2BADF5027D0446164600D0DBB9B6
:10E770001C4B1B78C3B1E023FC2E8DF8083016D853
:10E78000F51C55238DF809508DF80A3026B1324614
:10E790000DF10B0001F014F80023009302AAABB2B4
:10E7A00001212046FDF718FC0DF5027D70BD731D9B
:10E7B000002532468DF80A3003A855238DF80B301A
:10E7C0008DF8095000F0FCFF331D00959BB202AAA2
:10E7D00001212046FDF700FC0DF5027D70BD00BF54
:10E7E00009A7FF1F520EFF1F174B1B78632B26D163
:10E7F00000B5A5B04FF0E00C08238DF80CC08DF8E3
:10E800000E30EAB1033201395FFA82FC032303F1CF
:10E81000900201336A44DBB211F801EF02F884EC94
:10E820006345F4D11FFA8CF300220092012103AA60
:10E830008DF80DC0FDF7D0FB25B05DF804FB7047E7
:10E8400003239C46F0E700BF09A7FF1F174B1B7867
:10E85000602B26D100B58BB04FF0E00C09238DF86A
:10E8600008C08DF80A30EAB1033201395FFA82FC40
:10E87000032303F1280201336A44DBB211F801EFEC
:10E8800002F820EC6345F4D11FFA8CF300220092C9
:10E89000012102AA8DF809C0FDF79EFB0BB05DF8BF
:10E8A00004FB704703239C46F0E700BF09A7FF1F46
:10E8B00090F804323BB300B5A5B00A784FF0E00CF5
:10E8C000F1238DF80CC08DF80E30EAB14FF0030C37
:10E8D000ACF102030CF1900EEE44DBB20EF8842C86
:10E8E000CA5C0CF1010C5FFA8CFC002AF0D11FFA13
:10E8F0008CF30121009103AA8DF80DC0FDF76CFB8C
:10E9000025B05DF804FB704703239C46F1E700BF88
:10E9100090F804320BB1FDF7F9BB70472DE9F041D7
:10E9200090F80442A4B0002C4BD01E460C78E02393
:10E930008DF80C30F3238DF80E30002C44D04FF0BE
:10E94000030CACF1020E0CF190030DEB03055FFA22
:10E950008EFE05F8844C11F80E400CF1010E654650
:10E960005FFA8EFC002CECD16B1D05F1020EE91C48
:10E97000DCB204355FFA8EFEC9B2EDB223460CF16B
:10E9800090070DEB070C90310EF190070DEB070E81
:10E990000DEB010705F190010DEB0105C2F307280E
:10E9A000012100910CF8848C0EF8842CC6F3072208
:10E9B00007F8842C05F8846C03AA8DF80D40FDF748
:10E9C0000BFB24B0BDE8F08107231C46062505217A
:10E9D0004FF0040E4FF0030CD1E700BF2DE9F04FCC
:10E9E0001D46A5B090F80432BDF9B860002B61D087
:10E9F000E0230C788DF80C30F4238DF80E30002CC9
:10EA00005BD04FF0030CACF1020E0CF190036B44A1
:10EA10005FFA8EFE03F8844C11F80E400CF1010EE3
:10EA200063465FFA8EFC002CEDD1D91D03F1020A7A
:10EA300003F103091F1D03F1050E9C1D5FFA81F808
:10EA40005FFA8AFA5FFA89F9FFB25FFA8EFEE4B2E2
:10EA500043460CF190010DEB010C0AF190010DEB16
:10EA6000010A09F190010DEB010907F190010DEB8D
:10EA700001070EF190010DEB010E04F190010DEB79
:10EA80000104C2F3072B012100910CF884BC0AF8A1
:10EA9000842CC5F3072209F8842CC6F3072207F853
:10EAA000845C0EF8842C04F8846C03AA8DF80D8025
:10EAB000FDF792FA25B0BDE8F08F092398460824A7
:10EAC0004FF0070E06274FF005094FF0040A4FF0EC
:10EAD000030CBEE72DE9F04F9E46A9B090F8043232
:10EAE000BDF9C8A0BDF9CC90002B7AD0E0230C78FA
:10EAF0008DF81C30F5238DF81E30002C74D04FF0AB
:10EB0000030BABF102030BF1A005DBB26D44DC4655
:10EB100005F8844CCC5C0BF101035FFA83FB002CFD
:10EB2000EFD10CF102010CF10903C9B20CF1030899
:10EB30000CF104070CF105060CF106050CF10704B5
:10EB400003910CF1080CD9B25FFA88F8FFB2F6B263
:10EB5000EDB2E4B25FFA8CFC05910B460BF1A0011B
:10EB60000DEB010B0399A0316944039108F1A00159
:10EB70000DEB010807F1A0010DEB010706F1A00163
:10EB80000DEB010605F1A0010DEB010504F1A0015B
:10EB90000DEB01040CF1A00104940DEB010CC2F388
:10EBA0000724012100910BF8844C039C04F8842C69
:10EBB000CEF3072208F8842C049C07F884ECCAF3EF
:10EBC000072206F8842CC9F3072205F884AC04F860
:10EBD000842C059C0CF8849C07AA8DF81D40FDF739
:10EBE000FBF929B0BDE8F08F0B23042105934FF00A
:10EBF0000A0C09240825072606274FF0050803916B
:10EC00004FF0030BAAE700BF014B185C704700BF31
:10EC1000E8910100094AC3B2C0F3072CC0F30741D1
:10EC2000D35C12F80CC0515C000E125C03EB0C00BC
:10EC300051FA80F052FA80F0C0B27047E8910100BA
:10EC4000154AC3B2C0F3072CD35C12F80CC063445E
:10EC5000C0F3074C000E00B512F80CE012F800C02B
:10EC60005EFA83F05CFA80F05FFA81FCC1F307235F
:10EC700012F80CC0D35C5CFA80F053FA80F0C1F358
:10EC80000743090E12F803C0535C5CFA80F053FA94
:10EC900080F0C0B25DF804FBE891010070B500247B
:10ECA0000646214600F8044B142206F5805505F06F
:10ECB0004FF821464FF4965206F1180005F048F837
:10ECC000154BC5F8DC3242F20F7206F59750C5F8C5
:10ECD000E032A5F8E4222146C5F8D8422022C5F842
:10ECE000E842A5F8EC4285F8EE42103005F030F825
:10ECF00006F59850A5F8104320222146123005F061
:10ED000027F8632385F83433A5F83243C5F8384330
:10ED1000A5F83C43304670BD0F270F2700F5805300
:10ED2000002202700E49C3F8E8224FF0630C42F251
:10ED30000F7083F834C3C3F8D822C3F8DC12C3F8C9
:10ED4000E012A3F8E402A3F81023A3F83223A3F8F7
:10ED5000EC2283F8EE22C3F83823A3F83C23704753
:10ED60000F270F2770B5044682B0002A00F082807A
:10ED7000424E4FF47A5E00207546B44614E09C453E
:10ED8000B8BF9C469D42A8BF1D464B1D9BB2B3F524
:10ED9000166F00F10100A1F65B1138BF194683B26E
:10EDA00028BF89B29A420CD901F10C0334F913300F
:10EDB000002BE4DC9E45A8BF9E469E42B8BF1E467F
:10EDC000E3E70EEB06030CEB05025B1003EB6206B8
:10EDD0005510A5EB660542F34F021BB246F34F06F2
:10EDE0002DB22749274801950096FFF773FE04F5D9
:10EDF000805E9EF83433632B2CD004EB430202F583
:10EE000080520133DBB2A2F8F062A2F812530F2B4A
:10EE10008EF8343304F5975304F5985403F10E0338
:10EE200004F10E0422D800210A46AEF81013AEF801
:10EE3000321333F802CF588C614402449C4209B229
:10EE400012B2F6D109111211AEF81013AEF8322336
:10EE500002B070BD04F597530E3304F598540E3488
:10EE60001A4622F8026F94425584FAD100228EF895
:10EE70003423D8E7154616461346B2E780C1FFFF94
:10EE8000E892010020E6FF1F2DE9F047BDF8204081
:10EE9000BDF92470BDF92890002A00F08880023462
:10EEA000444EBFB2A4B2C9F1000800252DE04FEADC
:10EEB000DC0E0CF0070C16F80CA013F80EC02CEAB0
:10EEC0000A0C03F80EC004F1FF3CCCF3CC0E0CF09E
:10EED000070C13F80EA016F80CC04CEA0A0C03F845
:10EEE0000EC001F1050C1FFA8CFCBCF5166F05F184
:10EEF00001052CBFA1F65B1161461FFA85FC28BFF6
:10EF000089B202346245A4B251D901F10C0EA4F1C8
:10EF1000020C30F81EE0AEEB070E0FFA8EFEC6456F
:10EF20001FFA8CFCC3DBBEF1000F1CDBCE454FEAA1
:10EF3000DC0E0CF0070C13F80EA016F80CC04CEA0F
:10EF40000A0C03F80EC004F1FF3CCCF3CC0E0CF01D
:10EF5000070C23DA16F80CA013F80EC02CEA0A0CE2
:10EF600003F80EC0BDE74FEADC0E0CF0070C16F8F4
:10EF70000CA013F80EC02CEA0A0C03F80EC004F122
:10EF8000FF3CCCF3CC0E0CF0070C16F80CA013F8D9
:10EF90000EC02CEA0A0C03F80EC0A2E713F80EA06C
:10EFA00016F80CC04CEA0A0C03F80EC099E7BDE84D
:10EFB000F08700BF549301002DE9F04F00F5805613
:10EFC000534AB6F8DA32534903F60115ADB2B5F536
:10EFD000166F24BF5F3B9DB287B002F1130EA946A6
:10EFE0006FF0020A00244FF47A5C4FF6FD78032795
:10EFF00012E0BAF1FF3F24D013FB074409F10503E7
:10F000009BB2B3F5166F24BFA9F65B139BB296456E
:10F0100019D012F901AF994609F10C0330F91330F8
:10F020009942B8BF19469C45A8BF9C46BAF1010F4A
:10F0300005D0BAF1030FDCD113FB0844DEE7E41A74
:10F04000DCE71C44DAE7D6F8E832A3422DDA96F87A
:10F050003433632B4AD0B6F91023B6F93233029316
:10F060000023019200939846142204AB2946FFF72F
:10F070000BFF1F460378DFF8A09043450CBF4FF00D
:10F08000020B4FF0040B0DF1150AD42017F8013BC9
:10F090005840FFF7B9FD574540445FFA80F802D069
:10F0A00019F8010FF2E7D84503D9002007B0BDE8F1
:10F0B000F08FB6F8DA32A6F8E03203F6FB0292B22D
:10F0C000B2F5166F4FF0050128BF653B4FF0010008
:10F0D000C6F8E842A6F8EC12A6F8DC5234BFA6F84F
:10F0E000DE22A6F8DE3207B0BDE8F08F0CEB01029D
:10F0F000A1EB620344F63E1101FB03F342F34F021E
:10F1000043F3CF33A6F81023A6F83233A7E700BFA6
:10F110006493010080C1FFFF5C93010038B500F5E6
:10F1200080550446B5F8D832264804EB83035B6863
:10F13000C3F313035840FFF76DFD032829D8204679
:10F14000FFF73AFF28B395F8EE323BB3013BDBB251
:10F15000012B85F8EE321BD1B5F8E03203F65F12D1
:10F1600092B2B2F5166F28BF03F1FF32A5F8E22282
:10F170005A1C92B2B2F5166F2ABFA3F65F13A5F818
:10F18000E422A5F8E43201220023227085F8EE3251
:10F1900038BD95F8EE32002BD8D138BDC5F83833DC
:10F1A000A5F83C3308480121F9F7B6FA06480121D1
:10F1B000F9F7BEFA6322042385F8342385F8EE328A
:10F1C00038BD00BFADB50700D096FF1F70B500F584
:10F1D0008054A4B0B4F8E222B4F8E412B4F8DA32FD
:10F1E0008A42054607D29A4207D9B4F8DE229A42EB
:10F1F0001BD024B070BD9A4201D99942F5D3B4F81E
:10F20000D8324D4805EB83035B68C3F313035840C2
:10F21000FFF700FD032802D82846FFF7CDFEB4F81B
:10F22000DA32B4F8DE229A42E3D1B4F8EC32052B9C
:10F2300016D1B4F8E03203F65F1292B2B2F5166F4F
:10F2400028BF03F1FF32A4F8E2225A1C92B2B2F5B1
:10F25000166F2ABFA3F65F13A4F8E422A4F8E432E1
:10F26000B4F8DC124FF4F0722846FFF77BFDB4F9D6
:10F270003213B4F91033B4F9E02230480091304928
:10F28000FFF7ACFBB4F91033B4F932230193082330
:10F2900002920093B4F8DC1205AB4FF4F0722846EA
:10F2A000FFF7F2FDB4F8EC62013EB6B2A4F8EC62EE
:10F2B00046B3A6F10406B6FA86F6B4F83C337609EE
:10F2C0008DF8146073B91D48792205A9FEF7CCFFAB
:10F2D0000023C4F83833A4F83C330023C4F8E832E0
:10F2E00024B070BDD4F83823B2FBF3F3C3F3072185
:10F2F0008DF88D1011488DF88E307B2205A9FEF710
:10F30000B3FFE5E70D480F49FFF7D2FA0E48314643
:10F31000F9F702FA0C483146F9F70AFA0748FEF7FE
:10F32000DBFF42F20F7263232E70A4F8DE2284F812
:10F33000343384F8EE62D0E7ADB5070020E6FF1F56
:10F340000893010030930100D096FF1F002B4CD092
:10F350002DE9F04100F580545E1EF6B20546B4F882
:10F36000D832B4F8DA02A2F1020801EB46068F1E89
:10F3700016E0FFF7D3FEB4F8DA02B4F8D832013061
:10F3800080B201339BB2B0F5166F28BF0020052B69
:10F3900028BF0023BE42A4F8DA02A4F8D83222D053
:10F3A00038F8021FD4F83823B4F83CC305EB8303C4
:10F3B0000A440CF1010C37F9021FC4F83823A4F8F1
:10F3C0003CC35A6800294FEA4202B8BF42F001022A
:10F3D0005A602B780C30012B25F810102846C8D124
:10F3E000FFF7F4FEC7E7BDE8F081704770B504464B
:10F3F00000254FF47A60258120806581657325732F
:10F4000002F062FC294660604FF4966204F13C0011
:10F4100004F09EFC04F11C064FF49653F022A4F86D
:10F42000F024C4F8F434C4F8EC5484F8F254C4F86A
:10F43000F85420222946304604F08AFC034A044B43
:10F4400022616361A661204670BD00BF050009000E
:10F45000D80FFF1F792A01D0042070474289038901
:10F4600092B29BB29A4230B544D04289038992B29B
:10F470009BB29A4208D34389048902881B1B9BB222
:10F480009A420AD2052030BD04890288438912FAC3
:10F4900083F31B1B9BB29A42F4D3772BF2D901F171
:10F4A000780C4FF0010E18E0456803899BB2EA54CE
:10F4B000038901339BB203810289038892B29BB214
:10F4C0009A4228BF04810289438992B29BB29A4230
:10F4D00008BF80F80CE061450AD0037B11F8012FCA
:10F4E00003F0FF04002BDFD0614580F80DE0F4D17C
:10F4F000002030BD037B002BC4D10388CDE700BFC3
:10F500002DE9F04390F8F224DFF89C90DFF89C801E
:10F51000224F234E8FB00DF1080C04AC40F277253A
:10F5200040F2657E01F0C003802B2ED0C02B24D08A
:10F53000E3B1002A14BF4B464346ACF800300CF14F
:10F54000020C89006445C9B2ECD1224602A9042309
:10F55000103002F0BFFD002300931248142322460E
:10F560000321F8F7EFFF0FB0BDE8F083002A14BFC6
:10F570003B463346ACF80030E1E7002A14BF4FF4B5
:10F580006D737346ACF80030D9E7002A14BF4FF40E
:10F590009E732B46ACF80030D1E700BFC4FEFFFFDE
:10F5A00089FDFFFFD096FF1F4CFCFFFF9BF8FFFF7C
:10F5B000F0B5B0F8EC248FB0044612B35848594E59
:10F5C000F9F782F8054617E0B4F8EE345A1C2344E4
:10F5D000A4F8EE2493F83C10FFF792FF3378143D23
:10F5E000ADB21BB1D4F8F434C4F8F834B4F8EE2456
:10F5F000B4F8EC349A4275D2142D2046E4D80FB0FA
:10F60000F0BD4189038989B29BB299426FD041898B
:10F61000038989B29BB2994232D2038941895B1A2C
:10F620009BB2002B35D0404B1B78002B64D00020C0
:10F630001AE0616863899BB211F803C02073638983
:10F6400001339BB263816189238889B29BB299425D
:10F6500028BF6081531C9BB22244782BA4F8EC3461
:10F6600082F83CC055D01A462189638989B29BB281
:10F670009942DED1237B03F0FF0C002BD9D1E9E7BF
:10F6800041890088238910FA83F35B1A9BB2002B0F
:10F69000C9D1D4F8F834002BB1D02148204FF9F764
:10F6A00013F80026054613E0CDE9026602F012FDCC
:10F6B0001423009604AA03213846F8F743FFD4F830
:10F6C000F834143D013BADB2C4F8F834002B96D0A9
:10F6D000142D4FF0040304AA02A904F11000E3D88A
:10F6E0000FB0F0BD0023C4F8EC340FB0F0BD037BC5
:10F6F000002BCED0038894E7B4F8F01469B17720DA
:10F70000A318013292B28A4283F83C00F8D1A4F8DF
:10F71000EC240023A4F8EE3450E7A4F8EE14B8E784
:10F72000D096FF1F550EFF1F0AA7FF1F01EB4101D7
:10F73000890001F51671B1F5966F28BF4FF49661F7
:10F74000A0F8F014704700BF4289038992B29BB2BF
:10F750009A421DD04289038992B29BB29A4208D341
:10F76000438901890288581A80B282420AD2002055
:10F77000704702880389408912FA80F0C01A80B26B
:10F780008242F4D3084BA3FB0030C0F387107047CC
:10F79000037B002BEBD10088A3F17733A3FB003070
:10F7A000C0F38710704700BF898888884FF496633C
:10F7B00003FB02F280F8F214C0F8F424704700BF93
:10F7C00001B441EA000313F003036FD1403A41D37F
:10F7D00051F8043B40F8043B51F8043B40F8043B2B
:10F7E00051F8043B40F8043B51F8043B40F8043B1B
:10F7F00051F8043B40F8043B51F8043B40F8043B0B
:10F8000051F8043B40F8043B51F8043B40F8043BFA
:10F8100051F8043B40F8043B51F8043B40F8043BEA
:10F8200051F8043B40F8043B51F8043B40F8043BDA
:10F8300051F8043B40F8043B51F8043B40F8043BCA
:10F8400051F8043B40F8043B51F8043B40F8043BBA
:10F85000403ABDD2303211D351F8043B40F8043B5A
:10F8600051F8043B40F8043B51F8043B40F8043B9A
:10F8700051F8043B40F8043B103AEDD20C3205D36A
:10F8800051F8043B40F8043B043AF9D204320AD060
:10F89000D2071CBF11F8013B00F8013B03D30B78E2
:10F8A00003704B78437001BC704700BF0C2A4AD3E9
:10F8B00010F0030311D0C3F10403D21ADB071CBFFD
:10F8C00011F8013B00F8013B07D311F8013B00F8A8
:10F8D000013B11F8013B00F8013B11F003033FF439
:10F8E00075AF30B4043AC91AC3F1040C51F8044B93
:10F8F000022B19D0032B0BD0240A51F8043B1D0610
:10F9000044EA050440F8044B1C46043AF4D216E0DD
:10F91000240E51F8043B1D0244EA050440F8044B50
:10F920001C46043AF4D20AE0240C51F8043B1D04AE
:10F9300044EA050440F8044B1C46043AF4D204326D
:10F94000B1EB0C0130BC043AA0D3013A11F8013BF1
:10F9500000F8013BF9D20B7803704B7843708B7839
:10F96000837001BC704700BF08B50F4C636B580330
:10F970000DD4636B59050FD4636B1A0511D4636BF7
:10F98000DB04F3D501F0FEF8636B5803F1D501F009
:10F9900075FA636B5905EFD500F008F8636B1A052B
:10F9A000EDD500F04BFDEAE70080044008B5FFF715
:10F9B000DBFF00BF014B10221A807047002005407A
:10F9C000704700BF0B490A6848B108B5EC461318E8
:10F9D000ACF50050834204D20B60104608BD1046BF
:10F9E000704704F019FA0C234FF0FF320360104601
:10F9F00008BD00BF3410FF1FEFF31383CBB9EFF343
:10FA00001080A0B9EFF3058343B94FF48070EFF392
:10FA100011835BB1984228BF184670470F2BF6D967
:10FA2000054AD05CEFF31183002BF3D170471846E1
:10FA300070474FF0FF307047F0E300E0034B0022C7
:10FA400010215A615A6018605961704700D0034014
:10FA5000704700BF4FF0E02CF0B54FF0006ECCF8CF
:10FA600004E14FF0805ECCF804E14FF0005ECCF88A
:10FA700004E1244A24492548254C4FF0804ECCF817
:10FA800004E1282300274EF6FF7609254FF0004EAB
:10FA9000CCF804E183B04F608E60CB604B61CB61EA
:10FAA0004B62CB624B63CB634B64D3605361D361D6
:10FAB0005362D3625363D36353640D606760A6607F
:10FAC000E3606361256047608660C36043610560F1
:10FAD00057609660D3605361156002F075F9FFF7C7
:10FAE000B7FF0C4C23680093009B132BFAD901F04D
:10FAF0007FFD23680193019BB3F5967FF9D303B093
:10FB0000F0BD00BF00900B400080034000800B4020
:10FB1000009003408C0000203F2818D810B4124BEE
:10FB200053F8302092F8804234B1012381B982F831
:10FB300000315DF8044B704703EBC0035B681A6843
:10FB400059B142F003025DF8044B1A6070477047E8
:10FB500082F880305DF8044B704722F002025DF8B5
:10FB6000044B1A60704700BF789301003F2806D805
:10FB7000044B53F8303093F80002C0B270470020B5
:10FB8000704700BF789301003F2820D81B4A02EB42
:10FB9000C00301295B680FD004291DD052F8300042
:10FBA000002280F8802299B1022922D003290DD1A8
:10FBB0004FF481721A60704752F830004FF4A2720D
:10FBC00080F880121A601A6822F020021A607047CA
:10FBD0004FF480721A60704752F830104FF4A272DE
:10FBE000012081F880021A601A6842F020021A602F
:10FBF000704740F203121A60704700BF789301000B
:10FC00002DE9F843044672B6204F4FF0E022936985
:10FC10003D68D2F8042D62B6520102D5322B88BF5E
:10FC200001350CB9BDE8F883DFF86490DFF8648033
:10FC3000A9EB0303A8FB03234FF47A7202FB05F53B
:10FC400005EB93154FF0E02672B6B1693A68D6F825
:10FC500004CD62B6A9EB0103A8FB03031CF0806F7F
:10FC6000C5EB93134FF47A7002D0322988BF01326A
:10FC700000FB0233B3F57A7F04D3013CD2D005F503
:10FC80007A75E1E702F028F8DEE700BF8C0000207B
:10FC9000BFD4010089888888294A2A49536B70B4E7
:10FCA00043F40063284D5363284E294C32780023D7
:10FCB0002B700B70274923700B702749092A0B7092
:10FCC00031D03B2A03D1254B40F213325A60244BEA
:10FCD0001B780A2B2FD03A2B03D1204B4FF45172B3
:10FCE0001A6020281F4B38BF2020C0F344341C70FA
:10FCF000C0F3471400F01F005C70042198721A4C86
:10FD0000997002224FF0880C3C20DA74597583F800
:10FD100010C04FF0E021D870402384F8213070BC2F
:10FD2000C1F804217047114B40F21332DA600C4BDA
:10FD30001B780A2BCFD10D4B4FF451721A61D0E7CB
:10FD400000800440DC000020D40000204410FF1F8D
:10FD50001001002018010020E400002000D0044021
:10FD60004C10FF1F00B0064000E400E000B004406B
:10FD7000294B9B7800F0030203F0EC031343410787
:10FD800000F00F02244948BF43F01003042A8B708F
:10FD900003D18B7943F040038B711F4B5B79C20613
:10FDA00003F0EF031C4A48BF43F0100353719379EB
:10FDB000194A03F0EF0310F0200C18BF43F01003B2
:10FDC0009371C30506D553781178DBB241F0200159
:10FDD0001170537010F4007017D00F490F488B78D2
:10FDE0000F4A43F0A0038B7003780E4902EBC30265
:10FDF00040F24633506840F24732BCF1000F08BF72
:10FE00001346094A03600A607047064B064A1968A0
:10FE1000914208BF1860704700B006404C10FF1FA9
:10FE200078930100E0000020D400D642274B5B6BA2
:10FE30001B0549D510B5264C237823B101F04CFFA2
:10FE40002378002BFAD12349234B4FF0E0200224E2
:10FE50000022C0F88441CA701B78092B29D03B2BA3
:10FE60001AD01E4B1B7803F07F030A2B1CD03A2BB1
:10FE70000ED01B4B174A1B4C1B48196892F804C044
:10FE8000D27900232370037009B101230B7010BDD8
:10FE9000164B00221A60ECE7144B5A600F4B1B788C
:10FEA00003F07F030A2BE2D1114B40F203121A61D7
:10FEB000DFE70F4B40F20312DA60084B1B7803F0C8
:10FEC0007F030A2BD3D1EFE7704700BF00800440C7
:10FED000E400002000B006404410FF1F4C10FF1F3C
:10FEE00090000020D4000020DC00002000D004405E
:10FEF00000B004400A4A38B50546137803F0FF0401
:10FF0000002BFAD101212846FFF73EFE2146284664
:10FF1000FFF702FE034A044B52F835201A6038BD41
:10FF2000E400002078930100E000002009B140F0D7
:10FF300080001B4A1378834218D010B4194C646BAC
:10FF400024050FD503F07F030A2B24D03A2B16D0BB
:10FF5000002900F07F0314BF602144210A2B12D036
:10FF60003A2B04D010705DF8044B704770470E4B6D
:10FF700041F44071196010705DF8044B70470A4BF2
:10FF800000241C60E4E7094B41F4407119611070D2
:10FF90005DF8044B7047054B00241C61D8E700BF97
:10FFA0004C10FF1F0080044000D0044000B004400B
:10FFB000124B1A7882420CD01149496B090507D5BA
:10FFC000092A16D03B2A0AD009280DD03B2801D097
:10FFD000187070470B4A40F213315160F8E7094A34
:10FFE000002109285160F1D1074A40F21331D16054
:10FFF000EEE7054A0021D160E6E700BF4410FF1F8D
:020000021000EC
:100000000080044000D0044000B004400D4B5B6B06
:1000100013F4006313D03F2803D90B4B0020186062
:1000200070470A4B10B5084C53F83030236001215B
:10003000FFF7AAFD236800221A70012010BD1846A0
:10004000704700BF008004409000002078930100BA
:10005000104B5B6B13F4006312D017280BD03C28B5
:1000600010D10D4B40F202329A600C4A537B0120B2
:100070000343537370470A4B40F202329A60F4E72D
:1000800018467047054A537B03F0FE030020537364
:10009000704700BF0080044000D0044000B006401C
:1000A00000B004402DE9F84F334B5B6B1A053AD58D
:1000B000324B1B6806460BB101221A70DFF8D49050
:1000C000DFF8D48099F80040D8F800302C4D013486
:1000D000A3422B7829D99C425FFA84FA14D1294F84
:1000E000DFF8ACB005E03B791B0623D42B78A342A4
:1000F0000AD1FFF781FC4028F5DDFF28F6DD01F08D
:10010000EBFD2B78A342F4D0272C29D91E4B283C99
:100110001B68F6B21E551D4A1A4B01211170BC22F4
:1001200089F800A0DA70BDE8F88F03F0FF0AA3B9E0
:100130005446D4E72B78D8F800105A1C9142DBB211
:1001400008D9272A10D8D1B21BF80230DBB2FB71D4
:100150002970CBE700210A46F6E74FF0000A544623
:100160000B4BF6B21E55D6E7D1B2074A273B1268B1
:10017000D35CDBB2EBE700BF00800440E00000206E
:100180001801002000B0064014010020E400002007
:10019000E8000020100100204810FF1F2DE9F84F53
:1001A000394B5B6B1A053CD5384B1B680BB10122F0
:1001B0001A704718B84231D2354EDFF8EC80354C12
:1001C000DFF8E09000F1010A13E003F0FF0B53B3F6
:1001D0004FF0000B5D46304A1AF8013C5355524629
:1001E0002E490123BA420B700AF1010A86F800B0C9
:1001F00014D23578D8F800300135AB422378E4D9F1
:10020000AB425FFA85FB0FD0272DE4D9244B1AF8B7
:10021000012C1B68283D5A555246E1E7214BBC2270
:10022000DA70BDE8F88F5D466FF0430389F803305C
:1002300006E099F804301B060BD42378AB42E3D1D7
:10024000FFF7DAFB4028F4DDFF28F6DD01F044FD7E
:10025000F3E72378D8F800105A1C9142DBB203D997
:10026000272A0AD8D1B201E000210A460A4B9B5C3A
:10027000DBB289F807302170DFE7D1B2084A273BAB
:100280001268D35CDBB2F4E700800440E000002099
:100290001001002018010020E8000020E4000020E8
:1002A0001401002000B006404810FF1F10B5044C98
:1002B000237823B101F010FD2378002BFAD110BD73
:1002C000E4000020084A094B11781A789142C8B21C
:1002D000D3B202D2013B181A7047054A1268013A9C
:1002E0001344181A704700BF1001002018010020A5
:1002F0004810FF1F064A074B11781A789142D0B276
:100300003CBF054A1268CBB238BF9B18181A704719
:10031000D4000020DC0000204010FF1F1B4B1C49B4
:100320001A780B789A422ED010B55FFA82FE194ADD
:10033000D8B21268431C9A4219D93F2B1BD85FFAD6
:1003400083FC1548C05CC0B281F800C0134909683D
:1003500061B19E453CBF7244D31A114A126828BF4E
:10036000AEEB03039A4201D300230B7010BD4FF094
:10037000000C6346E5E70B4C3F382468205C5FFACD
:1003800083FCC0B2E0E74FF0FF307047D40000209C
:10039000DC0000204010FF1F94000020900000208F
:1003A0003C10FF1FD80000200D4A0E4B11781B781F
:1003B0009942DAB211D00C490968531C994207D905
:1003C0003F2B06D9094B3F3A1B68985CC0B2704777
:1003D0000023074AD05CC0B270474FF0FF3070472F
:1003E000D4000020DC0000204010FF1FD8000020B7
:1003F000940000200C4B5B6B1B0514D50B4B0C4879
:10040000DA78402102F0CB02DA705974DA780949BF
:1004100042F03402DA70084A03781268DBB20B70DB
:100420000AB10023137070470080044000B00640FA
:10043000DC000020D4000020900000202DE9F041D5
:10044000504C237913F0300F47D072B6A37D03F0E0
:10045000FF01002B58D062B6DFF85C814A4898F85B
:1004600000304A4A05781668494F5FFA83FC494BC9
:10047000EDB2D3F800E008E01DB14FF0000C07F832
:100480000C304A1E12F0FF0112D0E3790CF1010288
:100490009642DBB2F0D99542ACF13F00F1D03F2A51
:1004A0006DD994464A1E12F0FF010EF80030ECD1CF
:1004B0005FFA8CF388F80030374B196869B1AC45A6
:1004C0003CBF721B02EB0C03344A126828BFACEB32
:1004D00005039A429CBF01230B702A48C3781E066D
:1004E000DDB216D46A060DD5264B1B795B0609D5FD
:1004F0002B4B2C491B6800220A7003B11A70214B48
:100500003C22DA70BDE8F0814023E279637462B680
:10051000E3E703791C06E5D5234B244ADFF89CE08A
:100520001C7816689EF80030214A224FD2F800C08D
:10053000E4B2DBB207E003790023FA5CD2B2C27105
:10054000027D072A11D8A34203F101010ED08E4289
:10055000F1D927290279A3F1270301D80B46ECE74B
:100560001CF803200B46D2B2E9E7DCB2054B8EF84B
:1005700000401A79110644BF7C22DA70B2E7944633
:100580007DE700BF00B00640DC0000204010FF1FE8
:1005900094000020D8000020900000203810FF1F99
:1005A000E0000020E4000020100100204810FF1FA0
:1005B00014010020E8000020D400002018010020D1
:1005C000094B10B4186068B101F14004074B0848AA
:1005D00001F11A021A60074B046028315DF8044BE0
:1005E000196070474024F1E7D80000203C10FF1F3D
:1005F0004010FF1F3810FF1F054B186018B1054B46
:10060000283119607047034B28211960704700BFDB
:10061000140100204810FF1F2DE9F84F314B1B68D3
:1006200007460BB101221A70DFF8D090DFF8D080B6
:1006300099F80040D8F800302B4D01349C422B78BB
:100640002AD303F0FF0A002B3ED15446274EDFF891
:10065000A8B005E033791B0623D42B78A3420AD136
:10066000FFF7CAF94028F5DDFF28F6DD01F034FB7D
:100670002B78A342F4D0272C29D91D4B283C1B688A
:10068000FFB21F551B4A194B01211170AC2289F88A
:1006900000A0DA70BDE8F88F9C425FFA84FAD5D0EA
:1006A000E9E72B78D8F800105A1C8A42DBB203D253
:1006B000272A10D8D1B201E000210A461BF80230E7
:1006C000DBB2F3712970C8E74FF0000A54460A4BB9
:1006D000FFB21F55D6E7D1B2054A273B1268D35C5B
:1006E000DBB2EEE76C010020A401002000C0064050
:1006F000A001002070010020740100209C01002056
:100700005C10FF1F1D4A1E49536B2DE9F04343F453
:1007100080531C4DDFF87C80DFF87C901A4F1B4E15
:100720005363002388F80030202889F800303B709C
:1007300033702B7040F213358D6002F5103238BFE4
:1007400020204FF45175CD60C0F344311170C0F3D7
:10075000471E0F4C82F801E000F01F002C21907220
:100760004FF0E02C93701374D1704022082384F86A
:100770002320CCF80431BDE8F08300BF00800440A2
:1007800000C00440700100209C010020A401002052
:1007900000E400E06001002068010020294B9B7804
:1007A00000F0030203F0EC031343410700F00F02D3
:1007B000244948BF43F01003042A8B7003D18B797E
:1007C00043F040038B711F4B5B79C20603F0EF03CC
:1007D0001C4A48BF43F0100353719379194A03F040
:1007E000EF0310F0200C18BF43F010039371C30502
:1007F00006D553781178DBB241F0200111705370A7
:1008000010F4007017D00F490F488B780F4A43F04F
:10081000A0038B7003780E4902EBC30240F246330B
:10082000506840F24732BCF1000F08BF1346094A36
:1008300003600A607047064B064A1968914208BF78
:100840001860704700C006406010FF1F78930100D9
:100850006C010020D400D84238B5124B5B6BDB042E
:100860001FD5114C237823B101F036FA2378002BE1
:10087000FAD10E4A0E494FF0E024002340F2031053
:100880000825C4F88451D3708860C86009490A4CAF
:100890000A4809681579D2792370037009B10123D8
:1008A0000B7038BD008004407001002000C006407D
:1008B00000C004401C0100206001002068010020ED
:1008C0000A4A38B50546137803F0FF04002BFAD125
:1008D00001212846FFF758F921462846FFF71CF961
:1008E000034A044B52F835201A6038BD70010020CD
:1008F000789301006C01002009B140F08000124A99
:100900001378834217D010B4104C646BE4040ED5F6
:1009100003F07F03082B02D10D4B0024DC6000297B
:1009200000F07F0314BF60214421082B04D0107015
:100930005DF8044B70477047054B41F44071D96036
:1009400010705DF8044B70476010FF1F008004407A
:1009500000C00440704700BF0D4B5B6B13F4805325
:1009600013D03F2803D90B4B0020186070470A4B67
:1009700010B5084C53F8303023600121FFF704F91B
:10098000236800221A70012010BD1846704700BF6E
:10099000008004401C010020789301000C4B5B6B2D
:1009A00013F4805312D00E2809D10A4B0A4A40F2A0
:1009B00002315960537B0120034353737047064A49
:1009C000537B03F0FE0300205373704718467047B3
:1009D0000080044000C0044000C00640034B5B6B35
:1009E000DB0401D5FFF718BE704700BF008004404C
:1009F00079B170B5074E04464518736BDB0404F1FA
:100A0000010403D514F8010CFFF706FEAC42F4D143
:100A100070BD70470080044010B5044C237823B1AA
:100A200001F05AF92378002BFAD110BD7001002093
:100A3000084A094B11781A789142C8B2D3B202D24F
:100A4000013B181A7047054A1268013A1344181AF4
:100A5000704700BF9C010020A40100205C10FF1F14
:100A6000064A074B11781A789142D0B23CBF054A2A
:100A70001268CBB238BF9B18181A7047600100206B
:100A8000680100205810FF1F1B4B1C491A780B7877
:100A90009A422ED010B55FFA82FE194AD8B2126877
:100AA000431C9A4219D93F2B1BD85FFA83FC154887
:100AB000C05CC0B281F800C01349096861B19E45AD
:100AC0003CBF7244D31A114A126828BFAEEB03032D
:100AD0009A4201D300230B7010BD4FF0000C634607
:100AE000E5E70B4C3F382468205C5FFA83FCC0B21A
:100AF000E0E74FF0FF307047600100206801002000
:100B00005810FF1F200100201C0100205410FF1F5F
:100B1000640100200D4A0E4B11781B789942DAB21D
:100B200011D00C490968531C994207D93F2B06D9AB
:100B3000094B3F3A1B68985CC0B270470023074AD4
:100B4000D05CC0B270474FF0FF30704760010020AA
:100B5000680100205810FF1F6401002020010020C0
:100B6000054B064A1B7806491268DBB20B700AB1C6
:100B700000231370704700BF680100201C01002093
:100B80006001002030B43A4B1A79950624D5394DCE
:100B90003949DB792A780C68D8B2531C9C42D2B20E
:100BA00031D8364B1A7802F0FF0322B100221346E7
:100BB0003349C8542A703349096869B1324A1078F8
:100BC0009842C2B28ABFA21A9B1A9B182F4A126877
:100BD0009A429CBF01230B70254AD3781C06D9B2D8
:100BE0001ED44A060DD5224B1B795B0609D5284B2E
:100BF00028491B6800220A7003B11A701C4B2C2272
:100C0000DA7030BC70471D4909789942D3D03F2B28
:100C10002CD921493F3A09688854DAB22A70CAE7C8
:100C200013791806DDD51D4B17481D7803789D42B2
:100C3000DCB208D01A4A1268631C9A4206D9272BE4
:100C40000DD8DAB204E06C23D370CAE70022134651
:100C5000144CE35CDBB2064CE3710270C1E7124A4C
:100C6000273C1568DAB22B5DDBB2F4E7DAB29FE716
:100C700000C00640600100205810FF1F68010020DE
:100C8000200100201C010020A40100205010FF1FA3
:100C90006C01002070010020640100209C010020F4
:100CA0005C10FF1F74010020A0010020094B10B44C
:100CB000186068B101F14004074B084801F11A02BD
:100CC0001A60074B046028315DF8044B19607047C7
:100CD0004024F1E7640100205410FF1F5810FF1F4B
:100CE0005010FF1F054B186018B1054B28311960D3
:100CF0007047034B28211960704700BFA0010020F6
:100D00005C10FF1F431E032B16D872B60B4951F817
:100D1000230078B130B40A4CB0F800C034F8132086
:100D2000456841F82350A2EB0C0224F8132062B668
:100D300030BC704762B67047002070473802002010
:100D400088020020013803280BD872B6074B53F8ED
:100D5000203043B100205B680130002BFBD162B62C
:100D60007047002070471846F9E700BF6002002076
:100D700010B472B61A4A1B4C042312F8011B09075F
:100D800043F0010C05D554F8331069B154F83C1008
:100D9000C9B10433142BF0D162B6134B00221A7080
:100DA0005DF8044B00F092BC0F4904EBC30208301D
:100DB00050600A780D4844F83300013A0A7062B670
:100DC0005DF8044B7047084A094904EBCC0308302E
:100DD0005860137844F83C10013B137062B6EFE79B
:100DE000A09601000000FF1F900200208800400034
:100DF000C8004000421E032A0ED81C4B400140F0A0
:100E0000100010B4034472B6194CA05C03281DD81E
:100E1000DFE800F01416031970470520A05413F002
:100E2000080F088814BFC8228822083142EA00420D
:100E300059601A6062B65DF8044B70470320EDE715
:100E400008330220EAE708330420E7E7094B53F8A8
:100E5000220038B1084B53F82200416043F82210B9
:100E600062B6E8E743F82210034BF7E70000FF1FE4
:100E70008002002060020020700200202DE9F04F67
:100E8000DFF80CA3DFF80CB385B03DE0B04D9E0851
:100E900005EBC607013A796813F00803D4B2A1F153
:100EA000080040F0B88055F836204FEA124C120C7A
:100EB00021F808CC00F0A78021F8063C41F8043C5A
:100EC000A44B53F82420002A00F00182A24B53F8CF
:100ED0002420506043F82400A04B33F8142094449D
:100EE00023F814C000F0D2FB002800F0E98117F0CD
:100EF000080F9B4B00F1080018BF5B46786045F86F
:100F0000363008238AF880309AF880305907DCB2EE
:100F10001BD5944B1B78ABB193490A7802F0FF03C1
:100F20002AB1013BDBB20B70002B00F046838F49E6
:100F30000A7802F0FF032AB1013BDBB20B70002BF1
:100F400000F0EB8104238AF8803014F0080200F0EE
:100F5000CC819AF89020D3B2120997D1DFF8F091A2
:100F60009B0809EBC30459F833006468C0F383009D
:100F700009287CD00FD80138012808D87C4A158868
:100F800042F22100854200F0FB8149F833B0012391
:100F90008AF89430B5E70D28F9D1D4E90007754DEA
:100FA00049F833B0724E744CC9F8102083B240F245
:100FB000816CC9F818202A6063454FF00102C6E928
:100FC0000007227000F2FF80B3F5D06F80F0CB8273
:100FD000B3F5817F00F0268240F2DE8040F20232DB
:100FE00093427BD107F07F07042F00F20881020CA7
:100FF00040F00581614911F8273043F0020301F800
:101000002730134670E017F0080F554B18BF5B46AA
:1010100045F8363075E700F059FB5949594A51F8FF
:101020002430002B00F05781586841F82400115DEE
:1010300003F108007860032905D8DFE801F0120FFA
:101040001502042111551A8817F0080F14BFC82380
:10105000882343EA024345F8363052E7022111550E
:10106000F1E703211155EEE705211155EBE7414D5D
:101070002A683AB34449404C0F88444894F800E049
:101080000678402F3B4628BF4023BEF1000F8EF06C
:10109000010E84F800E046F0020486F001060670B6
:1010A00009EBC400426014BFC820882040EA034016
:1010B0001A44FB1A9BB249F834000B80002B00F055
:1010C00036812A602A4B1A88B2F5A06F7FF45FAF91
:1010D0009A788AF8982000225A7058E7B3F5A06FE2
:1010E00040F08D8000221346B6F806C0274894458C
:1010F00028BF944667460278402F28BF402742F019
:10110000020E3E0409EBCE0846F0C806C8F80430CB
:1011100049F83E6000263B442670BCEB070782F08E
:101120000106067040F01181BCF13F0F4FF0010540
:1011300009D946F00206027009EBC6022570536019
:10114000882349F8363001238AF894301FE700BF1E
:101150000000FF1F38020020480200208802002003
:10116000880040008402002085020020B002002098
:10117000580200202C02002029020020C020074035
:1011800060020020800200202A02002028020020A5
:1011900000200740C8004000802B00F08B81822B8C
:1011A0002DD107F07F07042F29D8A74A00231380E9
:1011B000A64B13F827309F0740F1FC8101231370E1
:1011C000A14B022290E742F2210C6345BBD01DD90E
:1011D00042F2212293420DD1BFB2002F82D19C4B0B
:1011E0001A689C4B1A609C4BC0F307400022187091
:1011F000134679E742F2213293423FF473AF0F2353
:101200008AF8C03001238AF89430C0E6B3F5086F3D
:1012100000F04A81B3F5106FF1D1904BC0F3074055
:101220000425187059F835301A0606D40135142DE6
:101230000CD059F835301A06F8D509EBC50301353D
:101240005868083800F042FA142DF2D1844A854BD0
:101250000292854A0192854E854ADFF848820394BE
:10126000009200251C4656F8047B2FB138467F6853
:1012700000F02CFA002FF9D1009BD8F8007043F849
:10128000045B46F8045C00932FB138467F6800F099
:101290001DFA002FF9D1029B48F8045B43F8045B68
:1012A0000293019B23F8025B01932378023B032BFB
:1012B00000F20981DFE813F03F0104013F0104015E
:1012C0006C4A45F8360013780133137019E643F879
:1012D0002400674BFEE5115D022926D07FF611AE92
:1012E00003291DD1012313550BE6E0076ED4210617
:1012F00021D4A20708D5604B93F888200221D2B2EE
:1013000083F8882083F88010E30603D55A4B102217
:1013100083F8802005B0BDE8F08F00F00DFB11E6EA
:1013200017F0080F14BF032302231355E9E53F2FDD
:1013300098BF0022C5E6504B80220D2183F8C010D3
:1013400083F88020A207DFD5D5E746F002060270B9
:10135000402F09EBC6003A4628BF402243601004E4
:10136000134440F088000121BA1A49F83600217070
:1013700055D02B60414B1A8001238AF8943006E641
:1013800092885AB93E4AE51D14F8011B02F8011F64
:10139000AC42F9D13B4A1268862A3CD03A4C3B48D1
:1013A00025780278002D85F00105257042F00204B1
:1013B00082F00102027009EBC4024FF0000050609D
:1013C00014BFC822882249F83420DEE52A4B2F4872
:1013D0002F49304C022583F8945002702E480C603F
:1013E0002E4D48608C600D24CD60FF200A618A611B
:1013F00083F8C04001219F2483F8880083F880008F
:1014000083F8982083F88C0083F8844083F8941044
:1014100005B0BDE8F08F224A0F201070BEE73F2FC5
:10142000A7D890E607F07F07042F3FF6E8AE000C40
:101430007FF4E5AE054A12F8273023F0020302F8E4
:101440002730002213464FE630020020C02007401C
:101450008C000020AC020020A802002084020020A2
:101460007002002080020020880200203802002044
:101470004802002090020020002007402A0200209D
:101480009F020020A0020020290200202802002044
:101490000000FF1F88004000A8010020E801002094
:1014A0008502002060020020484B49491B780B70E0
:1014B0000B4619E6464A00231380454B022213E6E9
:1014C0004FF001032370434BB34204F101047FF456
:1014D000CAAE414E039CDFF81481404F00233370A5
:1014E000042518F8013B3E4AAB541B0725D445F0B0
:1014F000020145F0030204350023142D49F8313070
:1015000049F83230EDD1374F25783A7842F0020071
:1015100009EBC00C85F00106CCF80430002D4DD14C
:10152000882382F0010226703A7049F83030012396
:101530008AF894302BE52570C5E700F0A7F800285D
:1015400032D009EBC5030830586049F8357000F017
:101550009DF808B345F0010309EBC3020830506061
:1015600049F833B0C3E7204A5368002B3FF447AE35
:10157000000CBFB204E013690C32002B3FF43FAE05
:1015800011888142F7D15188B942F4D1000A032869
:101590000CBF1A781289A7E533780133337045F010
:1015A000010349F83300A2E7337849F835000133E5
:1015B0003370CCE7064B022296E500BE2670C823A6
:1015C00082F001063E7049F83030BCE5840200200C
:1015D00030020020480200209002002088004000D5
:1015E000C0200740280200204C960100A096010070
:1015F00010B500F04DFC00231E4A194642F8331086
:1016000002EBC3000133142B4160F7D11A481B4C85
:10161000436B43F480234363D4F80008184B40F035
:101620004070C4F80008C2F3072CC2F30744120E3E
:1016300083F89CC083F8B04083F8B420114AFF209F
:101640004FF0010C83F8800083F88800187483F849
:1016500094C011700C4983F884C0702081F8350063
:101660004FF0E0214FF400101023C1F80401137271
:1016700010BD00BF0000FF1F0080044000D00040EC
:10168000002007400021074000E400E072B60D4949
:101690000B68B3FA83F00B2810DC4FF00042C24015
:1016A00023EA02030B6062B6074A00EBC000C100E8
:1016B00002EBC000002353504360704762B6002025
:1016C000704700BF6410FF1F9803FF1F0E4BC31A23
:1016D000B3F5587F10D20D4A127872B972B60C4A1F
:1016E0000C49A2FB032308684FF000421B0922FAB1
:1016F00003F303430B6062B67047074A1278002A6F
:10170000ECD0FFF735BB00BF9803FF1F900200200D
:10171000398EE3386410FF1F8402002038B50F4C67
:10172000206878B143880288C11801339A420D7A43
:1017300002D94380284638BDFFF7C8FF0023236045
:10174000284638BD064B1B782BB10320FFF7DAFA89
:1017500020600028E6D14FF0FF35EBE7940200202F
:1017600084020020084B094A1B6810B594881BB1FD
:101770001A885B88D31A1C440CB1204610BD00F0B7
:10178000ABFA204610BD00BF940200208802002062
:101790002DE9F04FDFF8F49083B0012289F80020A2
:1017A000019179B3374FDFF8E880019D364EDFF8BD
:1017B000E4A083463868A8B3B0F802E0CEF1400C4C
:1017C000AC4528BFAC460EEB0C040022A4B232702C
:1017D000A5EB0C05448000F10802BCF1000F0AD013
:1017E0000EF1FF3E7244DC441BF8014B02F8014F3E
:1017F000DC45F9D144883F2C0BD805228AF800201B
:10180000002DD7D10198002389F8003003B0BDE83E
:10181000F08F4022028001460420FFF7EBFA0022FD
:101820003A60EAE798F8002022B34DF2E90408E0B4
:10183000013C18D03278B2B900F04EFA98F8002086
:10184000C2B10420FFF77EFA0728F1D84FF0010358
:1018500089F80030FFF71AFF38600028ACD1013C4E
:1018600089F80000E6D101234FF0FF30337003B058
:10187000BDE8F08F00234FF0FF3089F8003003B04F
:10188000BDE8F08F9C020020980200209902002001
:1018900084020020B002002038B50E4D0E4C28689E
:1018A0000123237028B140880023C0F14000237039
:1018B00038BD0A4B1B7813B90020207038BD0420B6
:1018C000FFF740FA0728F7D8FFF7E0FE2860002866
:1018D000E9D1F1E79C020020990200208402002057
:1018E000F8B5114B1B788BB1104E114D34680127A0
:1018F0002F7064B10F4B00271F706388238021462F
:101900000420FFF777FA376000232B70F8BDFFF74C
:10191000BDFE084B014620B104201C70FFF76AFA97
:10192000F2E71F70F0E700BF840200209C02002055
:1019300099020020B002002038B50E4B1B7853B935
:101940000D4C216841B103F0FF054B880B8004204A
:10195000FFF750FA256038BDFFF798FE014620B129
:10196000BDE838400420FFF745BA044B01221A7045
:1019700038BD00BF990200209C020020B002002068
:1019800070B5EFF3108272B60C4C206880B10C4E2B
:1019900000254369236073B19D6102B962B6836813
:1019A00045779847EFF3108272B620680028F0D18F
:1019B00002B962B670BD3360EFE700BFBC02002021
:1019C000B8020020FFF7DCBF024A1368013313603E
:1019D000704700BF8C000020084B10B503EB51038B
:1019E0000446B3FBF1F0FEF757F9054B1B7803B142
:1019F00010BD2046BDE8104000F082BA001C4E0E1B
:101A00009010FF1F08B50846FEF74CFB012008BDEB
:101A100008B50846FEF746FB012008BD38B5084664
:101A20000D4602F02DFA044601462846FEF7B6FBA5
:101A3000204638BD10B5084614461146FEF7AEFBE9
:101A4000204610BD08461146FEF7D6BD0846114691
:101A5000FEF7B6BDFEF7CEBC08B50846FEF7F8FAAD
:101A6000003818BF012008BD08B50846FEF7CEFAB9
:101A7000003818BF012008BD08461146FEF756BAC7
:101A80000846FEF795BA00BF0846FEF733BA00BF16
:101A9000FEF7CCB910B50648144600EB5100B0FB78
:101AA000F1F0FEF7F9F82046BDE81040FEF760B906
:101AB000001C4E0EFEF778BCFEF730BCFEF71ABCD9
:101AC000FEF7F4BBFEF7FEBB0368064A1B689342B1
:101AD00005D110B5C8B2FEF7E5FA012010BDC9B2B4
:101AE000184700BF111A01000368064A1B68934299
:101AF00005D110B5C8B2FEF7D5FA012010BDC9B2A4
:101B0000184700BF111A01000368064A1B68934278
:101B100005D110B5C8B2FEF7C5FA012010BDC9B293
:101B2000184700BF111A01000368064A1B68934258
:101B300005D110B5C8B2FEF7B5FA012010BDC9B283
:101B4000184700BF111A0100084B10B503EB5103F1
:101B50000446B3FBF1F0FEF7D5FD054B1B7803B14E
:101B600010BD2046BDE8104000F0CAB9000E27079E
:101B70009110FF1F08B50846FEF730FF012008BD91
:101B800008B50846FEF72AFF012008BD38B508460B
:101B90000D4602F075F9044601462846FEF728FF77
:101BA000204638BD10B5084614461146FEF720FF02
:101BB000204610BD08461146FFF794B80846114666
:101BC000FFF774B8FEF7CCBF08B50846FEF7E6FE8F
:101BD000003818BF012008BD08B50846FEF7BCFE56
:101BE000003818BF012008BD08461146FEF784BE24
:101BF0000846FEF7AFBE00BF0846FEF761BE00BF55
:101C0000FEF72ABE10B50648144600EB5100B0FBA3
